:020000040800F2
:10000000F8E50120255E0308255D0308275D030848
:10001000315D0308335D0308355D0308000000000F
:10002000000000000000000000000000375D030831
:10003000395D0308000000003B5D03084BA8000881
:10004000B55E0308B95E0308BD5E0308C15E030820
:10005000C55E0308C95E0308CD5E0308D15E0308D0
:10006000D55E03084B170108CB150108E15E0308B4
:10007000E55E0308E95E0308ED5E03080B21010855
:10008000F55E0308F95E03088DEE0008015F0308C2
:10009000055F0308095F03080D5F0308B7AE00089A
:1000A000155F0308195F03081D5F0308215F03083C
:1000B0009BAA0008551401082D5F0308315F03084F
:1000C000355F0308395F03083D5F0308415F03089C
:1000D000455F0308495F03084D5F0308515F03084C
:1000E000555F0308595F03085D5F0308615F0308FC
:1000F000655F0308695F03086D5F0308311F01082E
:10010000755F0308795F03087D5F0308815F03085B
:10011000855F0308895F03088D5F0308915F03080B
:10012000955F0308995F03089D5F030863B20008A9
:10013000A55F0308A95F0308AD5F0308B15F03086B
:10014000B55F0308B95F0308BD5F03083D5D0308A1
:10015000C55F0308C95F0308CD5F0308D15F0308CB
:10016000D55F0308D95F0308DD5F0308E15F03087B
:10017000E55F0308E95F0308ED5F0308F15F03082B
:10018000F55F0308F95F030830B57B4D0846144658
:1001900069892A89521A944228BF144620B16B6893
:1001A0002246C91807F052FF688920186881204646
:1001B00030BD2DE9F84F1446884660882188401AE2
:1001C000451CE088A188401A461CADB2B6B2362064
:1001D00008F0F0F8DFF8A4B19BF87801000654BFEE
:1001E0008C204C2008F0FAF86349A7880869248815
:1001F000C9682A198A18531EF2198218521E2144FE
:1002000038449BB292B289B280B208F014F95C4FC4
:10021000102138460AF0E3F95A4C012120460AF031
:10022000DEF9DFF864912C2148460AF00DFA10211E
:1002300038460AF0D2F94FF0000A16E005FB00A09C
:1002400038F81000ADF8000048469DF801100AF09B
:10025000FBF99DF8001048460AF0F6F97F1CBFB282
:100260003846B042EADB0AF1010AAA45B8BF0027C6
:10027000F5DB012120460AF0B0F9362008F09AF8A3
:100280009BF87801000654BFA820682008F0A6F863
:100290000120BDE8F28F7CB5384E374C96F86701E7
:1002A00000F00C0004F6B445082802D1374900F0EC
:1002B0005CF896F8670100F00C00042802D134497C
:1002C00000F053F896F867010C21084202D1314939
:1002D00000F04BF800F068FD18BF032807D196F82E
:1002E000E00300280CBF2C492C4900F03EF860695F
:1002F0002B4E0AF0B8FA962824D300F039F8B0F55E
:10030000967F14D300F034F8B0F5E17F1AD300F0F3
:100310002FF8B0F5167F0AD300F02AF840F2EE214C
:1003200088420FD300F024F8B0F5617F04D200209A
:1003300001904FF6FF7012E000F01AF840F21A41F7
:10034000884202D200F0B4FC09E000F011F8B0F5E8
:10035000966F09D2134900F008F800200190009030
:1003600033462A4600F0B5FC73BD28460AF098BA19
:1003700060690AF078BA000078BC01206CC90120DD
:10038000000802400004024000300140545A0308B3
:100390005C5A0308645A03086C5A0308745A030829
:1003A000343C00207C5A03082DE9F84F2DED028BD8
:1003B00084B045F255500AF08DFA02200AF08DFA09
:1003C0004FF47A700AF08CFA0AF08DFADFF820897F
:1003D00008F20D05002068760120A8764FF4A06091
:1003E0000AF08CFA0AF024FA0AF0C4FA0AF010FCB7
:1003F0000AF09EFCDFF8FC78DFF8FC68387801280A
:1004000052D101210CF0FCFA01208DF80C000020E3
:100410008DF80E001020029001208DF80F008DF84D
:100420000D0002A9DFF8D44820460AF091F8012215
:10043000102120460AF0D5F8012102200CF0E0FA44
:100440004FF48070029002A9DFF8B44820460AF009
:100450007FF801224FF4807120460AF0C2F8002094
:1004600008F00DF8C82086F87A01FA200AF006FA9A
:1004700000F01EFC00903221DFF888380FF64C1295
:10048000782008F040F838780128FCD0BFF34F8F6F
:10049000DFF87408DFF87428016801F4E0611143A3
:1004A0000160BFF34F8FFEE70CF012FB01200CF050
:1004B000D3FC00200AF0BEFC002086F8F10596F877
:1004C000000610B1002086F80006002086F8F0052E
:1004D000012086F8F70540F61C43DFF834B80FF624
:1004E0004810DFF83018CBF804000BF1980247F2FF
:1004F0002420ABF808000020ABF80A000BF1040040
:1005000000900BF118000DF068FD8BF8000020B191
:100510004FF4FC6007F0B3FFFEE70022DFF8F817A6
:100520000BF118000DF0B0FE8BF8000020B14FF475
:10053000784007F0A4FFFEE74FF6FF70019000201F
:10054000DFF8D8970FF6C80200904B46002107F05D
:10055000DAFF01240A2707FB04F0C0B20AF06AFCA4
:100560001E200AF08BF9641C192CF4DB0124C4F161
:100570001A007843C0B20AF05DFC1E200AF07EF932
:10058000641C192CF3DB00200AF054FC002007F057
:1005900076FF00200AF0ACFC142740F23F14BBB2F7
:1005A000DFF87C0700EB470A40F20312BAF8280094
:1005B0000090B9B24FF4817008F0AAF8BAF8280098
:1005C0000090BBB22246B9B24FF49F7008F0A0F879
:1005D0007F1CDC2FE3DB4FF6FF70009013232246D5
:1005E0001321002008F094F84FF6FF700090DB23F1
:1005F00022461946002008F08BF800F040FB00204E
:1006000086F87001E875287E40F0040028760EF028
:100610000BF90EF050F90EF0B3F90EF0B1FA00F04C
:1006200039FB96F88B01032804BFDFF8F8060EF0BB
:10063000DDFA0EF039FB00F027FB0CF01DF80BF093
:10064000A6FB0BF088FC0FF0DCFF0BF037FE0BF085
:100650004AFE0BF083FE0BF08EFE0BF0ACFE0BF0AF
:10066000ECFE0BF011FF0BF027FF0BF03BFF0BF044
:100670009FFF10F027F910F0F5FC10F05FFD10F06F
:1006800041FF00F09EFB4CBF0122002200F005FB61
:1006900011F003F900F0E9FA012108F1380011F036
:1006A0004DFA08F12C040AF0DBF8A06096F8790105
:1006B00000F0BF0086F8790196F87A010AF0BAFBDB
:1006C0000AE001904FF4FC6000F007FB10F003FD1E
:1006D0000BF095FD0CF0F4FF0AF005F996F879019E
:1006E00000F0C000802817D1A0680AF0BCF896F886
:1006F000791101F03F0241F288335A4382420BD212
:10070000DFF824060122027096F87A01C000A0608A
:1007100041F0400086F87901DFF81006007848B112
:100720000BF035FB0BF017FC00F044FBDFF8FC0589
:1007300000210170E87D96F87011884250D008F1D0
:10074000380011F019FA11F0B3FD11F029FD4FF442
:10075000FA700AF093F896F8700158B900F08FFA21
:10076000422100F087FA00F02CFB4CBF012200224E
:1007700000F093FA96F8700101280BD100F021FBEC
:100780004CBF0022012200F088FA00F078FA4321E1
:1007900000F070FA96F8700102280DD100F011FBFC
:1007A0004CBF0022012200F078FADFF88405C6F879
:1007B0007301442100F05EFA0BF0E9FA0BF0CBFB79
:1007C00010F0BCFC4FF07E50C6F8F305012100F09C
:1007D0004CFA08F1380011F0B1F996F87001E8759B
:1007E00096F8F175287FB84200F0948000F0D6FAB0
:1007F000000409D500F04EFA96F88B01032804BFD7
:10080000DFF820050EF0F2F996F86D0181073CD56E
:1008100000F001000CF0DAFC96F86D01C1074CBF46
:1008200000F0FE0040F0010086F86D0196F86D01C1
:1008300000F001000CF01FFC00F0BCFA00F024FAFC
:100840000BF0A5FA0BF087FB0BF038FD0BF04BFD1E
:100850000BF084FD0BF08FFD0BF0ADFD0BF0EDFD0B
:1008600096F86601072806D12821DFF8C82411FB75
:100870000020406A804700F00DFA96F88B010328AB
:1008800004BFDFF8A0040EF0B1F996F8F10550B3FB
:1008900009F0E6FFCBF814000EF00DF896F86701AA
:1008A000C00704D400F080FA18BF032806D196F8D8
:1008B000DD03C0F164010122C9B201E001228021FF
:1008C000042011F093FD0BF0B8FD00F0EAF9CFA27F
:1008D0000021BE2007F017FE687E08B900F0EDF990
:1008E00010F005FA15E001220021042011F07EFD30
:1008F0000BF0A3FD002001904B464FF6F0700090E6
:10090000D1A20021BE2007F0FEFD687E08B900F0EC
:10091000D4F92F77687E10B112F004FA01E00FF0DD
:100920004BFD0FF078FE0EF07FFB96F8F1050128E5
:1009300002BF687E002810F0E5F93078D8F82C1056
:1009400000F08DF92CD00AF0C2FB96F88B01032839
:100950001FD13078DFF8E01300F081F904D2DFF81E
:10096000C4030EF043F914E001224FF40071DFF8E4
:10097000CC0309F036FEDFF8AC030EF037F90220A5
:1009800009F07CFFDFF8B40300224FF4007109F096
:1009900028FE307806EB8000D0F80100C8F82C0063
:1009A000DBF8140009F05FFFB0F5966F05D2FFF792
:1009B00072FCDFF88C036060F9E00BF6B447307826
:1009C00094ED010A06EB4000B0F86D00010441D53A
:1009D000410447BFDB4941EA000A4FEA804A4FEA37
:1009E0009A4A8004800C00EE900AF8EEE00AB4EE19
:1009F000600AF1EE10FADFD00FFA8AFA00EE10AAC0
:100A0000B8EEC00A10EE100A17F0F6F921F0004116
:100A1000BAF1010FACBF4FF02B0A4FF02D0A0022A4
:100A2000C94B17F011FACDE9000152460FF2A83177
:100A3000384609F035FF00F034F900F049F900F0CC
:100A4000ADF98004800C00EE100AB8EEC00A84ED07
:100A5000010AACE000F0FAF8012824D1BB4890ED7F
:100A6000008AB4EE480AF1EE10FA1CD018EE100A13
:100A700017F0C2F99FED9C1A41EC100BB4EE418ABD
:100A8000F1EE10FA53EC102B4CBF0FF254310FF271
:100A90005831384609F004FF00F0DDF800F014F991
:100AA000AA480068606000F0D1F8022836D1A84852
:100AB000006817F0F7FACDE90001A648006817F0C2
:100AC000F1FAA54B002217F0BFF902460B46DDE90B
:100AD000000117F0B9F917F0F3FAC0B26528A8BF02
:100AE0006420E876EA7ED4ED010A00EE102AB8EE22
:100AF000400AF4EE400AF1EE10FA0FD00FF2F021A6
:100B0000384609F0CDFE00F0A6F800F0DDF8E87EEA
:100B100000EE100AB8EE400A84ED010A00F096F8E3
:100B2000032844D18D48816900EE101A8169B5EE21
:100B3000400A00EE101AF1EE10FA10EE100A07D576
:100B400017F05AF921F0004302460FF2AC2106E0FB
:100B500017F052F921F0004302460FF2A421384663
:100B600009F09EFE00F077F87D4B00900021019186
:100B70003A46CA21D02007F0C6FC7848C16900EE89
:100B8000101A10EE100A17F037F902460B460FF252
:100B90007821384609F084FE00F05DF800210191CB
:100BA00000903A466E4BCA21C72007F0ACFC697E24
:100BB000A87E002904BF96F8F115002903D0009003
:100BC0003C23402229E03178891991F8A3100829A3
:100BD00018BF07291CD1009018232E224A2100207B
:100BE0000AF054FB00F0D2F85E4A382007F08BFC84
:100BF00000F0CCF85C4A262007F085FC00F0C6F82F
:100C00005A4A142007F07FFC0BE000BF5458000044
:100C100096F887310090C3F17C02142100200AF07D
:100C200035FB0FF0B9FE96F81B0200060BD55048B5
:100C3000007800283FF445AD00F03AF800F04DF898
:100C40004B480021017041E55258000096F87801A8
:100C500000F00300704798F80D000BF05EBD06EB46
:100C60008000D0F80100884270474248424B434A16
:100C700000907047424881725721C17270474BF60D
:100C80008030C6F87301704796F86D0100F00100DE
:100C90000BF0D0BC3B480DF0A9BF02213A4809F047
:100CA000A0BC002001904B464FF478400090704764
:100CB000002001904FF478407047009091234FF44A
:100CC0008072142107F094BD0021019100904B46E1
:100CD0003A46CA21C82007F016BC009003A2204B58
:100CE0000021CF2007F00FBC00007A4453514C0084
:100CF000A43100200C3A00206CC901200000024001
:100D0000000402403C3C00200CED00E00400FA0529
:100D100078BC012089010008B3010008343C0020A0
:100D200074CF012009AC0108013A0020C420002042
:100D30000077010084070108007E56030008024086
:100D4000000080BF00C0FFFF00408F40C4DC0120D6
:100D50006C3C0020E0DC012000005940343B0020C6
:100D60002C3C0020683A0020D8DB0120F0DB012079
:100D7000A0DC0120EC3B00205C3B0020D03B0020AD
:100D8000083C0020BFEB000800100240002001904A
:100D90004B464FF6FF70009000217047307806EB0D
:100DA0004000B0F86D0070473078801990F8A300CB
:100DB00002287047307806EB8000D0F801000AF076
:100DC00086B996F8670180067047000044465520B2
:100DD0004D4F444500000000256325342E32660047
:100DE00025352E316600000025352E3066000000C6
:100DF0002025336425250000702D25362E3466000D
:100E0000702025362E3466006D2025362E3466007F
:100E100056657220342E35205541432043444320EB
:100E20006279205233444900FFD8FFE000104A465F
:100E3000494600010101004800480000FFE10E841E
:100E40004578696600004D4D002A00000008000743
:100E5000011200030000000100010000011A00055A
:100E60000000000100000062011B000500000001FD
:100E70000000006A012800030000000100020000D9
:100E8000013100020000001C00000072013200026B
:100E9000000000140000008E8769000400000001BB
:100EA000000000A2000000CE000AFC800000271015
:100EB000000AFC800000271041646F6265205068C2
:100EC0006F746F73686F70204353352057696E6479
:100ED0006F777300323031373A30373A313220325F
:100EE000313A32393A3430000003A00100030000E7
:100EF000000100010000A002000400000001000049
:100F00000140A003000400000001000000F0000008
:100F100000000000000601030003000000010006BD
:100F20000000011A0005000000010000011C011B67
:100F3000000500000001000001240128000300005A
:100F40000001000200000201000400000001000096
:100F5000012C020200040000000100000D4F0000FF
:100F600000000000004800000001000000480000F0
:100F70000001FFD8FFDB004300080606070605084E
:100F80000707070909080A0C140D0C0B0B0C1912A2
:100F9000130F141D1A1F1E1D1A1C1C20242E27207F
:100FA000222C231C1C2837292C30313434341F27A1
:100FB000393D38323C2E333432FFDB00430109091E
:100FC000090C0B0C180D0D1832211C213232323253
:100FD00032323232323232323232323232323232F1
:100FE00032323232323232323232323232323232E1
:100FF0003232323232323232323232323232FFC076
:10100000001108007800A003012100021101031162
:1010100001FFC4001F0000010501010101010100E1
:101020000000000000000001020304050607080993
:101030000A0BFFC400B510000201030302040305FC
:101040000504040000017D010203000411051221C2
:1010500031410613516107227114328191A1082395
:1010600042B1C11552D1F02433627282090A1617B7
:1010700018191A25262728292A3435363738393AB7
:10108000434445464748494A535455565758595A78
:10109000636465666768696A737475767778797A68
:1010A000838485868788898A929394959697989960
:1010B0009AA2A3A4A5A6A7A8A9AAB2B3B4B5B6B785
:1010C000B8B9BAC2C3C4C5C6C7C8C9CAD2D3D4D5B1
:1010D000D6D7D8D9DAE1E2E3E4E5E6E7E8E9EAF1F0
:1010E000F2F3F4F5F6F7F8F9FAFFC4001F01000374
:1010F00001010101010101010100000000000001E6
:1011000002030405060708090A0BFFC400B5110015
:10111000020102040403040705040400010277002D
:1011200001020311040521310612415107617113B7
:1011300022328108144291A1B1C109233352F01522
:101140006272D10A162434E125F11718191A2627DC
:1011500028292A35363738393A43444546474849DD
:101160004A535455565758595A63646566676869B7
:101170006A737475767778797A82838485868788AE
:10118000898A92939495969798999AA2A3A4A5A6D2
:10119000A7A8A9AAB2B3B4B5B6B7B8B9BAC2C3C4FE
:1011A000C5C6C7C8C9CAD2D3D4D5D6D7D8D9DAE22A
:1011B000E3E4E5E6E7E8E9EAF2F3F4F5F6F7F8F94F
:1011C000FAFFDA000C03010002110311003F00F7DF
:1011D000FA2800A2800A2800A2800A2800A2800A19
:1011E0002800A2800A2800A2800A2800A2800A28DB
:1011F00000A2800A2800A2800A2800A2800A2800F3
:10120000A2800A2800A2800A2800A2800A2800A240
:10121000800A2800A2800A2800A2800A2800A28052
:101220000A2800A2800A2800A2800AE5B55F88DEAD
:1012300013D0F53974DD4F5986D6F22203C5223812
:10124000232011CEDC630473401D3A3AC881D08656
:101250005619041C8229D400514005140051401C29
:10126000B6B9E3BD2BC37E27D3B46D59BECC9A84E7
:1012700045A1BA76C461C1C6D6FEEF51CF4F5C56C8
:101280005FC49F1DEABE03B3B6D42DB448F50D3E2E
:1012900053B2597CF28627ED91B4F04743EA31DC32
:1012A000500725A87C75B8B0F16C1A27F6142E9259
:1012B000B5B0F3BED44604A88DD36F6DFF00A55919
:1012C000D0BE35DC6AFF001093C2F26871C486E6B6
:1012D000580CEB7058FC81B90BB475DBEB4019B6B8
:1012E0007FB414DA8C5AABDB78750359C1F688A346
:1012F0007BA3BA540EA1BF878215B77D14D322F801
:10130000FF00A85C787EE35683C330BADA4EB1DCC6
:10131000A7DACE63571F23FDCE848607D0EDF5A054
:1013200005D67F682B9D2A6B444F0F4330B8B38698
:10133000E726E88DA5D0315FBBD892335B3ACFC6A4
:10134000B4D33C7917869748531B3451B5DCB39519
:1013500001A45520EDDBF746E1939E99340195A455
:10136000FC77D5757D4EE34B8BC2D12EA091C8D1B1
:10137000406ECE6474E5A3FB9C36D0D8F5200EF405
:10138000C9BE3FDDC5E17B5D67FE11C84F9F7B3560
:10139000A98BED67E5F2D226073B7BF9847E1EF42C
:1013A00000BAB7ED0175A65968F70BE1E864FED104
:1013B000B2FB5106E88D87CE923DBF779FF579CF7E
:1013C000BD27C6AF0F5BF88FC23A3F8AA0458B544A
:1013D0006857F7639F3A331994AE7B95019874E090
:1013E000377C0A00BDF033C78FAD787A4F0DDD48EA
:1013F000ADA969D166D4C8D8F361E801FF0074E0F3
:101400007D08F4354F4FF8F97D7BA85EE9F2F86A64
:10141000282F20826748CDD93BE48C16643F2F07E4
:101420006ABE3DC01DE8023B4FDA0AE6F346D46FC0
:1014300053C3B0F9D62627687ED6798989567CEDC4
:10144000ECC631FF0003F6AF41F869E3F8FE20680F
:101450007717A6D56D2E6DE7F2A48049BF0300ABC8
:10146000670383C8FC0D0076B4500145007CFF0083
:10147000FB4C43CF866603FE7E509FFBF447F5ADE1
:101480005F839E20B4F1BF81AF7C1DAE62E24B58FA
:10149000BCBDAE7264B73D08F743819EDF2D007975
:1014A000A7C4BD266D03E2DC29223F9016CBC89568
:1014B000971E6AA471A161FF0002461F855BD1EDF2
:1014C00027D2FF00690582E2268DFF00B625650C54
:1014D000319472C54FD0AB03F8D00749E3BF0FF882
:1014E0002BC17F126C6E65B8D46C93500F25CC3035
:1014F000C0B240B1C9BA39075054302D900363B01F
:10150000E82B8CF87AB0689F1326F0D6ABB67D3BFB
:1015100052F334AB8C7DD9031FDDB2FD582107FD9A
:10152000AC8A00A7F153C3F27863C4F69A4BB9951D
:101530006DEC2244948C6F505803F90E7DF35EA538
:10154000F163C2DE1A93C23A5F8AB5292FADEF4C20
:10155000305BF99668AE65CA646E0C40C800F391C2
:10156000E9CF1800F2BF116A11E93E39D3BC57A385
:101570005C35C437262BF49593CB2D2A9C4A1972DF
:101580007692EAC48C9E18750413DE7C66F0E59CA6
:101590001E11B0D774481BFB3B50BE6BF90A8F96E7
:1015A000233451E3E81B667EA71E9401E73E24B373
:1015B0009CF827C1BA8188FD9DACEE2DC48071BD19
:1015C0006EA56C67E8E0D7B2FC4A9E78BE05F85776
:1015D00051B691A3B8B66B1B88E41D55BC9383F933
:1015E0009A00F198F529BC37AF699E2ED054430C70
:1015F000921916204ED8A41FEB603FECE1B8FF0013
:1016000061D7BE6B4FC717B6F67E3DB2F1868AA092
:10161000D9EA5E5EA70A9E824DD89636F7DEAD9176
:10162000FED7BD0050821B2D1BC7D2D897DBA3DF8E
:10163000830876ED6D70998DCFBA8747FAAD759FA7
:10164000033579BC37F126E741BDCC5F6E57B691C3
:1016500009C6D9E324AE7F275FAB5007D47450018D
:1016600045007867ED2A99D174093FBB7128FCD4F5
:101670007F85788F833C4D71E10F1558EB36F9610A
:101680000BE258C1FF005919E197F2E9EF83401FBF
:101690005A7887C27E1DF893A3E9D71766478576E7
:1016A000DCDADCDBB057DAC33D483C1E323D855600
:1016B000F1AFC3CB3F135D43AD5ACF3D97882CA20A
:1016C0006FB1DD40E172E394DF907201FD09A00E7D
:1016D0004B4997C39F1B3474B0F125B3DA788B4A1A
:1016E00025678E17F2E45E70CCB9072A48E41CED3A
:1016F0003F813B56BF057C396DE2DB7F107DA6FD47
:10170000E4B678E486DD9D7CB531801070B9206D3B
:101710005EFCE39CD006FF008D3E1EE87E3B86D536
:1017200035759D5ED9898E6B760AE01EAB920F1DD2
:101730000FE15A3A8F85B4AD5FC303C3DA8406E282
:10174000C0429100C70C3681B5811D186073401CE2
:101750001DE7C02F0C5D59D959ADFEA90DBDA97665
:101760000AB2212E5C82C4929D70147A71F5CFA0CA
:101770004BE1CD326F0C8F0ECB6E1F4C16C2D7CA09
:10178000639FDD850A39F5181CFA8CD00610F863C2
:10179000E1F3E045F07CA2E65D351CC91BC8E0CB57
:1017A0001B162D956C601E48E9D09156B57F01E956
:1017B0003AD782ED7C2B7525D0D3EDA38A3468DC33
:1017C0000931180172718EDCF1401CC43F023C27C4
:1017D0000E9D75602E3547B7B82AE55E743B1D4FE8
:1017E0000EBF27070597D30C7D886B7C06F0A3E915
:1017F00091E9EF77AB35BC72B4D1833A6519800DAE
:101800008F93A1DAB9FF00747BE401D7BF023C27B4
:101810007F0D9473DC6A87EC907908E274DCC9B9B7
:10182000986EF939237103D801DAB4AD3E10F86A25
:10183000D3C590F89035F4B7F13ACA3CC946C69082
:101840000037901412491B8F38C93C76A00EF68AD7
:101850000028A00F12FDA4D73E1AD15FD2F187E66F
:101860009FFD6AF9BD36EF1B812B9E71D71401F5E0
:1018700077C1AF11F86E6F0B5BE89A5EAF7135CC34
:10188000259BEC97E55668C1E485C70CA0E4E467A6
:1018900019E71D2BD324904513484310A0921549F6
:1018A00027E8075A00F947E23EB16DA17C566D7FEB
:1018B000C2B7934174489A78E4B692068A6E8E193C
:1018C000645190C393EBB8D7A9F833E3DE87AD79C1
:1018D000769AFA0D26F4F1E6939B773FEF754FF871
:1018E000171EF401EAD6F7D6976A1ADEE6198119AF
:1018F00006390367F2AB140051400514005140054E
:1019000014005140051401E15FB466AFA6CFA258A0
:101910006951DE42DA941782592D8365D10C6DC965
:101920001DBA8FCEBE75A009219E5B69926824788E
:10193000A5460C8E8C55948E8411D0D7B1F83BE31C
:10194000FEA9A6C2B63E2489F50B7C6D5BC8B02704
:101950004F720F0F8F7C1F526803BAF0BEBDE12F8C
:101960008C1E1D8ACBC4D6B64DAD4036491B36C938
:101970000FFB7130C360F520743C1ED92F3F675FA9
:10198000094F206B7BDD56D867945951863DB2B91B
:10199000FD68026B6FD9E7C1707FAD9755B8FF0046
:1019A000AE970A3FF415156EF7E06785DED047A5C0
:1019B0005C6A7A54EBD25B7BA66C9FF68313FA6267
:1019C0008020F0C5AEB9F0C2EE3D375FD546A9A084
:1019D0005FCFE5DBDFB6E0D6B31E8B2024ED47E812
:1019E0000E480DE99AF54A0028A0028A0028A002B4
:1019F0008A0028A00F32F8C1F0E478CB43FB7E9F29
:101A000010FEDAB14262C759D3A98CFBF75F7E3B67
:101A1000D7C9CCAC8C558156070411C834009450FA
:101A2000028241C8E08AF53F863F162FFC3FAC4555
:101A30006DE20D5EFEE346285044504E51BF848255
:101A40004EE503D067E9401F535BCF1DD5BC73C47F
:101A5000498E540E84823208C8E0F22A5A00E77C8C
:101A60006DA76A1ADF856EB4AD32DECA692F97C8DA
:101A700076BC63E5C487ABE002588EC38E707B559D
:101A8000DF0DE9B79A3F87ACB4EBED45F51B8B78DA
:101A9000C46D74E9B4BE3A6464F41C673938E680F6
:101AA0003568A0028A0028A0028A0028A002BE652C
:101AB000F8F3E0C8B4DF102EBBA6D95CAC3760BD2C
:101AC000E32404C2B27F7B70E016EE0E39E79CD0AF
:101AD000078D5140057D3BF067E1CE8761A1D87845
:101AE000ACC8351D42EA21244EC985B63D19547F44
:101AF0007810416F6E31CE403A5F10EA1E24B00379
:101B000052D4E5B6D3F47B5937B45A74A66B8BD64E
:101B1000242C508DD1AED2CC79209CF0063935B32F
:101B2000A668B79A86DD43C492096E5FE65D3D1BE9
:101B300036D6C3B2E3A48E3BBB679FBA14500746A8
:101B400006296800A2800A2800A2800A2800A28034
:101B50000A6BA2C8851C065618208C822803CD3C2F
:101B60005BF03FC2DE22F327B18CE917CDCF996A33
:101B7000A3CB27FDA8FA7FDF3B6BE76F1BF80B5762
:101B8000F01EA71DA6A5E5CB14CA5A0B8873B24058
:101B90000F2391C11C647B8A00E5ABD1FE1AEBDFF9
:101BA00011ADD8D8F8463B8BCB504EE8258C3C1174
:101BB00093DF736027AF519F7A00F5CD2BE18F8AB9
:101BC00035AD56CF59F1C78AEE269AD664B886CA83
:101BD000C8E238DD4E41E814720745FC6BD7280097
:101BE000A2800A2800A2800A2800A2800A2800A257
:101BF000800AE67C77E0FB4F1BF85EE34AB9DA9394
:101C00007FACB69C8C98A51D0FD3B1F626803E48BC
:101C1000D33C21A85EF8D0785E789A0D437C91146D
:101C20003D9D5188FC381CFA735F437ECF70DC43C6
:101C3000F0EAE04E1867519762B755015011FF0066
:101C40007D06A00F57A2800A2800A2800A2800A2C1
:101C5000800A2800A2800A2800A280390D4BC0D635
:101C6000973F11347F1841B63BBB45923B95C7FA6D
:101C7000E531B2A9FF007816C7D3E82BA0D2348B88
:101C80005D16D24B6B44DB1C9712DC118FE291CBBB
:101C90009FD5B1F414017E8A0028A0028A0028A0F2
:101CA000028A0028A0028A0028A0028A0028A00236
:101CB0008A0028A0028A0028A0028A0028A00FFF1C
:101CC000D900FFED179250686F746F73686F7020C2
:101CD000332E30003842494D04250000000000102A
:101CE00000000000000000000000000000000000F4
:101CF0003842494D043A00000000009300000010F3
:101D00000000000100000000000B7072696E744F4B
:101D100075747075740000000500000000436C725B
:101D200053656E756D00000000436C725300000037
:101D3000005247424300000000496E7465656E75AD
:101D40006D00000000496E746500000000436C7275
:101D50006D000000004D70426C626F6F6C010000FE
:101D6000000F7072696E745369787465656E4269AC
:101D700074626F6F6C000000000B7072696E7465A6
:101D8000724E616D6554455854000000010000001A
:101D90003842494D043B0000000001B20000001031
:101DA000000000010000000000127072696E744FA4
:101DB00075747075744F7074696F6E7300000012E3
:101DC000000000004370746E626F6F6C00000000D2
:101DD00000436C6272626F6F6C000000000052671B
:101DE000734D626F6F6C000000000043726E4362BF
:101DF0006F6F6C0000000000436E7443626F6F6C85
:101E000000000000004C626C73626F6F6C00000099
:101E100000004E677476626F6F6C00000000004532
:101E20006D6C44626F6F6C0000000000496E74724C
:101E3000626F6F6C000000000042636B674F626A64
:101E40006300000001000000000000524742430010
:101E50000000030000000052642020646F7562409F
:101E60006FE000000000000000000047726E206478
:101E70006F7562406FE0000000000000000000424B
:101E80006C2020646F7562406FE00000000000006D
:101E900000000042726454556E744623526C740004
:101EA0000000000000000000000000426C642055AB
:101EB0006E744623526C74000000000000000000A5
:101EC00000000052736C74556E74462350786C4059
:101ED000520000000000000000000A766563746F85
:101EE0007244617461626F6F6C01000000005067A2
:101EF0005073656E756D00000000506750730000F0
:101F0000000050675043000000004C656674556E39
:101F1000744623526C7400000000000000000000B2
:101F20000000546F7020556E744623526C7400008C
:101F30000000000000000000000053636C20556E9C
:101F4000744623507263405900000000000038427C
:101F5000494D03ED000000000010004800000001A2
:101F6000000200480000000100023842494D0426EA
:101F700000000000000E0000000000000000000053
:101F80003F8000003842494D040D0000000000046D
:101F9000000000783842494D041900000000000498
:101FA0000000001E3842494D03F300000000000904
:101FB000000000000000000001003842494D2710D9
:101FC00000000000000A0001000000000000000204
:101FD0003842494D03F5000000000048002F6666B6
:101FE0000001006C66660006000000000001002F82
:101FF0006666000100A1999A000600000000000139
:10200000003200000001005A00000006000000003D
:102010000001003500000001002D00000006000056
:10202000000000013842494D03F800000000007034
:102030000000FFFFFFFFFFFFFFFFFFFFFFFFFFFFAE
:10204000FFFFFFFFFFFFFFFF03E800000000FFFFAF
:10205000FFFFFFFFFFFFFFFFFFFFFFFFFFFFFFFF90
:10206000FFFFFFFF03E800000000FFFFFFFFFFFF8F
:10207000FFFFFFFFFFFFFFFFFFFFFFFFFFFFFFFF70
:1020800003E800000000FFFFFFFFFFFFFFFFFFFF6F
:10209000FFFFFFFFFFFFFFFFFFFFFFFF03E8000061
:1020A0003842494D0400000000000002000638429A
:1020B000494D040200000000000E00000000000076
:1020C00000000000000000003842494D04300000CC
:1020D0000000000701010101010101003842494DE2
:1020E000042D000000000006000100000006384238
:1020F000494D04080000000000100000000100002D
:10210000024000000240000000003842494D041E19
:10211000000000000004000000003842494D041A8D
:10212000000000000349000000060000000000005D
:102130000000000000F0000001400000000A00550F
:10214000006E007400690074006C00650064002D6E
:10215000003100000001000000000000000000004D
:10216000000000000000000000010000000000006E
:10217000000000000140000000F00000000000002E
:10218000000000000000000000000100000000004E
:10219000000000000000000000000000000010002F
:1021A0000000010000000000006E756C6C00000073
:1021B0000200000006626F756E64734F626A63000E
:1021C00000000100000000000052637431000000B4
:1021D0000400000000546F70206C6F6E67000000F8
:1021E00000000000004C6566746C6F6E67000000B4
:1021F000000000000042746F6D6C6F6E670000009D
:10220000F000000000526768746C6F6E6700000198
:102210004000000006736C69636573566C4C730074
:102220000000014F626A630000000100000000002E
:1022300005736C6963650000001200000007736C91
:1022400069636549446C6F6E670000000000000020
:102250000767726F757049446C6F6E67000000000D
:10226000000000066F726967696E656E756D00002B
:10227000000C45536C6963654F726967696E0000B5
:10228000000D6175746F47656E65726174656400F9
:1022900000000054797065656E756D0000000A4598
:1022A000536C6963655479706500000000496D677F
:1022B0002000000006626F756E64734F626A6300EF
:1022C00000000100000000000052637431000000B3
:1022D0000400000000546F70206C6F6E67000000F7
:1022E00000000000004C6566746C6F6E67000000B3
:1022F000000000000042746F6D6C6F6E670000009C
:10230000F000000000526768746C6F6E6700000197
:10231000400000000375726C5445585400000001E1
:102320000000000000006E756C6C544558540000AD
:1023300000010000000000004D73676554455854CB
:1023400000000001000000000006616C7454616729
:10235000544558540000000100000000000E636561
:102360006C6C54657874497348544D4C626F6F6C53
:10237000010000000863656C6C546578745445581E
:102380005400000001000000000009686F727A41EB
:102390006C69676E656E756D0000000F45536C6962
:1023A0006365486F727A416C69676E00000007646C
:1023B000656661756C740000000976657274416C25
:1023C00069676E656E756D0000000F45536C69633B
:1023D0006556657274416C69676E0000000764653C
:1023E0006661756C740000000B6267436F6C6F72FE
:1023F00054797065656E756D0000001145536C6908
:1024000063654247436F6C6F7254797065000000DA
:10241000004E6F6E6500000009746F704F75747325
:1024200065746C6F6E67000000000000000A6C6548
:1024300066744F75747365746C6F6E67000000008E
:102440000000000C626F74746F6D4F757473657467
:102450006C6F6E67000000000000000B7269676817
:10246000744F75747365746C6F6E670000000000C4
:102470003842494D042800000000000C0000000212
:102480003FF00000000000003842494D04140000F5
:1024900000000004000000093842494D040C00000F
:1024A00000000F3C00000001000000A000000078C8
:1024B000000001E00000E10000000F200018000112
:1024C000FFD8FFED000C41646F62655F434D000172
:1024D000FFEE000E41646F62650064800000000141
:1024E000FFDB0084000C08080809080C09090C111E
:1024F0000B0A0B11150F0C0C0F15181313151313D2
:1025000018110C0C0C0C0C0C110C0C0C0C0C0C0CF5
:102510000C0C0C0C0C0C0C0C0C0C0C0C0C0C0C0CFB
:102520000C0C0C0C0C010D0B0B0D0E0D100E0E10E7
:10253000140E0E0E14140E0E0E0E14110C0C0C0CA8
:102540000C11110C0C0C0C0C0C110C0C0C0C0C0CBC
:102550000C0C0C0C0C0C0C0C0C0C0C0C0C0C0C0CBB
:102560000C0C0C0C0C0CFFC0001108007800A00330
:10257000012200021101031101FFDD0004000AFF26
:10258000C4013F000001050101010101010000003B
:1025900000000000030001020405060708090A0BF9
:1025A000010001050101010101010000000000001E
:1025B00000010002030405060708090A0B100001C8
:1025C0000401030204020507060805030C33010099
:1025D000021103042112310541516113227181322C
:1025E000061491A1B14223241552C1623334728280
:1025F000D14307259253F0E1F163733516A2B283FC
:10260000264493546445C2A3743617D255E265F24A
:10261000B384C3D375E3F3462794A485B495C4D497
:10262000E4F4A5B5C5D5E5F55666768696A6B6C694
:10263000D6E6F637475767778797A7B7C7D7E7F73D
:10264000110002020102040403040506070706053F
:10265000350100021103213112044151617122132D
:102660000532819114A1B14223C152D1F0332462C9
:10267000E1728292435315637334F1250616A2B2B8
:1026800083072635C2D2449354A317644555367444
:1026900065E2F2B384C3D375E3F34694A485B4959D
:1026A000C4D4E4F4A5B5C5D5E5F55666768696A6F8
:1026B000B6C6D6E6F62737475767778797A7B7C7CF
:1026C000FFDA000C03010002110311003F00F55472
:1026D000924925292492494A49249252925CFE77D4
:1026E000D6CA28FADBD37EACE3ECB6FCA16D998E9A
:1026F000924D4C6536DF4321BFE1AF7D7BFDFF008E
:10270000428FF07FAC5562D6E9DD468EA343EFA33E
:10271000E85775D8E663E95163F19E74FCD73AAD8A
:10272000ECFE424A6D249249294924924A52492496
:102730009294924924A5249249294924924A7FFFE0
:10274000D0F5549249252924931200249803524A23
:102750004A5D637D6CFAC98BF56BA2DDD4AF1BECCF
:102760001FA3C6A7BD97381F4D9DBD9A7A96FF003F
:10277000C131EB17EB0FF8D5FAB5D203AAC47FED40
:102780005CB1C578E47A40E9FCE65FBABFFB63ED73
:102790000BC8BEB57D6DEA9F5A7359959FB58CA540
:1027A000A598F8F5C8AD8099711BDCEFD2D9EDF58D
:1027B0006CFCF494B74BFACF9B87F5907D62C9719E
:1027C000CACD0EB6C739D03759657654D98F6B6BE1
:1027D0006BACFE6D9FE0BF475AF55FF13565EFFAD0
:1027E000A777AB240CDB4564F769650F719FCEFDBD
:1027F0002BAD5E22BB0FA8DD1FEBFDCEFB5FD5B777
:10280000D9878CE2776458ED98EF73439BAD360B14
:102810001995B7F9BF6D177A4FFF0046929F7A4915
:1028200070381F5F3EB274ECEC6E97F5B7A2D94DCD
:10283000B956328A333140756FB2C2D654CFA6FA38
:102840001EFF00CEB3D1CAFF00D065DF24A52492BD
:1028500049294924924A5249249294924924A52410
:10286000924929FFD1F5549249252978BFF8DDFA1C
:10287000C95E6757FD9383936BAAC56ECCD636D3DA
:10288000E83AD0777A7F6767E8DD6E3FF85B1FBF75
:10289000F49FA1FD17A0BB6FF193F5D47D5CE9A374
:1028A0001309CD3D5739A455AEB557F45F965A3F3D
:1028B0003BF331B77F85F7FE93D0B2A5E0E4926495
:1028C000EA4A4A5249249294BDABFC58FD74E8B9D7
:1028D0007D371BEAF0AC74FCDC4AC32AADCE96DE31
:1028E0006375D752F21BFA7B2EF52EB31BF97FA22C
:1028F000F5BF4BE978AAEDFEA2FF008BCCEEADD47C
:1029000019775AC0C8ABA4EDDDEA39C282E3ED7D88
:102910006057631D7DF4DCDF67E87D1FDFFB4FFA46
:1029200044A7D27ABE27D62C868C1EA6C667F4ACE6
:10293000970659774F6BB1F2B19CD7B6CC1EA35E08
:10294000FC9BBD7751731AFC9AEAAD9E97E8EDABFC
:10295000ED35FAF42BD85D672B01DF61FAC405373A
:1029600031C194F53036E2E4823D96178FD1E065AF
:102970003BE8598993E9FE9BFA159915AD8C7A2AA3
:10298000C6A2BC7A416D54B1B5D6092E21AD1B1A31
:1029900037BCB9EEF68FCF53E742929749637D6B10
:1029A000CEEA1D33A25DD4BA7DD8F4BF047AD63303
:1029B00024135DB5B4383B1B731CC7D5759B99F6C2
:1029C0007DBF4EEF4E8FF0AADF45CECBEA1D2F1F05
:1029D00037370DDD3EFBDBBDD88F76F730127D3DFE
:1029E000EEDB5FB9F5EDB366CDF5FF003767E912B1
:1029F00053792492494A4924925292492494A492A8
:102A000049253FFFD2F5549249253E65FE3A3A6783
:102A10004DABA663F52AF1AB6750BF2995DB92D188
:102A20000F731B55BEC7BBF3FE855FE62F225EC347
:102A3000FE3B9D1D1BA733C725C7EE61FF00C92FB5
:102A40001E11237683B91A98494CAAAACBAC6555B6
:102A500031D659638358C682E739CE3B5AC635BE54
:102A6000E739CE5E85F567FC50752CCADB99D79E99
:102A7000EC2A08DCDC3AF69C97889DAE73FF004395
:102A80008BF9BFCE7A967E65B5D0BB2FF169D1BEEA
:102A9000ADD7D1D9D5BA5E0DB5D971735B979BB15E
:102AA000D7BDAD258E7D5E939ECA29DDBEAD8CF46B
:102AB0007D4F4BF4BEAFE8ED5D958C1656EAC92DFF
:102AC0000F05A5CD25AE12225AE1F45C929E0FA00F
:102AD000748FAADFE2F7A55799D76EA59D5F21A154
:102AE000F658F02CB5A7FEE360D4CF52DF4AADDB39
:102AF0006DB6BFE75FFA4BACF4BD1652D91FE3A326
:102B0000EAB56FDB563E65E244BC32B6B63F93EAA7
:102B10005CD7FF00D05C37D77E9F89D4BEBB1E8DAB
:102B2000F5771DF7648229BAD75D6DEFB6F89B9DE6
:102B300065D956DFB6BC567E8ACFF45E8DFEA2EE16
:102B40007EAC7F8A2E8DD37664F5970EA79620FAF9
:102B500044463B0FB4FF0035F4B276BB77F3FF0079
:102B6000A2B19FF6952524A3FC72FD51B4C3EBCC12
:102B7000A078D95308FF00C06EB51F2FFC6C7D599B
:102B80006521DD39B93D4EF74C53452F6ED3DBD56A
:102B90007DE2BFFC0BD65D8538F450D0CA2B654D65
:102BA000020358D0D103FAA88929E1FA0E4759FA4D
:102BB000ED7373BAD611E9DD130AD1663609DDBBB0
:102BC00023219F42CCAB2C6D6EBB170DDF42B65557
:102BD0004D36E4FF003BEB7D9FD35DC24924A52425
:102BE0009249294924924A5249249294924924A70D
:102BF000FFD3F5549249253E63FE3C1F181D2ABFA2
:102C0000DEB6D77F9AD60FFBFAF37FAB3D0723EBF7
:102C1000075BC6E974CB45CE9BAC027654DF75D614
:102C2000FF00659F43F7EDD95AF40FF1E6ED7A2BDB
:102C300067FEE5123FF61615EFF169D1F13EACFDE6
:102C400059C9FAD5D588A5F955FA81CE10598CDD28
:102C50006A6B3735AEF5336CFD2358C7FEB1FA9772
:102C6000F84494F53D7BEB2742FA99D3711992D73A
:102C7000B69F6E3E26350039FB2B686FB5B6D95F1F
:102C8000E8A967A6D7BF7FFA343FAD1F5CB1BA266B
:102C9000455D2A8A6CCBEB39D5B8E163D4D0E6EF39
:102CA0003FA3C6FB4EEB29D94D977EE7E6556AF266
:102CB0007FAEB9F7758FAF353EDDCCAEC6E08A6921
:102CC00071135B2EAA8C97532DF6FB6DC9B55BC0B3
:102CD000B6ECAFF1C0E75CF2F7B7A9DEC0E76A7601
:102CE000546DAEA67F629A995B1253D760D7F57B7D
:102CF000FC59F4F6E6F5AB1F99D77A9C9C8B6B1EBA
:102D0000A5AFD5AFBAAA3D5757B71EB7B9AEB6DB18
:102D10006C63F2ADFD27FA1A68D4ABFC66F407F5D4
:102D2000EA7A21AB21B6653AA6E3E416B4D4EFB44F
:102D30003596E23FDB61B98CC865D4EDDF4EFAFD14
:102D40004FD3D74FE91729F5A7AA7D4CFACDF5C384
:102D50001A87D59197F629AB2726BB9B4E29A28FC0
:102D6000533331FAD76DD757454323DF43F1BD7F46
:102D7000F016FF00317AE77EA8594F56FAE76FD672
:102D80000EA85B461601B3A9E49976DAC567F55A31
:102D9000A9FA4EFD15EFC765147FA3ABD2AD253E52
:102DA000BDF5A7EB9747FAAD550FEA3EAD8FC97356
:102DB0008554D0D6B9E4344BEC3EA3EA67A6DDCC0B
:102DC00067D3FF0009FD756F33AFF4CC1E8A3ADE7E
:102DD00065869C235B2D05C25F1606FA55FA6DDDEC
:102DE000FA476F5E21FE313A9DBD5BAB61F52B5B0F
:102DF000E99CBC1A6D14EE2E0C6BDD6BEBAD8E7680
:102E0000DFCC3EFF006FF3BEA2ED7FC61F5EFAB4BB
:102E1000CE8981F57FA9B723232995D3906BC57BF4
:102E20006B7545B5FA6CF5ECB5B6B1AEB1963FF43D
:102E30003E959FE97F47FA1F5129D4C8FF001B9F89
:102E400057A8C2C5CEFB2E63F1F2CD8C690DA81632
:102E5000BE92DF5AA7B1D7FD36B2DA2DF6FE8B65EA
:102E6000FF00CEFABEB575F55675AE9B57461D6E82
:102E7000CB833A79A1B922E7023F46F68B2BF61FA6
:102E80007EF7EE6ECABF9CDFFA35E15D770C66FD1A
:102E900063C1FAB1D399E8D589E8E0575EF36EDCF7
:102EA0008B087F50B2EB618DB6D666DD7D775D55C0
:102EB0005557E9E3FE8EBAEA63174DFE337ACE2505
:102EC0009D0317A4F48B5CDC0C0CB7E058C1F46CC8
:102ED000762538E5BEEFA4FAF1DD91E97F2EEFD239
:102EE0007FA2B1253DD0FAF7D107D576FD67B45B57
:102EF0004E0BDC595556060B9EF0F753E9D358B1EB
:102F0000D5D8F73AB7BBF9DFE6D9EA7F837A3F52E3
:102F1000FADDD37A6FD5DA3EB15F5DCEC3C96536CF
:102F2000318C6B4DA05E03EBDEC758DAFDBBBF49A9
:102F3000FA55E1FD7332F77D5DFAB9825E7ECF5EB0
:102F40003645E2BEDBECCCCBADCF3FD8A18BD07EFB
:102F5000BA51916FF8B6FABBD3F1985F7E5BB0318E
:102F6000ABAF404BDD43BD367BBDBEE7B1253AB4C8
:102F7000FF008D9FAB96E0E4E78C7CC6E3E29AD835
:102F8000E739950DD65A4FA5454DFB47BEDF4EBBE1
:102F9000AFFDCF468B3FE099631FF1B9F56DB82DBA
:102FA000CF76366B68B2D34564B2A97398D6D9761A
:102FB000C6FDA7E8D2DB68F53FE3EBFF0084F4FC35
:102FC000B6CC37758EA981F55BA2116D343DD5570E
:102FD0007180DB6F7C3BA87517398377D9FF00437D
:102FE000FA0FCFFD9F8B8FFA3F5FD5573EB46255E6
:102FF0009BF5AB0FEAAF493FAAF4FF004FA663B8B9
:103000009241B5CFDD9B937347D1B3ED775DF68FDA
:103010004DBFE09253E9199FE367EAE6155896DF42
:103020008D9A3EDB4FDA2B67A75870AF7D94566CB4
:103030000EBDBFCF7A3EAD5FF01E9D8ADD5FE31F00
:10304000A059D7ABE80F6645399639954BDAC35B83
:103050006D7B5AFF00B358EAADB5CDB9963FECD6BB
:10306000FB3D991FF6E2F26A2CC2EADF5BEDCEF47B
:10307000F7F47E9C1D78AE39C2C0AC330E87B6D74C
:103080007D2CAAB1F1B13DFF00E1F216BFF8A9E92C
:10309000D7F5AFADF7F5ACC26DFB187E4DB6100895
:1030A0007645E5CCAF7FF9D917B36FF84A5253EDA7
:1030B0008924924A7FFFD4F554924925387D5FEAEE
:1030C000974EEB5D6B13A975203229C1ADCDA70DCD
:1030D000CD961B1CE0F375DAFE95BB5ADFD0ECD819
:1030E000A97D77FAA7D53EB4D356155D45B83815F6
:1030F000FBECA7D22F759609D86CB3D4AFF4553733
:10310000E857FE93DF67F81F4FA949253E7D9BFED8
:103110002AECCAFAC5475AFDA2D6B697629F43D198
:1031200026462D7450EF7FABFE17ECFF00B88DD212
:10313000FF00C5A5D83F5C3FE72BFA836C9C8BF260
:103140000E33692DFE7C5BEC161B5FF43D6FDC5D7E
:10315000DA4929F36C2FF14166057D4198DD5BDF8B
:103160009D4FD9ABB0D1AD753DECB323FC2FBACB9D
:103170006AABECDEDF4FF456DCA35FF8A2CBA7A36B
:10318000DDD2E8EAEDADB97736DCBB052E9B1B50EE
:10319000FD531CB064ECF4ABB2DBEF7FEFDBE87FF8
:1031A000A05E96924A7CD7ABFF008A1BFA9DB8F6C8
:1031B0007ED465431B131F1437D02E9F42B6D2EB2B
:1031C0003F9E6FF38F6EF5A5D4FF00C59B33BEB64F
:1031D000B3EB18CD0D6B5F55A70DD56E05F432B668
:1031E00054DF54D9FCCBDF4B3D467A7FCDFB1770C3
:1031F000924A7CDFA6FF008A8EA1819B7F526F5985
:1032000016750B6BB5B5649A5E1D5D97FE8EFCB0AE
:10321000E6646E7DDE8D97FA5FF0D67AFF00E0D02F
:10322000ECFF0013D7BFA3E3F4BFDAAD028C9BF22F
:103230004D9E81D7D6662D2D66DF5FDBE9FD91DFE0
:103240009DFE117A624929F32CEFF139765E36053D
:103250003FB55AC3818C71E7D0277937E4E5EFFE9B
:103260007BD9FD2FD3FEC27FF19BD6AAE85D0BA7C9
:103270007D5EA1C2CEA2290DF560815D22A7E05B33
:1032800073585C7F4B975BEFC7AFF9DF4EAFB4FF6E
:1032900000376FA562F4C5859FF51FEAAF52CDB721
:1032A0003F3B01B9195790EB2D7BEC925A1B5B3DCC
:1032B000BEA6CDAD656C6EC494F31FE29FEA959DEA
:1032C00037A4BFAEDED6B73FA8D7189BE486507DA3
:1032D000D5B9EDF67F49B1ACBBE97F31E87FC221BA
:1032E00074EFF14B978795959CFEAC2FCCC8A6EA5E
:1032F000EBB8D4E69659903D1BF24EDBF758FF0031
:10330000B3DB93E9FF00C3FA76FE62F480000001AC
:10331000007013A4A7CD317FC4FDD8BD333B099DF8
:103320004EB36E79A58FBCE3996D35B8E4594B0760
:10333000AFFE1F2598766EFF00BADFF08BA8FA91DA
:10334000F53EBFAA7D3AEC5F58655F916FA965E1D4
:103350009E9FB400CAAADBBACF6D7EF7FF00D75795
:1033600046924A524924929FFFD5F5549249252905
:103370002492494A4924925292492494A49249257C
:10338000292492494A4924925292492494A4924968
:1033900025292492494FFFD6F55497CAA924A7EAB4
:1033A000A497CAA924A7EAA497CAA924A7EAA4971C
:1033B000CAA924A7EAA497CAA924A7EAA497CAA9D4
:1033C00024A7EAA497CAA924A7EAA497CAA924A76C
:1033D000EAA497CAA924A7EAA497CAA924A7FFD94F
:1033E0003842494D04210000000000550000000152
:1033F000010000000F00410064006F0062006500E2
:103400002000500068006F0074006F0073006800B7
:103410006F00700000001300410064006F00620044
:1034200065002000500068006F0074006F0073009A
:1034300068006F007000200043005300350000005A
:1034400001003842494D0406000000000007000456
:10345000000000010100FFE10DD0687474703A2F84
:103460002F6E732E61646F62652E636F6D2F7861AE
:10347000702F312E302F003C3F787061636B657484
:1034800020626567696E3D22EFBBBF222069643D03
:103490002257354D304D7043656869487A726553DF
:1034A0007A4E54637A6B633964223F3E0D0A3C784E
:1034B0003A786D706D65746120786D6C6E733A78D2
:1034C0003D2261646F62653A6E733A6D6574612F77
:1034D0002220783A786D70746B3D2241646F62658A
:1034E00020584D5020436F726520352E302D6330AB
:1034F00036302036312E3133343737372C203230C6
:1035000031302F30322F31322D31373A33323A3099
:10351000302020202020202020223E0D0A093C724D
:1035200064663A52444620786D6C6E733A726466F3
:103530003D22687474703A2F2F7777772E77332E69
:103540006F72672F313939392F30322F32322D7265
:1035500064662D73796E7461782D6E7323223E0D2F
:103560000A09093C7264663A44657363726970744F
:10357000696F6E207264663A61626F75743D2222D3
:1035800020786D6C6E733A786D703D22687474703B
:103590003A2F2F6E732E61646F62652E636F6D2FED
:1035A0007861702F312E302F2220786D6C6E733A37
:1035B000786D704D4D3D22687474703A2F2F6E7384
:1035C0002E61646F62652E636F6D2F7861702F318D
:1035D0002E302F6D6D2F2220786D6C6E733A7374C0
:1035E0004576743D22687474703A2F2F6E732E6185
:1035F000646F62652E636F6D2F7861702F312E308E
:103600002F73547970652F5265736F7572636545BA
:1036100076656E74232220786D6C6E733A64633D18
:1036200022687474703A2F2F7075726C2E6F7267E7
:103630002F64632F656C656D656E74732F312E3149
:103640002F2220786D6C6E733A70686F746F736898
:103650006F703D22687474703A2F2F6E732E616400
:103660006F62652E636F6D2F70686F746F73686F14
:10367000702F312E302F2220786D703A43726561A1
:10368000746F72546F6F6C3D2241646F626520509D
:10369000686F746F73686F70204353352057696E7D
:1036A000646F77732220786D703A43726561746538
:1036B000446174653D22323031372D30372D31323F
:1036C0005432313A32393A34302B30333A303022B6
:1036D00020786D703A4D6574616461746144617401
:1036E000653D22323031372D30372D313254323171
:1036F0003A32393A34302B30333A30302220786D38
:10370000703A4D6F64696679446174653D22323068
:1037100031372D30372D31325432313A32393A3453
:10372000302B30333A30302220786D704D4D3A498D
:103730006E7374616E636549443D22786D702E69C5
:1037400069643A344144323344364532443637456D
:1037500037313139373034413331434146383141E3
:103760003541442220786D704D4D3A446F63756D3C
:10377000656E7449443D22786D702E6469643A34F4
:10378000394432334436453244363745373131399E
:103790003730344133314341463831413541442299
:1037A00020786D704D4D3A4F726967696E616C4457
:1037B0006F63756D656E7449443D22786D702E643B
:1037C00069643A34394432334436453244363745F5
:1037D0003731313937303441333143414638314163
:1037E000354144222064633A666F726D61743D22F4
:1037F000696D6167652F6A706567222070686F74F4
:103800006F73686F703A436F6C6F724D6F64653D94
:103810002233222070686F746F73686F703A494367
:103820004350726F66696C653D227352474220496E
:10383000454336313936362D322E31223E0D0A09B6
:1038400009093C786D704D4D3A486973746F72790F
:103850003E0D0A090909093C7264663A5365713ED6
:103860000D0A09090909093C7264663A6C692073FA
:10387000744576743A616374696F6E3D2263726554
:1038800061746564222073744576743A696E73744A
:10389000616E636549443D22786D702E6969643AB2
:1038A0003439443233443645324436374537313182
:1038B0003937303441333143414638314135414461
:1038C000222073744576743A7768656E3D223230F3
:1038D00031372D30372D31325432313A32393A3492
:1038E000302B30333A3030222073744576743A737B
:1038F0006F6674776172654167656E743D224164DD
:103900006F62652050686F746F73686F70204353E7
:10391000352057696E646F7773222F3E0D0A0909AF
:103920000909093C7264663A6C69207374457674BF
:103930003A616374696F6E3D22736176656422201B
:1039400073744576743A696E7374616E6365494445
:103950003D22786D702E6969643A344144323344B3
:1039600036453244363745373131393730344133D3
:103970003143414638314135414422207374457604
:10398000743A7768656E3D22323031372D30372DED
:1039900031325432313A32393A34302B30333A30D2
:1039A00030222073744576743A736F66747761724F
:1039B000654167656E743D2241646F6265205068A1
:1039C0006F746F73686F70204353352057696E644E
:1039D0006F7773222073744576743A6368616E67FB
:1039E00065643D222F222F3E0D0A090909093C2F4B
:1039F0007264663A5365713E0D0A0909093C2F78D5
:103A00006D704D4D3A486973746F72793E0D0A09B5
:103A1000093C2F7264663A44657363726970746915
:103A20006F6E3E0D0A093C2F7264663A5244463E60
:103A30000D0A3C2F783A786D706D6574613E0D0A01
:103A40002020202020202020202020202020202076
:103A50002020202020202020202020202020202066
:103A60002020202020202020202020202020202056
:103A70002020202020202020202020202020202046
:103A80002020202020202020202020202020202036
:103A90002020202020202020202020202020202026
:103AA000202020200A20202020202020202020202C
:103AB0002020202020202020202020202020202006
:103AC00020202020202020202020202020202020F6
:103AD00020202020202020202020202020202020E6
:103AE00020202020202020202020202020202020D6
:103AF00020202020202020202020202020202020C6
:103B00002020202020202020200A202020202020CB
:103B100020202020202020202020202020202020A5
:103B20002020202020202020202020202020202095
:103B30002020202020202020202020202020202085
:103B40002020202020202020202020202020202075
:103B50002020202020202020202020202020202065
:103B600020202020202020202020202020200A206B
:103B70002020202020202020202020202020202045
:103B80002020202020202020202020202020202035
:103B90002020202020202020202020202020202025
:103BA0002020202020202020202020202020202015
:103BB0002020202020202020202020202020202005
:103BC00020202020202020202020202020202020F5
:103BD0002020200A202020202020202020202020FB
:103BE00020202020202020202020202020202020D5
:103BF00020202020202020202020202020202020C5
:103C000020202020202020202020202020202020B4
:103C100020202020202020202020202020202020A4
:103C20002020202020202020202020202020202094
:103C300020202020202020200A202020202020209A
:103C40002020202020202020202020202020202074
:103C50002020202020202020202020202020202064
:103C60002020202020202020202020202020202054
:103C70002020202020202020202020202020202044
:103C80002020202020202020202020202020202034
:103C9000202020202020202020202020200A20203A
:103CA0002020202020202020202020202020202014
:103CB0002020202020202020202020202020202004
:103CC00020202020202020202020202020202020F4
:103CD00020202020202020202020202020202020E4
:103CE00020202020202020202020202020202020D4
:103CF00020202020202020202020202020202020C4
:103D000020200A20202020202020202020202020C9
:103D100020202020202020202020202020202020A3
:103D20002020202020202020202020202020202093
:103D30002020202020202020202020202020202083
:103D40002020202020202020202020202020202073
:103D50002020202020202020202020202020202063
:103D6000202020202020200A202020202020202069
:103D70002020202020202020202020202020202043
:103D80002020202020202020202020202020202033
:103D90002020202020202020202020202020202023
:103DA0002020202020202020202020202020202013
:103DB0002020202020202020202020202020202003
:103DC0002020202020202020202020200A20202009
:103DD00020202020202020202020202020202020E3
:103DE00020202020202020202020202020202020D3
:103DF00020202020202020202020202020202020C3
:103E000020202020202020202020202020202020B2
:103E100020202020202020202020202020202020A2
:103E20002020202020202020202020202020202092
:103E3000200A202020202020202020202020202098
:103E40002020202020202020202020202020202072
:103E50002020202020202020202020202020202062
:103E60002020202020202020202020202020202052
:103E70002020202020202020202020202020202042
:103E80002020202020202020202020202020202032
:103E90002020202020200A20202020202020202038
:103EA0002020202020202020202020202020202012
:103EB0002020202020202020202020202020202002
:103EC00020202020202020202020202020202020F2
:103ED00020202020202020202020202020202020E2
:103EE00020202020202020202020202020202020D2
:103EF00020202020202020202020200A20202020D8
:103F000020202020202020202020202020202020B1
:103F100020202020202020202020202020202020A1
:103F20002020202020202020202020202020202091
:103F30002020202020202020202020202020202081
:103F40002020202020202020202020202020202071
:103F50002020202020202020202020202020202061
:103F60000A20202020202020202020202020202067
:103F70002020202020202020202020202020202041
:103F80002020202020202020202020202020202031
:103F90002020202020202020202020202020202021
:103FA0002020202020202020202020202020202011
:103FB0002020202020202020202020202020202001
:103FC00020202020200A2020202020202020202007
:103FD00020202020202020202020202020202020E1
:103FE00020202020202020202020202020202020D1
:103FF00020202020202020202020202020202020C1
:1040000020202020202020202020202020202020B0
:1040100020202020202020202020202020202020A0
:10402000202020202020202020200A2020202020A6
:104030002020202020202020202020202020202080
:104040002020202020202020202020202020202070
:104050002020202020202020202020202020202060
:104060002020202020202020202020202020202050
:104070002020202020202020202020202020202040
:104080002020202020202020202020202020200A46
:104090002020202020202020202020202020202020
:1040A0002020202020202020202020202020202010
:1040B0002020202020202020202020202020202000
:1040C00020202020202020202020202020202020F0
:1040D00020202020202020202020202020202020E0
:1040E00020202020202020202020202020202020D0
:1040F000202020200A2020202020202020202020D6
:1041000020202020202020202020202020202020AF
:10411000202020202020202020202020202020209F
:10412000202020202020202020202020202020208F
:10413000202020202020202020202020202020207F
:10414000202020202020202020202020202020206F
:104150002020202020202020200A20202020202075
:10416000202020202020202020202020202020204F
:10417000202020202020202020202020202020203F
:10418000202020202020202020202020202020202F
:10419000202020202020202020202020202020201F
:1041A000202020202020202020202020202020200F
:1041B00020202020202020202020202020200A2015
:1041C00020202020202020202020202020202020EF
:1041D00020202020202020202020202020202020DF
:1041E00020202020202020202020202020202020CF
:1041F00020202020202020202020202020202020BF
:1042000020202020202020202020202020202020AE
:1042100020202020203C3F787061636B657420650E
:104220006E643D2777273F3EFFE20C584943435FCA
:1042300050524F46494C4500010100000C484C6962
:104240006E6F021000006D6E747252474220585912
:104250005A2007CE00020009000600310000616309
:1042600073704D534654000000004945432073527B
:1042700047420000000000000000000000010000B4
:10428000F6D6000100000000D32D48502020000089
:10429000000000000000000000000000000000001E
:1042A000000000000000000000000000000000000E
:1042B000000000000000000000000000001163701A
:1042C00072740000015000000033646573630000E5
:1042D00001840000006C77747074000001F000002D
:1042E0000014626B70740000020400000014725825
:1042F000595A00000218000000146758595A00006B
:10430000022C000000146258595A000002400000BC
:104310000014646D6E640000025400000070646D4F
:104320006464000002C400000088767565640000C3
:10433000034C0000008676696577000003D4000016
:1043400000246C756D69000003F8000000146D65B1
:1043500061730000040C00000024746563680000B1
:1043600004300000000C725452430000043C000072
:10437000080C675452430000043C0000080C6254CF
:1043800052430000043C0000080C7465787400007F
:104390000000436F70797269676874202863292070
:1043A00031393938204865776C6574742D506163F4
:1043B0006B61726420436F6D70616E79000064659B
:1043C000736300000000000000127352474220494E
:1043D000454336313936362D322E3100000000008B
:1043E0000000000000001273524742204945433646
:1043F000313936362D322E31000000000000000029
:1044000000000000000000000000000000000000AC
:10441000000000000000000000000000000000009C
:104420000000000000000000000058595A20000061
:1044300000000000F35100010000000116CC5859A3
:104440005A200000000000000000000000000000F2
:10445000000058595A200000000000006FA2000020
:1044600038F50000039058595A2000000000000061
:1044700062990000B785000018DA58595A200000E8
:104480000000000024A000000F840000B6CF646587
:104490007363000000000000001649454320687463
:1044A00074703A2F2F7777772E6965632E636800D3
:1044B000000000000000000000001649454320688D
:1044C0007474703A2F2F7777772E6965632E63683F
:1044D00000000000000000000000000000000000DC
:1044E00000000000000000000000000000000000CC
:1044F00000000000000000000000000000006465F3
:104500007363000000000000002E4945432036314F
:104510003936362D322E312044656661756C742033
:1045200052474220636F6C6F7572207370616365D0
:10453000202D2073524742000000000000000000C0
:1045400000002E4945432036313936362D322E3182
:104550002044656661756C742052474220636F6C1D
:104560006F7572207370616365202D20735247420E
:10457000000000000000000000000000000000003B
:10458000000000000000646573630000000000008C
:10459000002C5265666572656E63652056696577A5
:1045A000696E6720436F6E646974696F6E20696E0F
:1045B0002049454336313936362D322E3100000040
:1045C00000000000000000002C5265666572656EF8
:1045D00063652056696577696E6720436F6E64690D
:1045E00074696F6E20696E2049454336313936361D
:1045F0002D322E31000000000000000000000000FD
:1046000000000000000000000000000000007669CB
:104610006577000000000013A4FE00145F2E001058
:10462000CF140003EDCC0004130B00035C9E0000CC
:10463000000158595A2000000000004C0956005053
:10464000000000571FE76D65617300000000000067
:104650000001000000000000000000000000000059
:1046600000000000028F0000000273696720000054
:104670000000435254206375727600000000000071
:10468000040000000005000A000F00140019001EBD
:1046900000230028002D00320037003B0040004579
:1046A000004A004F00540059005E00630068006D2E
:1046B00000720077007C00810086008B00900095DE
:1046C000009A009F00A400A900AE00B200B700BC91
:1046D00000C100C600CB00D000D500DB00E000E543
:1046E00000EB00F000F600FB01010107010D0113D2
:1046F0000119011F0125012B01320138013E01453D
:10470000014C0152015901600167016E0175017C84
:104710000183018B0192019A01A101A901B101B9A3
:1047200001C101C901D101D901E101E901F201FA97
:104730000203020C0214021D0226022F023802415B
:10474000024B0254025D02670271027A0284028EF9
:10475000029802A202AC02B602C102CB02D502E06C
:1047600002EB02F50300030B03160321032D0338AC
:104770000343034F035A03660372037E038A0396BF
:1047800003A203AE03BA03C703D303E003EC03F9A8
:10479000040604130420042D043B04480455046358
:1047A0000471047E048C049A04A804B604C404D3DF
:1047B00004E104F004FE050D051C052B053A05492E
:1047C0000558056705770586059605A605B505C54F
:1047D00005D505E505F6060606160627063706483A
:1047E0000659066A067B068C069D06AF06C006D1F2
:1047F00006E306F507070719072B073D074F076173
:1048000007740786079907AC07BF07D207E507F8C3
:10481000080B081F08320846085A086E08820896D6
:1048200008AA08BE08D208E708FB09100925093ABA
:10483000094F09640979098F09A409BA09CF09E563
:1048400009FB0A110A270A3D0A540A6A0A810A98D2
:104850000AAE0AC50ADC0AF30B0B0B220B390B510B
:104860000B690B800B980BB00BC80BE10BF90C120A
:104870000C2A0C430C5C0C750C8E0CA70CC00CD9CC
:104880000CF30D0D0D260D400D5A0D740D8E0DA956
:104890000DC30DDE0DF80E130E2E0E490E640E7FA5
:1048A0000E9B0EB60ED20EEE0F090F250F410F5EB6
:1048B0000F7A0F960FB30FCF0FEC1009102610438D
:1048C0001061107E109B10B910D710F51113113123
:1048D000114F116D118C11AA11C911E8120712267E
:1048E00012451264128412A312C312E3130313239A
:1048F00013431363138313A413C513E5140614277A
:104900001449146A148B14AD14CE14F01512153416
:1049100015561578159B15BD15E016031626164974
:10492000166C168F16B216D616FA171D1741176594
:10493000178917AE17D217F7181B18401865188A71
:1049400018AF18D518FA19201945196B199119B70C
:1049500019DD1A041A2A1A511A771A9E1AC51AEC66
:104960001B141B3B1B631B8A1BB21BDA1C021C2A79
:104970001C521C7B1CA31CCC1CF51D1E1D471D704E
:104980001D991DC31DEC1E161E401E6A1E941EBEE0
:104990001EE91F131F3E1F691F941FBF1FEA20152A
:1049A0002041206C209820C420F0211C2148217532
:1049B00021A121CE21FB22272255228222AF22DDF6
:1049C000230A23382366239423C223F0241F244D73
:1049D000247C24AB24DA250925382568259725C7AA
:1049E00025F726272657268726B726E8271827499A
:1049F000277A27AB27DC280D283F287128A228D446
:104A000029062938296B299D29D02A022A352A68A6
:104A10002A9B2ACF2B022B362B692B9D2BD12C05C1
:104A20002C392C6E2CA22CD72D0C2D412D762DAB94
:104A30002DE12E162E4C2E822EB72EEE2F242F5A1D
:104A40002F912FC72FFE3035306C30A430DB311260
:104A5000314A318231BA31F2322A3263329B32D456
:104A6000330D3346337F33B833F1342B3465349E02
:104A700034D83513354D358735C235FD3637367266
:104A800036AE36E937243760379C37D7381438507C
:104A9000388C38C839053942397F39BC39F93A364A
:104AA0003A743AB23AEF3B2D3B6B3BAA3BE83C27CA
:104AB0003C653CA43CE33D223D613DA13DE03E2000
:104AC0003E603EA03EE03F213F613FA23FE24023E7
:104AD000406440A640E74129416A41AC41EE423082
:104AE000427242B542F7433A437D43C044034447D0
:104AF000448A44CE45124555459A45DE46224667CE
:104B000046AB46F04735477B47C04805484B489180
:104B100048D7491D496349A949F04A374A7D4AC4E3
:104B20004B0C4B534B9A4BE24C2A4C724CBA4D02F5
:104B30004D4A4D934DDC4E254E6E4EB74F004F49BA
:104B40004F934FDD5027507150BB51065150519B30
:104B500051E65231527C52C75313535F53AA53F656
:104B60005442548F54DB5528557555C2560F565C28
:104B700056A956F75744579257E0582F587D58CBAF
:104B8000591A596959B85A075A565AA65AF55B45DF
:104B90005B955BE55C355C865CD65D275D785DC9C1
:104BA0005E1A5E6C5EBD5F0F5F615FB3600560574C
:104BB00060AA60FC614F61A261F56249629C62F08B
:104BC0006343639763EB6440649464E9653D659275
:104BD00065E7663D669266E8673D679367E9683F0B
:104BE000689668EC6943699A69F16A486A9F6AF74E
:104BF0006B4F6BA76BFF6C576CAF6D086D606DB939
:104C00006E126E6B6EC46F1E6F786FD1702B7086D4
:104C100070E0713A719571F0724B72A67301735D19
:104C200073B87414747074CC7528758575E1763E0C
:104C3000769B76F8775677B37811786E78CC792AA8
:104C4000798979E77A467AA57B047B637BC27C21EC
:104C50007C817CE17D417DA17E017E627EC27F23DD
:104C60007F847FE5804780A8810A816B81CD823077
:104C7000829282F4835783BA841D848084E38547BB
:104C800085AB860E867286D7873B879F88048869A6
:104C900088CE8933899989FE8A648ACA8B308B963B
:104CA0008BFC8C638CCA8D318D988DFF8E668ECE79
:104CB0008F368F9E9006906E90D6913F91A892115C
:104CC000927A92E3934D93B69420948A94F4955FEC
:104CD00095C99634969F970A977597E0984C98B81F
:104CE0009924999099FC9A689AD59B429BAF9C1CF9
:104CF0009C899CF79D649DD29E409EAE9F1D9F8B7C
:104D00009FFAA069A0D8A147A1B6A226A296A306A1
:104D1000A376A3E6A456A4C7A538A5A9A61AA68B70
:104D2000A6FDA76EA7E0A852A8C4A937A9A9AA1CE6
:104D3000AA8FAB02AB75ABE9AC5CACD0AD44ADB8FF
:104D4000AE2DAEA1AF16AF8BB000B075B0EAB160BA
:104D5000B1D6B24BB2C2B338B3AEB425B49CB5131E
:104D6000B58AB601B679B6F0B768B7E0B859B8D128
:104D7000B94AB9C2BA3BBAB5BB2EBBA7BC21BC9BD2
:104D8000BD15BD8FBE0ABE84BEFFBF7ABFF5C07021
:104D9000C0ECC167C1E3C25FC2DBC358C3D4C45116
:104DA000C4CEC54BC5C8C646C6C3C741C7BFC83DAC
:104DB000C8BCC93AC9B9CA38CAB7CB36CBB6CC35E4
:104DC000CCB5CD35CDB5CE36CEB6CF37CFB8D039C0
:104DD000D0BAD13CD1BED23FD2C1D344D3C6D4493C
:104DE000D4CBD54ED5D1D655D6D8D75CD7E0D8645C
:104DF000D8E8D96CD9F1DA76DAFBDB80DC05DC8A1D
:104E0000DD10DD96DE1CDEA2DF29DFAFE036E0BD7F
:104E1000E144E1CCE253E2DBE363E3EBE473E4FC83
:104E2000E584E60DE696E71FE7A9E832E8BCE94627
:104E3000E9D0EA5BEAE5EB70EBFBEC86ED11ED9C6B
:104E4000EE28EEB4EF40EFCCF058F0E5F172F1FF50
:104E5000F28CF319F3A7F434F4C2F550F5DEF66DD5
:104E6000F6FBF78AF819F8A8F938F9C7FA57FAE7FC
:104E7000FB77FC07FC98FD29FDBAFE4BFEDCFF6DBD
:104E8000FFFFFFDB004300020101020101020202F9
:104E900002020202020305030303030306040403E0
:104EA00005070607070706070708090B0908080A88
:104EB0000807070A0D0A0A0B0C0C0C0C07090E0F49
:104EC0000D0C0E0B0C0C0CFFDB0043010202020365
:104ED0000303060303060C0807080C0C0C0C0C0C4F
:104EE0000C0C0C0C0C0C0C0C0C0C0C0C0C0C0C0C02
:104EF0000C0C0C0C0C0C0C0C0C0C0C0C0C0C0C0CF2
:104F00000C0C0C0C0C0C0C0C0C0C0C0CFFC0001141
:104F10000800F0014003012200021101031101FF0A
:104F2000C4001F0000010501010101010100000092
:104F300000000000000102030405060708090A0B2F
:104F4000FFC400B5100002010303020403050504B9
:104F5000040000017D01020300041105122131410A
:104F60000613516107227114328191A1082342B1C5
:104F7000C11552D1F02433627282090A161718192A
:104F80001A25262728292A3435363738393A434412
:104F900045464748494A535455565758595A6364E9
:104FA00065666768696A737475767778797A8384D9
:104FB00085868788898A92939495969798999AA2DC
:104FC000A3A4A5A6A7A8A9AAB2B3B4B5B6B7B8B901
:104FD000BAC2C3C4C5C6C7C8C9CAD2D3D4D5D6D726
:104FE000D8D9DAE1E2E3E4E5E6E7E8E9EAF1F2F369
:104FF000F4F5F6F7F8F9FAFFC4001F010003010108
:105000000101010101010100000000000001020393
:105010000405060708090A0BFFC400B511000201C8
:1050200002040403040705040400010277000102DE
:105030000311040521310612415107617113223217
:105040008108144291A1B1C109233352F015627253
:10505000D10A162434E125F11718191A2627282910
:105060002A35363738393A434445464748494A5342
:105070005455565758595A636465666768696A7328
:105080007475767778797A82838485868788898A29
:1050900092939495969798999AA2A3A4A5A6A7A847
:1050A000A9AAB2B3B4B5B6B7B8B9BAC2C3C4C5C673
:1050B000C7C8C9CAD2D3D4D5D6D7D8D9DAE2E3E49F
:1050C000E5E6E7E8E9EAF2F3F4F5F6F7F8F9FAFFCE
:1050D000DA000C03010002110311003F00FDFCA2E5
:1050E0008A2800A28A2800A28A2800A28A2800A270
:1050F0008A2800A28A2800A28A2800A28A2800A260
:105100008A2800A28A2800A28A2800A28A2800A24F
:105110008A2800A28A2800A28A2800A28A2800A23F
:105120008A2800A28A2800A28A2800A28A2800A22F
:105130008A2800A28A2800A28A2800A28A2800A21F
:105140008A2800A28A2800A28A2800A28A2800A20F
:105150008A2800A28A2800A28A2800A28A2800A2FF
:105160008A2800A28A2800A28A2800A28A2800A2EF
:105170008A2800A28A2800A28A2800A28A2800A2DF
:105180008A2800A28A2800A28A2800A28A2800A2CF
:105190008A2800A28A2800A28A2800A28A2800A2BF
:1051A0008A2800A28A2800A28A2800A28A2800A2AF
:1051B0008A2800A28A2800A28A2800A28A2800A29F
:1051C0008A2800A28A2800A28A2800A28A2800A28F
:1051D0008A2800A28A2800A28A2800A28A2800A27F
:1051E0008A2800A28A2800A28A2800A28A2800A26F
:1051F0008A2800A28A2800A28A2800A28A2800A25F
:105200008A2800A2BE20FF0082BAFF00C168749FF6
:10521000F82415DF842EBC59F0BFC69E2CF0CF8C2D
:105220009668ADF5BD1E6816DADAF23E5AD65F31E1
:1052300086C73191227F7C0936FF00AB7AF8E348BC
:10524000FF0083D73E08EA3ABD9C179F09FE275806
:1052500059CD7091CF75E7D94A6DE3270F26C12745
:10526000CFB579DBDE803F69A8AC5F0478DB49F815
:1052700091E0ED27C43A0EA367AC689AF59C3A8694
:105280009D7D6D20920BDB79515E296361F79191D1
:105290008303DEB6A800A28A2800A28A2800A28A78
:1052A0002800A28A2800A28A2800A28A2800A28AAE
:1052B00028021B8B88ED61F324748D57EF331DABEF
:1052C000535787FF00C14C3C3ADE30FF008272FC2E
:1052D0007ED2225DD36ABF0E3C43691FBB3E9772EC
:1052E000A3F9D7E2FF00FC1023FE0E875F0D45A255
:1052F000FC17FDA735D93FB357CBB1F0EFC41BD98D
:10530000377D93F863B7D5243FC1D96ECFDDFF0059
:1053100096DF2EE95003F7EFC4FE2CD2FC0FA2DC7F
:105320006A9AC6A563A4E9768375C5E5ECEB04101B
:105330008271F33B90ABCD731FF0D4BF0CBFE8A2DA
:105340007817FF0007D6BFFC5D5DF8B9F097C33F43
:10535000B457C22D77C21E2AD32CFC41E15F1658E8
:1053600049A7DFD9CDF345776F22E0F23F3565E5F8
:1053700078606BF8DBFF0082BA7FC1327C4DFF00A2
:1053800004AEFDB0B58F87BAC1B8D4BC37719D4BA0
:10539000C29ADB05D9AD69AE7E4638C6D9A3E629E7
:1053A000578F9D32BF2346CC01FD91EB3F1E3C1130
:1053B000E1EB7B09B52F19784EC22D52DFED765205
:1053C0005C6AF6F12DDC27FE5A45B9BE74FF006811
:1053D0007150E93FB467C3FF0010EB16FA769FE304
:1053E000AF076A1A85F3F956D6B6FAD5B4B35C3F5F
:1053F000F75115F7337B0AFE5CFF00E0BBED6979DE
:10540000FB037FC13CEEEDE245924F842B6F249B62
:105410007E67F2E3B25C1F6DFBF1F5AF95FF00E034
:105420008FDA9A697FF0559FD9C66926F257FE1622
:1054300046809BB1D77EA10AEDE3D775007F665AFF
:1054400097ED21F0F744D4AE2CAF7C75E0FB2BDB5D
:10545000395A0B8B7B8D6ADA296091782AEACF90D2
:10546000C2B43C15F17BC25F12EFAEADFC3BE26F04
:105470000EEBD7164AB2DC47A6EA30DD340AFB82CF
:10548000B38463B7383D7D2BF8D1FF0082DAE9564B
:10549000FA37FC15C3F68B86D6158626F1E6A93BAE
:1054A0002AF7924B8691DBF17663F8D7E837FC193F
:1054B0007FADEA5A67C7DF8FF0E983CCB8FF00847D
:1054C0002A0B9862D81BCDB88EE1BCAFD5CD007F3A
:1054D00044FE33F8CFE0FF0087178B6BE22F15787F
:1054E0006F41B8990C8916A5A9436ACE9FDE01D8F1
:1054F000715535FF008F9E05F0ADC5BC5AA78CBC19
:1055000027A6CB796EB7904777AB5BC2D3C2FF00BB
:105510007265DCE3721ECDD2BF85BF8A9F123C4507
:10552000F17FE22EB5E27F176A9A86B9E28D72EEBC
:105530004BDD4EFEFE4692E6EE776CBB3B1EF5F76A
:1055400037ED9D65FF000D9BFF000451FD9E3E362B
:1055500043FE91E2AF817A85CFC16F164A4334B2E0
:1055600058A2FDB744703F820860778371FBD24B2D
:10557000401FD5D69DFB46FC3ED6EEBC8B3F1D782A
:105580003AF6758A494C76FACDB4AE1235DEED8521
:105590007276AA8CB1EC2A18FF006A4F8632C619BF
:1055A0003E23781595BA37FC2416BFFC72BF88FFDE
:1055B00000D8F7F6839BF653FDA7FC07F1123B4496
:1055C000D4A1F0AEAF0DE5EE9EC8AF1EAB67BB6DCC
:1055D000D59BAB0DA52781A585B3FC329AFA03FEB6
:1055E0000B69FF0004DDB6FF00827BFED511DC787D
:1055F00035CEA7F057E29598F157C3AD563792587C
:105600006E34D9823FD9BCC7C977B7F35172599963
:10561000A278246E64C5007F5F577F1FBC0BA7F87C
:105620007EC756B8F1AF84E1D2754964B7B2BE9374
:1056300055812DEEE44DDBD6390BED765DAD9C55F5
:10564000793F6A4F8650C7B9BE22781557D7FB7A83
:10565000D7FF008BAFE55FE3BF8857C4BFF06C7F17
:10566000C0B8BF7ECDA07C64D6B4F532FDD4DF6770
:1056700025C6D4FF0063F7BFF7D66BF39E803FBE0D
:10568000CBED7AC74BD1A4D4AE2EEDEDEC6187CF34
:1056900092EA59024691E33B8B9E36FBD737A67EB2
:1056A000D03E03D6ECB50B9B2F1AF84EF2D747B677
:1056B0003797F2C1ACDBCA9636E3ACB2B2BFC89F33
:1056C000ED3715FCF6FF00C1D79F1CFC73AA7ECEF8
:1056D0005FB21F8715EE34AF879E24F052EBF25A6B
:1056E000C170FE45FEA4B6F68ACB2AF47FB3C52A64
:1056F0007967FE9EA4AF867FE083BF1C745F85BF81
:10570000F050DD07C27E2EFDE7C3FF008E3A6DEF3D
:10571000C2EF1646563FDE58EAEAB047F3B7116DBE
:10572000BC16B233F658CD007F5E3FF0D45F0CFF5D
:1057300000E8A27817FF0007D6BFFC7292E3F69547
:10574000F8736261371E3EF05C2B7917DAADCBEB54
:1057500096A82E21DEC9E627EF3E64DE8EBB871BAE
:1057600091876AFE1DBF689F823AC7ECD7F1DFC6FA
:105770005F0F7C40B18D73C11AD5E6857C53EE3C3A
:10578000D6F3344CCBFEC9D995F635F7AFFC13DF11
:10579000F6451FF057AFF82607C41F85BA2AC37114
:1057A000F1D7F673B87F1578095E4DB2EBBA15E9FB
:1057B00066BED1571FC2B748D3C5BFEEDC5F6DCA06
:1057C0002CD2B5007F53DE1CF8FF00E05F186B7130
:1057D000697A3F8D7C27AAEA571BBC9B4B2D5ADE6A
:1057E000E279368C9C22392702AA37ED41F0CD1D93
:1057F00095BE22781772FCACA75DB5E187FC0EBFA1
:10580000944FF83622C9ACFF00E0BA7F0561B88A30
:10581000459ADDB5C56465DAC8C343D4057C57F144
:10582000F7C3B6FE0FF8EBE35D26D7CCFB2E97AEA1
:10583000DF5A43BFEF6D8EE2445CFE5401FDCD594B
:10584000FC7AF03EA3E1DBED62DFC65E15BAD274EE
:10585000A78E2BEBF8B5581ED6D247DA1165915FAB
:105860006A16DEB8CFAFD2AAFF00C352FC32FF00E7
:10587000A289E05FFC1F5AFF00F175FCB8FF00C170
:105880003E649352FF008371BF6F4B166DB15BEBAB
:105890001E0DB853B7E6DDFDAD016FFD14B5F99BE4
:1058A000401FDBD7FC140FF62FF05FFC1507F6291D
:1058B000F137C35D62E6CEE34AF1559ADD68DAD589
:1058C000BEDBAFECDBC5F9ED6FA0656F9B6BE33B17
:1058D00058799199133B5CD7F17FFB43FC03F14F5F
:1058E000ECB5F1ABC51F0EFC69A649A478A7C21A96
:1058F0008CBA66A36CDCED9233F791BF8A361874CC
:105900007FBAE855870457F633FF000443D43FB508
:105910003FE0917FB3ACBE5F95B7C09A6C381DF67F
:1059200042A99FC76E6BF17BFE0E58F82DA1FED8E1
:10593000BFB40FC70F14785F46B5D1FE307ECD736C
:10594000E9D078BF4CB775797C57E12BAB3B69AD9B
:1059500075C44DC1CC96535C7D9EE36A385865B6DC
:1059600066915536D007B87FC1A0DFF05638FC618C
:10597000E0BBAFD96FC75AB1FED8D0A39B52F01489
:10598000D7127CF7969F34975A7AEEFBCF0FCD341F
:105990006BF37EE8CDF7521AFDCAD7F5FB3F0CE852
:1059A000F77A8EA3776F61A7D842D7173737122CB3
:1059B00051411A2EE77776E0205EA7B57F087F0376
:1059C000BE367893F673F8BDE19F1E784351934934
:1059D000F13784F518754D3AF23EB0CD13065C8E62
:1059E000EA7A329E194953C66BFB2EFD857F6B4FB9
:1059F00000FF00C1633FE09DF67E285B5B5BCD0F3F
:105A0000C7DA3DC787BC5BA1B49E67F67DCBC3E414
:105A1000DFD83F7DB890ED2705E29237C7CF401E13
:105A2000C7FF000D45F0CFFE8A27817FF07D6BFF19
:105A300000C72A7BAFDA03C09A5E8961AA5C78D37B
:105A4000C276FA6EAC645B0BB9759B74B7BE68DB4B
:105A500012F94E5F0FB0F0DB73B6BF87EFDAAFF627
:105A60007CD53F64DFDA4FC79F0DB5C39D4BC0DACD
:105A7000EDDE8B349B36F9FE44AD1ACCBFECC8A0EA
:105A80003AFB115F617ECB3327ED9DFF00043CF8AC
:105A9000E1F08E6F2EEBC63FB3A6B307C59F0B2E6A
:105AA0004BDD4BA3CDFE89ACC49C7C96F07EEAE531
:105AB000F1F79E5FC803FAB787F69BF86F3DDC509D
:105AC000C3F103C1534F70EB1451C7AE5AB3C8ECC6
:105AD00070AAAA1F924F6A9B5BFDA17C03E19D66A1
:105AE000E34DD4BC71E10D3752B36DB716B77ACD23
:105AF000BC53DBB6376D7467CAF06BF843B3BC9B1D
:105B00004DBB8AE2DE5921B88595E3911F6B46C3F0
:105B1000904115F7E7FC176D6DFF006918FE05FE53
:105B2000D5FA5C3FB9FDA33C1307FC246CB0F94ADD
:105B30009E27D1F6E9DA9AAA7F045F241B3FBF8231
:105B4000DDE803FACDF067C66F08FC45D466B3F014
:105B5000FF008A3C3BAF5D5BA79B243A7EA50DD43A
:105B6000889BB1B98231C0AEA6BF8DDFF837B7F6DA
:105B7000CE5FD883FE0AB7F0CBC417D726DBC39E0F
:105B80002ABCFF0084435E3E6AC49F65BF2B124956
:105B9000233748E1B9FB34EDFECC15FD91500145AA
:105BA0001450014514500145145001451450073B51
:105BB000F15FC27FF0B03E17789741FBDFDB7A558B
:105BC000CE9E47FD758593FF0066AFE096BFBFCAC6
:105BD000FE073E20785E4F0478EF5AD125CF9BA375
:105BE000DFCF62FF00EF472327FECB401FD05FFCD3
:105BF0001A03FF000552BCF881E1DD6BF665F1D6B2
:105C0000BF35DEA3A05B9D63C073DE4FBA592C5134
:105C1000556E74D42C7FE5861668A31B8F96F71DEE
:105C20001225AFD0EFF82DB7FC12A746FF0082AEC9
:105C30007EC6DA8F857CBB2B3F885E19F3755F05C6
:105C40006AD28C7D92FBCBE6DA47EA2DEE36AC7257
:105C5000765FDDC9B59A2515FC887ECB7FB47F8938
:105C60007F642FDA1BC21F133C1D79F63F12782F79
:105C7000548753B36DECA92146F9E193691BA395B1
:105C80003746EBFC48ECBDEBFB67FD8EBF6A7F0D32
:105C9000FEDB7FB30F827E2BF846612F87FC6DA65B
:105CA000477F0C6D2877B593949AD9F1C7990CCB9F
:105CB0002C2FFEDC46803F9B7FF82FF783351F8714
:105CC000DFF04C3FF8277E93AF68F7DA0F88F47F58
:105CD000086B9A56A767A85AB5ADE5A4D6E348461F
:105CE000865470186C7DFF009D7C1FFF0004C8BDAA
:105CF000FECBFF0082927ECF775B77FD9BE25F87D2
:105D000025DBFDFDBAA5B1AFDFAFF83C47F60EF1DC
:105D100087ED23FB247817E2B78561FED2B5F81F23
:105D20002EA536BDA745033CFF00D9F7DF630F78EA
:105D3000B8FE1B76B44320DBFEAE57932AB1357F05
:105D40003CBFB13EB13F873F6CBF849A85AC9E4D4E
:105D5000D58F8CF47B889CFF000325F42CADCFD22B
:105D6000803E80FF00838634E7D33FE0B39F1FE38C
:105D7000787ECED2788239B695DB957B381C37FC9D
:105D80000B766BEC8FF83286F0C7FF000506F8A1A2
:105D90006FE715F37E1F4B288B77DFDBA9588CE369
:105DA000DB77EB5E7BFF00076CFEC41E2EF815FF51
:105DB000000527D5BE2D5E47F6CF05FC638ADAE3E2
:105DC0004DBF8A33B6D2EAD2CE0B59ACE53FF3D3FE
:105DD0001124ABFDE4978FB8F8E97FE0CB29BCBF75
:105DE000F82A778E55BAB7C2CD4517FF0006DA43B9
:105DF00050076BFF0005F4FF008367FE217823E363
:105E00009F893E2F7ECF3E15BEF1C782BC59752EAD
:105E1000ABAAF8634783CED4FC3F773499945B5B9D
:105E20002FCD716CEEFB91615678B25766C4DF5E80
:105E300003FF000469FD9C7E227C404FDA0FF65779
:105E4000F16780FC61A1DBFC76F054DFD94BAB68D5
:105E50007359C565E28D1F75FE98D2CB347FE8E992
:105E6000FEBD1FFBDE627FB35FD207FC1563F68BBE
:105E7000F157EC95FF0004EBF8BDF123C0F6B1DD5E
:105E800078AFC25E1E9AF34DDF6FE7ADAC9F2A7DFF
:105E9000A193043084319886F94F95F37CB9AFE62D
:105EA000C7F61EFF00839F7F69AFD9A3E3BD8EB9FC
:105EB000E3BF1D6ADF15BC1779761B5CF0FEB221CB
:105EC000669E26FBCD6B3EC0F6D228FB814F959F88
:105ED000BC86803F37E589AD249239232ACA76B241
:105EE000B0F994D7F435FF0004E0F82FA47FC17D0A
:105EF000FF00E0DD55F83BAF5F467E277C0FBF9784
:105F000047F0D6AD74DBA5D3E5823F374EDD8FBBBE
:105F10006CF6D2FD89BFD880B60BA263F28FFE0B60
:105F200099F097C3FE04FF0082817883C63E0991F1
:105F3000A6F877F1C2C6D7E27F8567D9E5F9D67AA8
:105F4000AAB4D28D9FF2CF65D8BA8FCBFE0F2F6D3A
:105F50007D63FF0006757ED7B2FC17FF00828EEBD3
:105F60001F0B2E1E66D27E32E853450C491F1FDAE6
:105F70003A7472DE41231FE14FB37DBD7DD9D280DB
:105F80003C77E24780FC45F0DFFE0DBDD43C37E2B4
:105F90003B0BDD375AF07FED597BA2EA561741BC27
:105FA000DD3AE22F0D2ACB0B2FF06D9564C8FEF57C
:105FB0007E7657F503FF000768FECB11C3FF000490
:105FC000BAD7FC47E07F0AFF00A45C7C48D33C6161
:105FD000E33B8B2FF968A9A6CFA6FDB654DDFED50D
:105FE0009C4C547FB4DD0B57F2FD401FD687ED2942
:105FF000FF0004C6B1FF0082C6FF00C10CBE0878D6
:1060000066EAF34ED17E2058F813C3FAFF0085F5F7
:10601000A96DC9B7B5D41B4A837C32ECCBADB4EAC9
:10602000C51F66ED9FBB9364862087F9C3FDA1BFA2
:10603000E0959FB4B7EC65E3F6B1F15FC23F887AB3
:1060400045E69F70BF65D574DD327BCB19A41F3246
:10605000B5BDE5BAB44EDDFE47DCB5FD757FC12B9D
:10606000256B9FF825FF00ECE0CCDB99BE17786B21
:10607000737FB5FD936D5F8ABFF07387FC161BF6C7
:106080008BFD9B3FE0A2E3E1BFC39F1CEB9F0E7C17
:1060900027E17D12C6F6DFFB29D22935A9AE23F30D
:1060A0005E795F692E81BF7423FB9FBA3C7CD4016B
:1060B000F1EFFC1C09E13B8F8ADE2EF831FB4E7FAD
:1060C00063DF68EFFB457826DA7F11DBDC5A496A2B
:1060D000D6BE26D2D534FD4E3589D4148BF7706CDC
:1060E000FEFF00CEFDEB93FF008374FF006C9FF872
:1060F00062EFF82B17C33D52F2E7ECFE1DF1A5D776
:10610000FC215ACFCEA8861D4196389DD9880A9188
:10611000DD2DACAE7FBB09AFA6BE287FC143F5EF36
:10612000F82F7FFC1243E227837E215BD95CFED0EF
:106130001FB38C2BF12B4DD4ECAD63B54F146870AD
:10614000116FAA33A8DB1C32410DC79CEB1E3CDF4C
:106150002A2D91FCAD5F90314AD1C9B97EF5007FFF
:10616000523F1FFF00E08DEDF023FE0E00F81BFBF9
:106170004C7C39D1E56F06F8DB5DBF4F1AD9595A0F
:10618000EE5D17569B4DBEFF004FF907C905CB7F4B
:10619000AC66FBB71FC5FE90AABFCE07EDC1A0C776
:1061A000E18FDB4FE306976ED249069BE36D6AD21F
:1061B000376FBCEA97D32AE7FEF9AFEC8BFE0949AB
:1061C000FB563FEDB7FF0004E8F843F13AEA6136C9
:1061D000A7E26F0F42355931B77EA10335ADE1FC1F
:1061E0006E6096BF963FF82F8FEC15E2CFD833FE46
:1061F0000A3FE3FB7F102C975A27C42D56F7C59E04
:106200001CD59136C37F69777324AD1FFD7685DC7D
:10621000C522F5E03636C886803D53FE09410D8E15
:10622000B7FF000441FF008289E9D75F332695E17B
:106230001BD58F9FBD1DF5DBA37FDF68B5F9A35F7D
:10624000B01FF06C5FECEB77FB647ECA5FB717C2E0
:106250001B1B8B5B2D43C7DE11D1ECACAE6E90B433
:10626000105C86D4BC96751FC22465E7F871F85798
:10627000E50FC52F869AE7C18F88DAF7847C4DA693
:10628000DC68FE24F0CDFCDA66A7613FFACB4B88D0
:106290005D9258DB1C7CAEA6803FB14FF837FF0003
:1062A000549B58FF0082367ECFB34EDB993C30B012
:1062B0002F6F9639A58D3FF1D515F88BFF0005C9D5
:1062C000FDA8359FF827F7FC1C95E28F895A2D8E83
:1062D0009BAC42FA6E92BACE897415ECFC49A5CFFC
:1062E000A5416B7B61748EAC8527843A72AC17E450
:1062F0007C6E5AFD9AFF00836DEF24D47FE0893FC6
:106300000164926F39974DBF8B27E6E1354BC55538
:10631000FC15715F88DFF078C786FF00B0FF00E0F2
:10632000ADB6575B7FE431E03D32EFFD5EDE97179F
:106330007075FE2FF55401F1CFFC14D7F63AD17FDA
:10634000654F8E1A76ADF0FF0050935EF831F15331
:106350004A8FC5FF000F3586C3349A5DC16CD9CE14
:10636000C19B179672ABDBCC84EF0D16E654DFB6FB
:10637000BE9FFF008364FF00E0ACDFF0EF0FDB2186
:106380007C17E30D516CFE13FC5A9A0D3B5492E1BD
:10639000D560D1350195B3BF2CDF71373F9329CA42
:1063A000AF972F98D9F214579BFF00C138F55B1FA8
:1063B000DBE7F66DF107EC77E27BAB187C51797780
:1063C000378B3E0B6AFA8491A0D37C4091E6EB4474
:1063D000F35F1E5DB6A70A600F35235BA8A27D920E
:1063E0003B8AF8835ED06F3C33AC5D69DA8DADC516
:1063F00085FD84CD6F736D711B452C12236D7474F4
:106400006E55811C8ED401FB05FF000793FEC65F0D
:10641000F0A7FF006E5F0B7C63D3EDF6E93F1774C6
:106420007FB36A2F966FF89AE9CB1C0CC78C206B50
:1064300046B30A3F88C329AF89BFE0883FB47E973F
:10644000FB37FF00C1483C03278A23B7B9F00F8F01
:10645000DE4F0178BED2E64D96B79A56AABF639436
:106460004FC8FDCA3C914CDFF5C2BEF7D3FF0069AF
:10647000F6FF0082D7FF00C1BA7E3AF00F88AE6106
:10648000BFF8E1FB26DBDA78AA092E275FB4EB9A86
:106490002D946F135E65F0EEE964D711CDF78B494B
:1064A00015BBB7CF70B5F8A1401EABFB6B7ECC3AE5
:1064B000A7EC5FFB5AFC45F855AD34D2DE78175E89
:1064C000BAD256E258FCB6BEB7493F7172179DABBF
:1064D00034262957FD99057D5DFB165927ED9BFF55
:1064E00000045EFDA27E0D33472F8B3E05DFC3F116
:1064F000B3C2D1E17CC96C523165ADA6F3C8863B0D
:10650000768A6D83EF49B293FE0B4771FF000D57FA
:10651000F06FF671FDAB206FB46A1F163C1EBE17FC
:10652000F1B5C6434B2F89B43D967717136D002103
:10653000B883C8745EBB23AF27FF008231FED656F6
:106540007FB1C7FC146BE1CF8935B9236F05EB77B9
:106550008DE17F15DBCF215B59F47D457ECB7266E3
:106560000BF7D225944FB7BB40B401F2AD7F6CDF7F
:10657000F0486FDAFCFEDD9FF04DEF84BF12AE2EC7
:106580000DD6B1AC6891DA6B523FDF7D4AD59AD611
:10659000ED8FA6F9A2771FECB8AFE3F3F6FCFD94FC
:1065A000F51FD883F6CEF895F0A7545B9593C13AC2
:1065B000EDC58DAC9709B5EEECF76FB4B8FF00B63A
:1065C000D6CF14A3FEBA0AFD9FFF0083287F6CB6C6
:1065D000920F8B1F00754B8F963F2FC6FA0C5B3DB9
:1065E0007CBB3BF05BFF00000AA7BCADEB401FBFCC
:1065F00054514500145145001451450014514500B3
:1066000015FC2C7EDC5A5FF607EDAFF182C7EE8BEE
:106610003F1B6B56FF00F7C5F4EB5FDD3D7F0F3F7F
:10662000F0544D3C697FF0531FDA2AD57EEDB7C494
:10663000EF12C4BF45D56E4500784D7EE47FC19D05
:106640003FF052FF00F857DF163C41FB34F8A352ED
:10665000DBA578D1A4D77C20653F2C1A9471FF006C
:10666000A55AAFFD7682312AFF000EEB77FE296B2B
:10667000F0DEBA2F865F1275AF839F11F41F167874
:106680006EFE6D2FC45E17D46DF56D32F623FBCB15
:106690004BA82459629173DD5D41A00FEF3757D2AB
:1066A0002D3C45A4DC595EDBC179677913433C136B
:1066B000209239E361865653C3291DABF9C8FDB456
:1066C000BFE0D3EF8C7E0CFDBCEF75AF807A3F87C7
:1066D000F58F84B73ABDB6B5A5C57BAEC36971A2C7
:1066E000A34A1E5B16597E774848F91FE726229970
:1066F0002CFBABF713FE099BFB73689FF051AFD8DF
:10670000A3C0FF0016B47FB3C337886C15358D3E28
:10671000190B7F64EA717C9776DCFCD85955B61664
:10672000E5E331BFF1D7D01401E0BFF051AFD82F6E
:10673000C23FF0526FD91FC51F0A3C631A476FACA6
:1067400045E7E99A9083CC9B42D42356FB3DE45D18
:106750003E6462770046F8DE48F215CD7F3B3F0C81
:106760007F618FDB27FE0DB0F8870FED2D7DE13FB8
:106770000EDF784F45B98F40F124363ABC5796FA70
:10678000A69D7332831CBB0799045249141B25DB59
:10679000F24DE4654F287FAA0AF3CFDA7FF678F04E
:1067A000F7ED6DFB3DF8CFE1AF8B2DFED3E1FF00A0
:1067B0001AE913E9377F20678048B859533FF2D26E
:1067C00036DB221FE174068038AFD93FF6ACF853B0
:1067D000FF00055BFD8F61F1778566B6F13780FCC0
:1067E00071613E93ACE917E8BE6DA33C7E5DD69B1C
:1067F0007D064EC902B9574E55D1C3AB3C7223B783
:10680000E09FEDC9FF000678FC6AF067C6ED4A6FAD
:1068100081779E1DF1A7C3ED46E1A4D3A2D5B5545F
:10682000B0D4F498CB65609FCCF925D830BE6A36D9
:106830005FAF969D2BE5DFD83BF6EEF8ADFF000687
:10684000F5FF00C143BC5BE1CD4ADEE352D1F47DEC
:10685000624F0FF8E7C31E6B25BEB50C1232ADCCEC
:1068600019E04CAA7CD825EEB263EE48D9FEB03FC1
:1068700065FF00DA87C13FB63FC0BF0FFC47F87B1A
:10688000ADDBEBDE15F12DB89ED2E623878DBA3C49
:1068900052A7549A37CA3A1E5585007F3AFF00F036
:1068A00055CFF82167ED316FE02FD9F7E1CF81BEE9
:1068B00015EB5F1034EF843E065D1353F1369935C6
:1068C000B4916A5A9DDDE5CDFDCC30234A27FB2CDF
:1068D0000F3F951C92C71F43F2AF19F56FF8371F92
:1068E000FE0DF9F8F5FB3E7EDDDE1BF8DDF17FC322
:1068F000ABF0FF00C3FE04B7BC9B4ED3AF6EE19F6D
:1069000050D62EAE6CE4B551E544EDE4C71A4EEE18
:10691000C642ADB9235D8D9629FD0C514018BE3B92
:10692000F02E8FF137C13AC786FC41A6D9EB1A1772
:10693000882C66D3752B0BA8FCC82F6DA68DA3964B
:106940001753F791D19948EE0D7F321FB5AFFC1A5E
:1069500029FB477873F68FF17DAFC25D27C3FE2513
:10696000F86FF6F925F0F5EDE6BF6F6B75F647F9B0
:10697000D22952560DE6479F299BA394DDFC55FD75
:1069800044D1401E1FFF0004DAF831AFFECE3FB005
:1069900007C1BF00F8B2DEDED3C49E0DF0869BA314
:1069A0006A90C332CF1C77105BA46E15C70DF32F0E
:1069B000515F26FF00C17E3FE082FA7FFC15BFC217
:1069C0003A3F8A7C27AAD8F85BE32783ED9ECAC2A8
:1069D000F2F91BEC1AE58EE690595CB202F1EC91EB
:1069E000D9E395436DF325528DBF747FA4545007AE
:1069F000F397FF0004E4FF008379BF69AFD84EEF3F
:106A0000E2F7C46F13784349D735687E1F6B1E19B0
:106A1000F0CF85748D66D6E67F12DFEA708B35F392
:106A200059DD214B485647965F325573B06C47AFDE
:106A3000853C31FF0006E7FEDA1E2DF13A69717CD4
:106A400009F1159CCEFB5A7BCBEB2B5B54E7058CF5
:106A5000AF384C7D0D7F63F45007CDBFF049AFD800
:106A6000AAFBFE09E7FF0004F6F867F08754BED3DF
:106A7000F50D67C2B632BEA77365B8DBC97973710D
:106A80002DD4FE53300591649D9558AA96503E55DD
:106A9000E95C87FC168FFE0965A1FF00C1573F63C3
:106AA0002D5BC172C76767E3AD07CCD57C17AC4DD2
:106AB000F2FD835009FEA5DD7E6FB34FC4728C30AA
:106AC000FB926D678A3AFB068A00FC6DFF008362C9
:106AD000BFE0905F1F7FE0987F19BE296A1F16B440
:106AE0004D2747D17C5DA2D95BDA7D8B58B7BEF3C9
:106AF000EE219E46F996363B708EFF009D1FF07189
:106B0000D7FC1BCBE23FF8282FC49D0BE2F7C0FD5A
:106B100037483F11AE8AE97E2BB0BBBA8ECA3D62C0
:106B2000DE38F6DB5EF9AF81E744A8216DDF7E3FFA
:106B30002B18F2BE7FD92A2803E45FF8218FEC9747
:106B4000E36FD86FFE0977F0D7E16FC44B1B3D3779
:106B5000C61E177D57EDD05ADDA5D469E7EA9777B1
:106B6000316244F95B31CC95F9F7FF00072B7FC107
:106B7000117F680FF8296FEDB5E11F1C7C29F0FE2D
:106B800089AB683A3F81EDB42B996F75B82CD92E3B
:106B900063BFBE9D9764841C6CB98FE61D7F0AFDA0
:106BA000BEA2803F943F0AFF00C1AB5FB71781BC14
:106BB0004FA76B5A2F867C37A5EB1A3DCC57B6579B
:106BC00096DE2FB38A7B5B88D95D24470F95756568
:106BD000C83DB15F46FF00C14D3FE0DC0FDA43F630
:106BE000CFF147837E31787BC07E0DF0F7C4CF1C98
:106BF000695FF173FC376FAEDA47670EBD03B44FC0
:106C0000AA5BC836C453508952E1E25CB45299374A
:106C10003C8CFBABFA2FA2803F99DFF827BFFC101A
:106C200053F6EEFF00827A7ED61E1BF89DA1FC3E35
:106C3000F07EB70E9AED67AD6832F8BECA2B5F12D0
:106C4000E973A94BBB09B3B9364B1E705D1F63F9DD
:106C50006FB18A579FFC76FF0083493F6A4D2FE34F
:106C60005F8B6DFC05E19F0FEA5E078759BB5F0FE5
:106C70005CDDF89ED22BA9F4FF0039FECCD2AB30FC
:106C8000C49E56CDDFED57F54545007F3D3F007F63
:106C9000E0DF7FDA7AE7FE0935F1BBF67DF1FF0030
:106CA000853C3F0EA1FF00090697E3DF86D2AF883F
:106CB000EDE6853588F75A5FC529473B7CDB13B67F
:106CC0003DFB503F24FA7C8FFF001095FEDA5FF405
:106CD00026F84FFF000ABB3FFE2ABFACEA2803F9A3
:106CE000E5FF0082A6FF00C1BD9FB4E7EDCB0FC159
:106CF0005F889A5F857C2E9F14A4F025A7877E2449
:106D0000DBBEBF6A9F68D4F4E3F67835269F84958E
:106D1000EEADBCAE23FF0057E405F7AF62FF008382
:106D200071FF00E0DEFF008C3FF04F3FDACB54F8FC
:106D3000B9F182E741D1DAD741B8D2349D174AD4AC
:106D40007ED93DC493C91EF9A774FDD88D523F95D5
:106D500032DB99C37CBB3E6FDB8A2800A28A280005
:106D6000A28A2800A28A2800A28A2800AFE21FFE79
:106D70000ACF0B5AFF00C153FF006950DFF454FCE7
:106D80004CDF9EAD726BFB78AFE28FFE0B4FA7FF1F
:106D90000065FF00C15ABF68D8FF00BFF10B5897CC
:106DA000FEFBBA77FF00D9A803E5FAD4F0C785F552
:106DB0000F1A7886CF49D22C6F355D4F51996D6D82
:106DC0002CED2069AE2EA573B523444C97727A0141
:106DD000D6B2EAD58DF4DA75E45716F2C90DC42E91
:106DE000AE8E8FB59187420D007F411FF069F7C2CB
:106DF0003FDA9BF639F8BDE28F05F8FF00E0EFC4FB
:106E00002F0E7C1EF1D5B7F693DDEBB62DA6A68529
:106E1000AAC31FC932C139593F7F12F9326D4DDB08
:106E2000A3B7CE152BF7AABF967FF82517FC1D5DDB
:106E3000F16BF6327D37C23F18FF00B4BE327C36AC
:106E400087F771DC5CDC6EF12E8D1E7FE595CBB68D
:106E50002E907CDFBAB8F9BEE0596355DA7FA26F95
:106E6000D88BFE0A0FF08FFE0A23F0C7FE12AF8404
:106E7000FE32B0F12D9C3E5FDBECFF00D46A1A5469
:106E80008E388EEADDB1246DC36091B1F076B32FF8
:106E90003401EE54515CBFC5CBDF18D87816FA6FB9
:106EA0000269BE1BD63C4E9B7EC76BAEEA7369B6C9
:106EB000121DDF37993C305C489F2FA44D401F8046
:106EC000BFF0798FFC13D23F0A7C47F07FED29E1B8
:106ED000DB158ED7C51E5F85BC58624C66F628D878
:106EE000D95CB1EED25BC6F0313C28B3B71D5EBEB3
:106EF0001CFF008214FF00C16BFC4DFF000497F8DB
:106F0000F7F65D4E4BED7BE0D78C2E1478A342470D
:106F1000DCF66FF71752B30785B98D7EF2FDD9E322
:106F20001B1BE658A48BF46FFE0BA3FF000594F81F
:106F3000ADE1FF00D9CBC73F03BF685FD8AAFBC252
:106F4000FA2F8EEC1AC34BF11C3E3B37BA4FDB17BE
:106F5000F7B6B756D711E9FE54B2433451CFE479AE
:106F600088FB536BAAEEAFE7B6803FBB6FD9B3F691
:106F7000B1F86FFB607C39B7F16FC31F1A683E36FA
:106F8000F0FDC6DCDD69B74B2790C7FE59CB1FDF8C
:106F9000864FFA6722ABFB57A357F097FB337ED699
:106FA0005F11FF00637F89D67E30F85FE32D7BC1E0
:106FB0003E22B5DBFE95A75C6D59D41DDE5CD13653
:106FC000639E3CF58E55646EEB5FBA7FF04D2FF8F3
:106FD0003C9745F10A699E16FDA73C38DA1DE7C9C2
:106FE00007FC26BE1CB7696CE4EDE65E588CC91739
:106FF0001CB3DB799B98F10C6B401FBC34578C7C25
:1070000038FF008284FC0AF8B7A3DADF7873E3273D
:10701000C2FD620BE8BCD885BF8A2CDA4DBB437C2D
:10702000C9E66F561DD586E5EF8AF50F0EF8E345E4
:10703000F17C1E7693ABE9BAA45B55B75A5D24EB9D
:1070400083D3EE93D68035E8A28A0028A28A00284E
:10705000A28A0028A28A0028A28A0028A28A0028E0
:10706000A28A0028A28A0028A28A0028A28A0028D0
:10707000A28A0028A28A0028A28A002BF8C1FF0059
:1070800082F9699FD95FF058EFDA121FEF78B6697D
:10709000BFEFE471BFFECD5FD52FFC149FFE0AA3A6
:1070A000F0CFFE0957F0CB49F15FC4EB7F18DD69E3
:1070B000FAEDCC96361FD87A1C979E7DC22093C9D4
:1070C000698ECB786574DC5165950C822976E7CBA7
:1070D0007DBFC917FC1553F6ADF0DFEDC7FF000506
:1070E00002F89BF167C23A76B5A5F877C6DA8C77D5
:1070F0009656BAAC71A5E46AB6F1447CD58E4910B7
:107100003168D8FCAEDD7AD007CF3451450015DEAA
:10711000FC00FDA33C75FB2A7C52D37C6DF0EFC5CF
:107120007AD7837C55A53EF8350D32E0C5285C86BC
:1071300031B8E9246D8F9E37DC8E3E56522B82A2E9
:10714000803FA2EFF82567FC1E03E1BF883FD9FE10
:107150000FFDA7F4FB7F096B2C3CA8FC6DA3DB485B
:10716000FA5DE363E5FB5DAAEE92073FF3D22DF1F2
:10717000EE3F721415FB307E32E95E2EF81F75E388
:107180007F046A3A2F8D34D934B9B52D2AEB4DD40A
:10719000A3B8B1D57646CC9B2E23DC9B188C6F19F7
:1071A000AFE0E6BDEBF623FF008293FC69FF0082AF
:1071B0007978BE4D4FE1578EB56F0FDADE331BFD88
:1071C00021F6DD693A96576B79F6728685DB67CBD7
:1071D000BCAEF5FE161401FD7A7EC65FB5A7C27F70
:1071E000F82BDFEC5163E2FD374FD13C51E10F1535
:1071F0005BFD83C43E1AD5E086FD34DBB45469F4EC
:10720000EBC8245D8CD19656F9970E8639172AEA79
:107210006BF3B7FE0A1DFF000674FC2DF8DDA8CF46
:10722000AFFC03F124BF09F5899F7CBA16A1E66A79
:107230005A14B9EBE53126E2DB9F9BEF4A9FC2B1BE
:10724000A0AFC73FF822F7FC15D7C45FF0496FDA4B
:107250009D3C456915E6ADF0E7C50D1DAF8BFC3DC6
:107260006F2FCD776AA5B64F087213ED506F668CFD
:10727000B63765D0B2AC8587F559FB1E7FC14CFE91
:1072800004FEDE7E17B1D43E17FC4AF0CF88AEAEC6
:10729000A1F39B4837896FAC5A751B67B37C4F1FAE
:1072A0002A792BB5B1F2965E6803F9CDF8BFFF00DD
:1072B00006817ED81F0D6D5A6D0ECFE1CFC42F48C9
:1072C000F42F122DBC9FF93F1DB2FF00E3D5E03A29
:1072D0008FFC1BE5FB66E97E306D065FD9FF00C6BB
:1072E000AF7CBD6484DACB67FF0081492983FF004E
:1072F0001FAFECC28A00FE447C27FF0006B1FEDB14
:10730000DE29BA8D27F84963A2C322861717FE2CFF
:10731000D1F68CFAAC572F27FE3B5EC5E10FF83350
:107320001FF6AAD7628A5D4BC4FF000634256FBFE3
:107330001DC6B97D2CC9F84564CBFF008F57F519E0
:1073400045007F3BFE01FF0083337E357847459A39
:10735000E21FDA33C3BE1FD5A18A436F0E93637D4C
:10736000E53B91F75A51246501E324237D2BE6DFA9
:10737000DA77FE099FFF00052EFF00827BACD7362F
:10738000BE24F8D1E24F0EDBED1FDAFF000EBC6920
:10739000A9EA76FB635DDB9A085D6EE348D7F8E502
:1073A00081117D6BFAB2A2803F91DFF8258FFC1C22
:1073B00027F1BBF629FDAFF49D67E2B7C45F895F93
:1073C000147E1CEA0FFD99E26D1FC45E21BCD5A599
:1073D000B4B766E6EAD16E246D9730B7CFB46DF3DB
:1073E000177C6DB77074FEB13E1AFC45D0FE2F7C41
:1073F0003FD17C55E18D52CF5BF0EF882CE3D43444
:10740000DD42D1F7C1796F22EF4910FA1522BC7322
:10741000F6BCFF00825DFC00FDBBACEE7FE1687C4A
:107420002BF09F89352B98FC9FED7FB27D97568D71
:1074300076E176DE43B67F97B0DFB6BF333FE09AA2
:107440007F1EFC59FF000417FDBEEE3F62FF008D5A
:107450009AB5C5DFC17F1C5E49A87C25F17DE37F1D
:10746000A3C0F713165B676E91ACB23149138F2A34
:10747000E8EFC79773E6D007EDA514514005145106
:107480004005145140051451400514514005145154
:107490004005145140051451400514514005145144
:1074A00040051451401E5BFB5FFEC9BE0DFDB8BF19
:1074B000673F14FC2FF1F69EDA97867C5169F679C6
:1074C000F66D59ED5D4868AE2172A424D1BA8746A5
:1074D000C1F9BD46457F19FF00F0519FD817C67FFF
:1074E000F04D3FDAC7C47F0ABC6D179971A5B7DAB2
:1074F00034CD4D2031DBEBBA7C85BC8BD8B39F9566
:10750000F6B06196D9224899DC86BFB82AF843FEC6
:107510000BCDFF00047ED27FE0ABBFB28CD69A4C7D
:1075200016B63F16BC12926A1E0FD4DF6A2CEE7E8E
:107530006974F9D8FF00CB19F6819FF967208DFE99
:10754000E874700FE3CA8AD8F19783354F871E2DF0
:10755000D5341D734EBCD235CD12F25B0BFB0BC87C
:107560001A1B8B2B889DA3962951B9474752ACA76C
:10757000906B1E800A28A2800A28A2800AB5A76AFA
:10758000571A25FC5756B3496D756EEB245344E5E5
:107590005E361D1948AAB45007E847EC3DFF0007C6
:1075A00033FED55FB15A5A69B2F8D23F8A1E15B67A
:1075B000F9068FE3446D45917E51FBABC0CB7698C5
:1075C00045C2832B46BFF3CCD7F461FF000467FFAD
:1075D0000082B3697FF057DFD9B754F1C59783753F
:1075E0002F03DF7877596D1751B09EEC5FC1E70824
:1075F000A39834370113CC5D92AE7722B2FBFDE342
:10760000FC65C7234122B2B6D65F99596BF413FECD
:10761000097DFF00070AFED15FF04FE97C3FE0BF24
:107620000DAE8DE3EF02FDB9553C2175A3429717CE
:10763000D2CD2287F2AEADE3173F6993EEAB486639
:107640001B88FDDBF4A00FEBD28AF38FD96FE37DAB
:10765000E7ED21F00FC33E36D43C13E31F87379E7E
:1076600020B632CDE1BF1458FD8F56D2A459191956
:107670002688F233B7729382C855B6AFDDAF47A004
:10768000028A29AEEB0C7B9BE555A00757E56FFC02
:107690001DB77BF03E3FF8269FD9FE27498F1F4B31
:1076A0007FBFE1BA5918FF00B51B505DBE795CF38E
:1076B000F63F2987DA33F27307FCB5F22BF52AD2AD
:1076C000FE1BFB7F3619A39A3FEF44FBD78FA57CA7
:1076D00083F1A3FE0865FB3F7ED27FB6F5C7C78F57
:1076E000893A1EB5F113C47259DBDAC1A1788B5502
:1076F00092F7C3B61E47DD78ACDB8DA79DD0C8CF0F
:107700006E4BBB795BD8B500785FFC1B0DFF0005A5
:107710002EF881FB76FEC70DE1FF0088DE1FF165C4
:10772000C6B3F0E522D3ED3C69756327F6778AECA2
:10773000C6E8D3FD29B896F61D9B26FE261E5BB62D
:107740005DA4C7E9D567E85A259F86747B6D3B4FDA
:10775000B3B7B1D3EC61582DEDA0458E28235185E8
:107760004441C2803B5685001451450014514500E8
:107770001451450014514500145145001451450061
:107780001451450014514500145145001451450051
:10779000145145007E127FC1D87FF04556F1DE8935
:1077A000A87ED4DF0C747964D6347B65FF008587AE
:1077B000A5DA47BBED96B1AED4D595473BE141B6CE
:1077C0007EDE50493E5F2A567FE77ABFBA8FDB07DD
:1077D0004CF8ADAB7C0BD52DFE0D47F0DAE3C713AB
:1077E0006D4860F1DC37726897309E254945A912D3
:1077F00072BD3A8AFE397FE0A11FF04F7F8DDFB165
:1078000027C54D5A4F8AFF000A2E3E1F5AEB9A8C0D
:10781000F359CBA7C1E6F87C991DA416F67728D2B8
:1078200047B157EEC5E6191500DD401F38D14514A4
:10783000005145140051451401EADFB237EC6BF1F9
:1078400023F6EAF8C3A7F813E18F85F52F13EBD7DA
:10785000EE9BFC88DBECF631B36D33DC4BF7218417
:1078600067977E2BFAAEFF00822DFF00C107FE1D39
:10787000FF00C125FE1E26A922D9F8CBE316B56E5E
:10788000175BF14CD07CB6AA7AD9E9EADCC36C3F2D
:1078900089BFD64C7E67C2F97145E0DFF06767EDBE
:1078A0000FE1BF8A1FF04DCD63C1165A6E8BA6F84B
:1078B000B3E1AF8825B6D59AD2DA38EEB52B5BB6F0
:1078C0007B8B3BAB8651977DDF69814B7F0DA8AFEA
:1078D000D69B989A6B6655924859976875DBB93D67
:1078E000F9C8A00E2FC65F1FBC3BE19F176A9E150B
:1078F000B6BB87C41E3ED33C3F378A23F0869B7BB2
:107900006FFDB77F628FE52C91412CB18DAF37EEC3
:107910005249192332705D6BE09FD8EFFE0B55F191
:107920002FFE0A85FB71CDE16F807F0E349B5F8255
:107930003E10FB0DC78B7C6BE2E86EE3BDB712C255
:10794000924FA7456A8C8897CB279B08F9E58FF75C
:10795000465F9936EEF4CF897FF06EBFECADF17BD8
:10796000C45AA788BC47E10F186ADE35D6B73DF781
:107970008A6E3C73ADCBAB5DC842AF98F235D15641
:107980002022ED5D9B171F2AD7CEFF00F0552F8ACE
:107990006DFF0004C2F809F08FF62DFD8F747B7F18
:1079A0000DFC51F8E178FA6E9D3DA5C335EE876771
:1079B0002C8A971AA4D37CD2ACF33B37FA5367CB0B
:1079C000482E1D4A98536807BF7ED75FF0579D52D7
:1079D000E7F6859BF67EFD967C2565F19FE3C5BCA9
:1079E000BE4EB93DC4CD1784FE1F46ADB659B56B2A
:1079F000A461B9D1BE5FB3C4DBF7064DC25090C9D4
:107A0000D8FC10FF0082676A9E21B8B1F147ED2DC6
:107A1000F12BC41F1EBC6CA7CD3A5DC7FC4B3C13B9
:107A2000A537CF88EDB45876DBCFB15F679D782658
:107A300091F607FDD9E075FF00F04C9FF8270F8005
:107A4000FF00E097DFB3469BF0FF00C1B0FDA6FA50
:107A500042B75E21D7A58C2DE7892FCAFEF2797A2D
:107A6000ED5ED1C79C469C7277337D214015EDEDCC
:107A7000E3B2B748E3448E28D76AAAFCAA8A2AC58B
:107A8000145001451450014514500145145001454E
:107A9000145001451450014514500145145001453E
:107AA000145001451450014514500145145001452E
:107AB00014500158FE36F0468FF11FC2B7FA0F88F6
:107AC00034AD375CD135585ADEFB4FD42D63BAB58F
:107AD000BC88F58E589C14743E8456C51401F90771
:107AE000FF000511FF0083433E09FED232DF788399
:107AF000E0CEA775F05FC5570ED31D39636BFF004D
:107B00000EDD485998FEE19BCCB6C96C7EE5FCA41D
:107B100051F2C35F861FF0503FF822C7ED11FF00FE
:107B200004D8BABABAF88DE03BA9FC290BED4F1581
:107B3000E879D43427CB2AAEE9D17741976DAAB73B
:107B40002B13B765AFED2EAB5ED943AA594904F1AB
:107B5000C735BCCA637491772BA9E0A906803F8022
:107B6000CA2BFA84FF0082CF7FC1B15F0A7F687F92
:107B7000829E2AF1B7C07F04D9781FE2EE976CD7B6
:107B8000F69A5688C2D749F11B47F33DAFD97FD546
:107B900043348A088DE2F2D7CCC6FEA587F30DA93F
:107BA00069B3E917D35ADD4325B5D5B3B452C52A15
:107BB00015911C1C15607A30A00A945145007D1D5A
:107BC000FF0004E8FF0082A0FC5AFF00825C7C5C9E
:107BD000BAF177C2BD5B4CB76D5A04B5D5F49D4E72
:107BE000D05DE9BACC28DB92399372BAED6E43C40A
:107BF000F1C839F9F6B303FB85FB2D7FC1E89F0877
:107C00003C5BF0FAE9FE307803C61E0DF14585BEF7
:107C1000F58FC3A23D5AC75561FC3117689A173FCB
:107C2000DD93E51FF3D2BF9D0F871F0BBC4DF19372
:107C3000C6567E1DF08F87B5CF157883517D96BAD5
:107C4000668F6135F5E5DB7FB1144ACEFF0080AF6A
:107C5000D5BFD837FE0CFDF8EDFB40C563AD7C61A8
:107C6000D6749F833E1D94249FD9EE1756D7A78CB8
:107C7000EC6FF511B8860DCAC47EF25F3236FBD0C8
:107C8000F6A00E93F6DFFF0083CB3E307C566B8D63
:107C90002FE06F84B45F859A4E76A6B3AA226B3A22
:107CA000D3E1810C88EBF65873FC48D1CDECF5CFCD
:107CB000FF00C1107F64BFDB53F69DFF008298FC7C
:107CC0002BFDA7BC43A378D35ED0F45D4E27D43CF4
:107CD0005FE3DBF9225BCD22E239209C597DA4F9D8
:107CE000B709F66B99FCAF213C90DF2EE4AFDA0FB9
:107CF000D83BFE0DF3FD987F6026B1D43C3FE02BCE
:107D00007F1778BACF6BAF897C59B754BF8E45DAED
:107D100056585594416CE08E1E1891FF00DAAFB7AB
:107D20002800A28A2800A28A2800A28A2800A28A03
:107D30002800A28A2800A28A2800A28A2800A28AF3
:107D40002800A28A2800A28A2800A28A2800A28AE3
:107D50002800A28A2800A28A2800A28A2800A28AD3
:107D60002800AFE72BFE0ED4FF008237AFC29F1B67
:107D70004BFB50FC3AD1FC8F0E789EEC45E3FB5B4D
:107D80005876C5A6EA52B2AC5A9617854B976092C0
:107D9000B71FE9051BE67B838FE8D6B9DF8A5F0C46
:107DA000741F8D1F0DF5CF0878A34CB7D63C3BE26E
:107DB0006B19B4DD4EC6E06E8AEADE55D8F1B7D550
:107DC0004D007F04B5B5E1BF03EADE29D135AD43EF
:107DD0004FD3EE6F2CBC3B6AB7DA94D147B96CA194
:107DE00069A381647FF64CB2C4BF57AFA5BFE0B0B2
:107DF0003FF04C6F107FC12AFF006C9D67E1EEA43D
:107E00002EAFBC2B7E5B52F09EB5328C6ABA6BB73C
:107E1000C9B99703CF88E629570BF3A6E0363A1382
:107E2000F537FC1AE7FB165A7EDB1E2CFDA8FC2357
:107E3000A93470E9BE24F84D73E16FB4CA9BD6C66D
:107E4000EAF6EE092DAE36FF007A292CFCC1EE943D
:107E500001C67FC1A87F122F3C0BFF0005ABF87F46
:107E6000A6DAC922DBF8C348D6B48BC0B9F9E14D14
:107E70003E7BC5071FF4D6CE235FD6CD7F2CBFF047
:107E800069EFECDFA95A7FC16E6FECFC4563369752
:107E9000AF7C23F0DEB9777B6571F2CB6974B245B4
:107EA000A54B130FEFA9BC71F81AFEA6A800A28A71
:107EB0002800A28A2800A28A2800A28A2800A28A72
:107EC0002800A28A2800A28A2800A28A2800A28A62
:107ED0002800A28A2800A28A2800A28A2800A28A52
:107EE0002800A28A2800A28A2800A28A2800A28A42
:107EF0002800A28A2803E31FF82DF7FC12BB48FFD5
:107F00000082AEFEC67A9785238ECED3E21F864CC2
:107F1000BAAF82F53987FC7BDF05E6D5DFAAC170F1
:107F2000A0472765223936B189457E78FF00C19682
:107F30001F0675CF8597BFB5347E24D26E347D572A
:107F40004DD5F44F0EDD5ADD46639EC6F2D3FB538A
:107F5000ED56EEA7EEB23488187622BF772B83F861
:107F600073FB3EF84FE13FC43F1D78A3C3FA42695B
:107F7000DAC7C47BF8353D7A6590E2FAE61B78ED06
:107F8000524DB9C21F2E24076E371F98E4D007C97F
:107F9000BFB1BFFC139EDBF66CFF0082D37ED3DF44
:107FA00016ACF4D92D747F895E1CD0B50D3674875C
:107FB0006DBFDAAEA6BBFED48F77FCF433D8C13BDD
:107FC0007FD7D8AFBBA8A2800A28A2800A28A280A7
:107FD0000A28A2800A28A2800A28A2800A28A28051
:107FE0000A28A2800A28A2800A28A2800A28A28041
:107FF0000A28A2800A28A2800A28A2800A28A28031
:108000000A28A2800A28A2800A28A2800A28A28020
:108010000A28A2800A28A2800A28A2800A28A28010
:108020000A28A2800A28A2800A28A2800A28A28000
:108030000A28A2800A28A2800A28A2800A28A280F0
:108040000A28A2800A28A2803FFFD90062B38B07CA
:1080500008D0521E11F8013B00F8013B00F02480CB
:108060008B07F6D1830740F0208000BF103A07D37A
:1080700030B4B1E83810103AA0E83810F9D230BC6A
:10808000530724BFB1E80810A0E8081044BF51F816
:10809000043B40F8043BD20724BF31F8022B20F800
:1080A000022B44BF0B7803707047083A07D3B1E83E
:1080B0000810083A40F8043B40F804CBF7D25307C5
:1080C000E4E750F8041B61B150F8042BD30744BF18
:1080D000A9F101039A18002342F8043B091FFAD1C1
:1080E000EFE7704730B583B00121042004F088FC2D
:1080F0001020009003208DF8050001208DF8040069
:108100000020ADF8060000A9DFF8F04A204602F092
:108110001FFA0121022004F073FC0120009000A945
:10812000DFF8DC5A284602F013FA0121042004F09B
:1081300067FC01208DF8070000A920200090204650
:1081400002F006FA00F062F90021DFF8B80A02F046
:108150005FFA00F00FF8DFF8B00A00218160F0212B
:1081600001804FF4A071418001210171002000F0D5
:1081700086F937BD10B5DFF8844A2021204602F089
:108180002EFA0A2002F07AFB2021204602F025FA7E
:10819000012000F00FF9642002F070FBCB2000F00A
:1081A00009F9392000F01AF92C2000F017F900F035
:1081B0000DF9342000F012F9022000F00FF9CF2061
:1081C00000F0F8F800F002F9C12000F007F93020C3
:1081D00000F004F9E82000F0EDF8852000F0FEF84A
:1081E00000F0F4F8782000F0F9F8EA2000F0E2F866
:1081F00000F0ECF800F0EAF8ED2000F0DBF8642085
:1082000000F0ECF8032000F0E9F8122000F0E6F8A6
:10821000812000F0E3F8F72000F0CCF8202000F0F7
:10822000DDF8C02000F0C6F8232000F0D7F8C12008
:1082300000F0C0F8102000F0D1F8C52000F0BAF826
:108240003E2000F0CBF8282000F0C8F8C72000F04E
:10825000B1F8862000F0C2F8362000F0ABF84820D4
:1082600000F0BCF83A2000F0A5F8552000F0B6F870
:10827000B12000F09FF800F0A9F8182000F0AEF847
:10828000B62000F097F8082000F0A8F8822000F04F
:10829000A5F8272000F0A2F8F22000F08BF800F0FB
:1082A00095F82A2000F086F800F090F800F08EF89B
:1082B00000F08CF8EF2000F091F82B2000F07AF815
:1082C00000F084F800F082F8012000F087F83F20E9
:1082D00000F084F8262000F06DF8012000F07EF810
:1082E000E02000F067F80F2000F078F8312000F06F
:1082F00075F82B2000F072F80C2000F06FF80E20BB
:1083000000F06CF8082000F069F84E2000F066F8E4
:10831000F12000F063F8372000F060F8072000F04B
:108320005DF8102000F05AF8032000F057F80E20F6
:1083300000F054F8092000F051F800F047F8E1206F
:1083400000F038F800F042F80E2000F047F8142052
:1083500000F044F8032000F041F8112000F03EF84E
:10836000072000F03BF8312000F038F8C12000F081
:1083700035F8482000F032F8082000F02FF80F20E0
:1083800000F02CF80C2000F029F8312000F026F83D
:10839000362000F023F80F2000F020F8112000F024
:1083A00009F8322002F06AFA292000F003F8BDE84B
:1083B00010402C2038B5044600F0A0F900F020F859
:1083C00000F019F82846BDE8344004E0002005E03C
:1083D0005046BDE8F44F012102F0FFB838B504461D
:1083E00000F091F900F00CF800F005F8044600F0F8
:1083F0000DF8204632BD2146DFF8080802F024B906
:10840000DFF8FC570121284602F0E9B8012128468F
:1084100002F0E3B810B514460B46024600F00BF824
:108420002C20FFF7C7FF2004000EFFF7D7FFE0B2B4
:10843000BDE81040D2E7F8B504460D4616461F4683
:108440002A20FFF7B7FF200AFFF7C8FFE0B2FFF7C7
:10845000C5FF300AFFF7C2FFF0B2FFF7BFFF2B20C6
:10846000FFF7A8FF280AFFF7B9FFE8B2FFF7B6FF4A
:10847000380AFFF7B3FFF8B2BDE8F240AEE770B5D7
:108480000446DFF88407418800884B1E421E2504FD
:108490009BB292B200210020FFF7CDFF2C20FFF706
:1084A00089FF4FF49636280EFFF798FFE0B2FFF7EA
:1084B00095FF761EF7D170BD38B5044600F00FFB6E
:1084C0004FF4A0752CB95820FFF788FFF020012148
:1084D00013E0012C08BF8820F6D0022C05D100F053
:1084E00051FC4CBF6820A82002E0032C02D1E820F8
:1084F000FFF774FF2846F0250021DFF8442A1171A8
:108500001080558031BD2DE9F043DFF8346A83B027
:108510008846A6F8088070810A9F0B9C15469946EC
:1085200001E030816D1C95F90000D0B171890A28F5
:108530000CD199F80100401C4018708195F9010098
:108540000D2806BF00206D1C4046EAE70D28E9D043
:108550000194009715F9012B30894B4600F003F880
:10856000E1E7BDE8F7832DE9F04F93B006461D988B
:10857000DFF89456DFF88C86DFF8C8991D908B469B
:108580001C46202A2ED100F0AAFA99F8780100069C
:1085900054BFA8206820FFF721FF607821781D9A3A
:1085A000ADF8002010FB01F75BFA80F0431E56FA8D
:1085B00081F0421EBFB200F097F800F09FF800F083
:1085C00098F82C2100F009FB00F09DF8002606E049
:1085D0009DF8011000F001FB00F0FDFA761CBE4290
:1085E000F6DB69E0617800200AE06768A2F1200309
:1085F00001FB030337F8133002AF27F81030401C9B
:108600008842F2DB2E81A5F80AB03146227828880C
:1086100012FA81F1884205DA61780BEB010068817A
:108620000020288100F05BFA99F87801000654BF19
:10863000A8206820FFF7D2FE6078217810FB01F2B5
:1086400092B25BFA80F00192431E56FA81F0002745
:10865000421EBA4600F048F800F050F800F049F821
:108660002C2100F0BAFA00F04EF81C9EBB460FE039
:1086700020780AF1010A824504BF7F1C4FF0000AEE
:108680009DF8011000F0A9FA00F0A5FA0BF1010B1A
:108690000198834510DA6078C01B02A901EB400005
:1086A00030F8020C00FA0AF000044EBFADF800608A
:1086B0001D98ADF80000DBE70121DFF8440501F06B
:1086C0008CFF00F00CFA99F87801000601D4A8207C
:1086D00000E06820FFF782FE2889217850FA81F0B7
:1086E000288113B0BDE8F08F9BB292B25946304654
:1086F000A1E6DFF80C05012101F071BF1021DFF8C0
:10870000FC0401F06CBF1021DFF8F00401F065BF3C
:108710002DE9F84F0446DFF828080E460188154673
:108720001F468C4228BF4C1E8D4228BF4D1E4088DC
:10873000864228BF461E874228BF471EA4B2ADB25C
:10874000AC4234BF281B601BB6B2BFB20FFA80F830
:10875000BE4234BFB81BF01B0FFA80F94FF0FF3B4D
:10876000AC423ABF01200090CDF800B0BE4238BF05
:108770004FF0010BC145B4BF4046C9F1000000EB0A
:10878000D0704FEA600A0A980A900EE00FFA8AFA4F
:108790005046C8F10001814203DA0099AAEB090AA8
:1087A0000C194845BCBFC2445E440A9AB1B200F0FD
:1087B000EDF8A4B2AC4204BFB6B2BE42E6D1BDE809
:1087C000F18F2DE9F04182B00446089F0D46164610
:1087D000984605E000972B46324600F006F86D1CDF
:1087E000ADB24545F6D3BDE8F381294620468FE773
:1087F0002DE9F84306460F4614461D4600F06FF972
:1088000000F0F5F954BFA8206820FFF7E7FDA01B92
:10881000E91B01FB00F96B1E621E9BB292B2394646
:108820003046FFF708FEDFF8DC6B1021304601F020
:10883000D6FEDFF8CC73012100F05BF9DFF80847C2
:108840002C21204601F000FF1021304601F0C5FE2A
:108850000898089000260AE09DF82110204601F0B3
:10886000F3FE9DF82010204601F0EEFE761CB14587
:10887000F2DA012100F037F900F031F998F87801C7
:10888000000654BFA8206820B2E02DE9F34F15463A
:1088900081B06800C0F1000B9846C5F10109691864
:1088A000BDF804000FFA89F94FF0010A002442468E
:1088B00089B2FFF7AFFDBDF90800411BBDF8040008
:1088C000424689B2FFF7A6FDBDF90400BDF80810C5
:1088D0002818424680B2FFF79DFDBDF90400BDF89F
:1088E0000810401B424680B23FE00FFA89F0002892
:1088F00004D4681E0BF1020B05B2D944601C04B20B
:10890000BDF904002018ADF800000AF1020ABDF913
:1089100008002F18BDF80000D14400F032F8BDF96E
:108920000400061B00F027F8BDF90800471B00F003
:1089300026F800F020F8BDF904002818ADF8000072
:108940004246BDF908002718BDF8000000F01AF8EB
:10895000BDF90400461B00F00EF8BDF90800071B26
:1089600000F00DF84246B9B2B0B2FFF753FDAC4289
:10897000BBDBBDE8F78F4246B9B2B0B24AE5BDF8FD
:1089800000004246B9B245E5424689B2A0B241E58F
:108990002DE9F84304460D46174600F0A0F800F014
:1089A00056F854BFA8206820FFF718FDBBB2AAB242
:1089B00000F088F800F09AF800F0A2F800F086F8CD
:1089C00000F090F808E09DF8011000F082F89DF8A2
:1089D000001000F07EF8641CAC42F4DB00F08CF870
:1089E00000F07DF896F87801000654BFA8206820B2
:1089F000BDE8F243F2E42DE9F84300F06DF800F031
:108A000026F854BF8C204C20FFF7E8FC00F057F804
:108A100000F06CF800F074F800F058F800F062F81C
:108A200008E09DF8011000F054F89DF8001000F0E7
:108A300050F8641CAC42F4DB00F05EF800F04FF834
:108A400096F87801000654BFA8206820D0E7DFF828
:108A5000F46496F87801000670472DE9F84300F0B9
:108A60003BF8FFF7F4FF54BF8C204C20FFF7B6FC17
:108A700000F025F800F03AF800F042F800F026F88F
:108A800000F030F8FF2100F024F8FF2100F021F879
:108A900008E09DF8011000F01CF89DF8001000F0AF
:108AA00018F8641CAC42F4DB00F026F800F017F86C
:108AB00096F87801000654BFA820682098E74FF484
:108AC000A0731A46B9B2A0B2FFF7B5BCDFF878942C
:108AD0002C21484601F0B8BD07460C461546362005
:108AE000FFF768BC1021384601F077BDDFF8147934
:108AF0001021384601F073BD0121404601F06DBDE3
:108B0000DFF804890121404601F069BD2DE9F047F5
:108B10002DED028B054682B00F4616469946B0EE03
:108B2000408AF0EE608AFFF7DAFF00F04EF854BF9B
:108B30008C204C20FFF752FC4FF4A0731A46A9B2C8
:108B4000B8B2FFF778FCDFF8B4A0102100F065F9A7
:108B5000FFF756FCDFF8F0832C2100F03EF81021DF
:108B6000504601F03AFDF01B86B200271AE0384665
:108B70000FF08EFA53EC182B0FF0CEFA0FF0A0FA8C
:108B8000C0B2323080B2FF28C8BFFF2039F81000D1
:108B9000ADF8000040469DF8011001F055FD00F0D1
:108BA0001AF87F1CB742E2DBFF2100F016F8FF2124
:108BB00000F013F8FFF72AFCFFF791FF94F8780113
:108BC000000654BFA82068200AE0DFF8784394F834
:108BD0007801000670479DF80010404601F034BD52
:108BE00002B0BDEC028BBDE8F047FFF7F7BBDFF842
:108BF000548398F87801000670470000000802408E
:108C0000000402400030014078DC01202DE9F04FE3
:108C1000DFF8F867044630699B4685B088461746FA
:108C2000584506D01022002130460FF046FBC6F80A
:108C300010B01022002101A80FF03FFB3A46DFF8E8
:108C4000D01701A801F02CFE0027FFF748FF00F025
:108C500099F854BFEC202820FFF7C0FBB948DDF895
:108C600038A090F8780130210DF1040908423D4602
:108C700037D115F90920302A08BF002F01D1012D65
:108C800020D1A857904208D0CDF800A05B464146BD
:108C9000204600F0C5F800F065F801272034012DCA
:108CA00008BF241D6D1C052DE3DB261D002700F0E9
:108CB00061F84146304600F06AF814367F1C032FF5
:108CC000F5DB35E0A857904201D12034EAE7CDF832
:108CD00000A053464146204600F0A2F800F042F8BA
:108CE000F3E715F90920302A08BF002F01D1012D23
:108CF00026D1A857904206D0CDF800A05B4600F0E0
:108D000035F800F02FF801272334012D08BFA41CEB
:108D10006D1C052DE5DBA61C002700F02BF8A8F143
:108D20000201304600F0E0F812367F1C032FF4DB1E
:108D3000FFF7D5FE00F026F854BFA82068200CE00D
:108D4000A857904201D12334E2E7CDF800A0534662
:108D500000F00CF800F006F8F5E7FFF73FFB05B070
:108D6000BDE8F08F15F80900A8557047A8F1020179
:108D7000204615E301A83818CDF800A05B4690F90D
:108D8000052070476F4890F87801000670472DE97C
:108D9000F84F1C46A2F130030A2B39D2303AC023D7
:108DA00003FB02F8C1F1D50101F1190300F113022F
:108DB00000F085F800F092F800F02CF8DFF888B1A8
:108DC0002C2100F084F800F085F80A9EDFF8449624
:108DD0001A2518F809008DF80300142700F063F82D
:108DE0000098000303D500F070F8E1B203E031040D
:108DF00000F06CF8F1B200F06AF8009840000090C2
:108E00007F1EEDD108F104086D1EE2D1FFF7E0BA34
:108E1000BDE8F18FDFF8F0A50121504601F0DFBB7E
:108E20002DE9F84F1C46A2F130030A2B39D2303A13
:108E3000C02303FB02F8C1F1BF0101F12F0300F1D0
:108E40001F0200F03CF800F049F8FFF7E3FFDFF8FD
:108E5000F8B02C2100F03BF800F03CF80A9EDFF857
:108E6000B895302518F809008DF80300202700F088
:108E70001AF80098002803D500F027F8E1B203E0C3
:108E8000310400F023F8F1B200F021F8009840001E
:108E900000907F1EEDD108F104086D1EE2D1FFF7AE
:108EA00097BABDE8F18F08EB090041788DF8021000
:108EB00081788DF80110C0788DF8000070479BB262
:108EC00092B289B280B2FFF7B6BA2104090E5846B1
:108ED00001F0BABB1021284601F07FBBDFF8245512
:108EE0001021284601F07BBB2DE9F04F9846A2F1F6
:108EF000300383B00A2B21D2124C0FF2500301F041
:108F0000D3FA05D004F03003202B02D10FF2342322
:108F10000093009B93F90030009E0193C1F1EF0193
:108F2000009B93F90140019B96F902606343921BF9
:108F30009E1003EB5673DB1001F0BDBABDE8F78F4E
:108F400078DC01206CC90120003001401019300A82
:108F500000000000FC3FFE7FFFFFFFFF3FFC1FF80B
:108F60001FF81FF81FF81FF81FF81FF81FF81FF849
:108F70001FF81FF83FFCFFFFFFFFFE7FFC3F0000D4
:108F8000000000000000003F803FC03FE03FF03F96
:108F9000F83FFC3E783E303E003E003E003E003E44
:108FA000003E003E003E003E003E003E003E003ED1
:108FB0000000000000000000FC3FFE7FFFFFFFFFFD
:108FC0003FFC1FF81FF800F800FC00FFC07FF03FD7
:108FD000F80FFC03FE007E003F00FFFFFFFFFFFFD6
:108FE000FFFF0000000000000000FC3FFE7FFFFFCD
:108FF000FFFFFFFF3FFC1FF800F800FCC07FC03FF1
:10900000C07F00FC00F81FF81FF83FFCFFFFFFFFC8
:10901000FE7FFC3F0000000000000000007C007E9E
:10902000007F807FC07FE07FF07FF87DFC7C7E7CCE
:109030003F7CFFFFFFFFFFFFFFFF007C007C007C09
:10904000007C007C007C0000000000000000FF7F2E
:10905000FF7FFF7FFF7F3F001F001F003F00FF3F9C
:10906000FF7FFFFFFFFF00FC00F81FF81FF83FFC29
:10907000FFFFFFFFFE7FFC3F00000000000000003C
:10908000FC3FFE7FFFFFFFFF3FFC1FF81F003F007C
:10909000FF3FFF7FFFFFFFFF3FFC1FF81FF81FF898
:1090A0003FFCFFFFFFFFFE7FFC3F000000000000D1
:1090B0000000FFFFFFFFFFFFFFFF00F800F800F8D0
:1090C00000F800F8007C007E003F801FC00FE00722
:1090D000F003F801FC00FC00FC00FC0000000000B4
:1090E00000000000FC3FFE7FFFFFFFFF3FFC1FF87A
:1090F0001FF81FF83FFCFE7FFC3FFE7F3FFC1FF880
:109100001FF81FF83FFCFFFFFFFFFE7FFC3F000042
:10911000000000000000FC3FFE7FFFFFFFFF3FFC60
:109120001FF81FF81FF83FFCFFFFFFFFFEFFFCFFCB
:1091300000FC00F81FF83FFCFFFFFFFFFE7FFC3F35
:109140000000000010192E0C0000000000000000BC
:10915000000000000000000000000000000000000F
:1091600000000000000000000000000000000000FF
:1091700000000000C001C001C001000000000000AC
:1091800000000000000000000000000000000000DF
:1091900000000000000000000000000000000000CF
:1091A00000000000000000000000000000000000BF
:1091B000E03FCC9F9CCF3CE73CE03CF03EF01E7093
:1091C0001E700E600640000006400E601E701E7885
:1091D0001F780F7C0F3CE73CF339F933FC27000084
:1091E00000000000008000C000E000E000F000F09F
:1091F00000700070006000400000004000600070DF
:1092000000780078007C003C003C003800300020F2
:1092100000000000E03FC09F80CF00E700E000F0CA
:1092200000F000700070C067E04FF01FE60FCE073F
:109230001E001E001F000F000F00E700F301F903DE
:10924000FC0700000000E03FC09F80CF00E700E087
:1092500000F000F000700070C067E04FF01FE04FBA
:10926000C067007000780078007C003CE03CF0397A
:10927000F833FC270000000000000C801CC03CE01C
:109280003CE03CF03EF01E701E70CE67E64FF01FD3
:10929000E04FC067007000780078007C003C003C24
:1092A00000380030002000000000E03FCC1F9C0F81
:1092B0003C073C003C003E001E001E00CE07E60FAF
:1092C000F01FE04FC067007000780078007C003C21
:1092D000E03CF039F833FC2700000000E03FCC1FF1
:1092E0009C0F3C073C003C003E001E001E00CE07C9
:1092F000E60FF01FE64FCE671E701E781F780F7CBA
:109300000F3CE73CF339F933FC2700000000E03F55
:10931000C09F80CF00E700E000F000F00070007018
:10932000006000400000004000600070007800789D
:10933000007C003C003C00380030002000000000B1
:10934000E03FCC9F9CCF3CE73CE03CF03EF01E7001
:109350001E70CE67E64FF01FE64FCE671E701E7878
:109360001F780F7C0F3CE73CF339F933FC270000F2
:109370000000E03FCC9F9CCF3CE73CE03CF03EF05F
:109380001E701E70CE67E64FF01FE04FC067007082
:1093900000780078007C003CE03CF039F833FC2792
:1093A0002DE9F04F9846A2F1300383B00A2B27D263
:1093B0001A4C0FF26C0301F077F805D004F030037B
:1093C000202B02D10FF2DC730093009B93F9003045
:1093D0000193202A009B93F9014093F9023008BFC2
:1093E0002F2202D03A2A08BF2E22019E6643D21AAB
:1093F000B31006EB5373DB10C1F1EF0101F05BB862
:10940000BDE8F78F000802400004024020DC012084
:109410007C15030884150308041D03086CC901208A
:109420002030300A000000000000000000000000B2
:10943000E0FFFF03F8FFFF0FFCFFFF1FFEFFFF3FF2
:10944000FEFFFF3FFFFFFF7FFFFFFF7FFF03E07F88
:10945000FF01C07FFF00807FFF00807FFF00807FD3
:10946000FF00807FFF00807FFF00807FFF00807F04
:10947000FF00807FFF00807FFF00807FFF00807FF4
:10948000FF00807FFF00807FFF00807FFF00807FE4
:10949000FF00807FFF00807FFF00807FFF00807FD4
:1094A000FF00807FFF00807FFF00807FFF00807FC4
:1094B000FF00807FFF00807FFF01C07FFF03E07F10
:1094C000FFFFFF7FFFFFFF7FFEFFFF3FFEFFFF3F2E
:1094D000FCFFFF1FF8FFFF0FE0FFFF03000000008D
:1094E000000000000000000000000000000000007C
:1094F0000000F80F0000FC0F0000FE0F0000FF0F3F
:109500000080FF0F00C0FF0F00E0FF0F00F0FF0F13
:1095100000F8FF0F00FCFF0F00FEFF0F00FFF70F2A
:1095200080FFF30FC0FFF10F80FFF00F007FF00FFF
:10953000003EF00F001CF00F0008F00F0000F00FCD
:109540000000F00F0000F00F0000F00F0000F00F1F
:109550000000F00F0000F00F0000F00F0000F00F0F
:109560000000F00F0000F00F0000F00F0000F00FFF
:109570000000F00F0000F00F0000F00F0000F00FEF
:109580000000F00F0000F00F0000F00F0000F00FDF
:109590000000F00F0000F00F0000F00F00000000CE
:1095A00000000000000000000000000000000000BB
:1095B000E0FFFF03F8FFFF0FFCFFFF1FFEFFFF3F71
:1095C000FEFFFF3FFFFFFF3FFFFFFF7FFF03E07F47
:1095D000FF01C07FFF00807FFF00807FFF00807F52
:1095E000FF00807FFF00807FFF00807F0000807F82
:1095F0000000807F0000807F0000C07F0000E07FCF
:109600000000F03F0000FC3F0000FF3F00C0FF1FD4
:1096100000F0FF0F00FCFF0700FFFF0180FF3F008D
:10962000C0FF0F00E0FF0300F0FF0000F83F000064
:10963000FC1F0000FC0F0000FE070000FE070000FA
:10964000FFFFFF7FFFFFFF7FFFFFFF7FFFFFFF7F2A
:10965000FFFFFF7FFFFFFF7FFFFFFF7F0000000096
:1096600000000000000000000000000000000000FA
:10967000E0FFFF07F8FFFF1FFCFFFF3FFEFFFF3F7C
:10968000FEFFFF7FFFFFFF7FFFFFFF7FFF03E07F06
:10969000FF01C07FFF00807FFF00807FFF00807F91
:1096A000FF00807FFF00807F0000807F0000807FC0
:1096B0000000C03F0000E03F00FCFF1F00FCFF0F68
:1096C00000FCFF0300FCFF0F00FCFF1F00FCFF3F3E
:1096D00000FCFF3F0000E07F0000C07F0000807FB3
:1096E0000000807F0000807FFF00807FFF00807F80
:1096F000FF00807FFF00807FFF01C07FFF03E07FCE
:10970000FFFFFF7FFFFFFF7FFEFFFF7FFEFFFF3FAB
:10971000FCFFFF3FF8FFFF1FE0FFFF070000000016
:109720000000000000000000000000000000000039
:109730000000F01F0000F81F0000FC1F0000FE1FCB
:109740000000FF1F0080FF1F00C0FF1F00E0FF1F81
:1097500000F0FF1F00F8FF1F00FCFF1F00FEEF1FBF
:1097600000FFE71F80FFE31FC0FFE11FE0FFE01FD6
:10977000F07FE01FF83FE01FFC1FE01FFE0FE01F1F
:10978000FF07E01FFF03E07FFFFFFF7FFFFFFF7F7B
:10979000FFFFFF7FFFFFFF7FFFFFFF7FFFFFFF7FD9
:1097A000FFFFFF7FFFFFFF7F0000E01F0000E01FC3
:1097B0000000E01F0000E01F0000E01F0000E01FAD
:1097C0000000E01F0000E01F0000E01F0000E01F9D
:1097D0000000E01F0000E01F0000E01F000000008C
:1097E0000000000000000000000000000000000079
:1097F000FFFFFF3FFFFFFF3FFFFFFF3FFFFFFF3F79
:10980000FFFFFF3FFFFFFF3FFFFFFF3FFF000000A5
:10981000FF000000FF000000FF000000FF0000004C
:10982000FF000000FF000000FF000000FF0000003C
:10983000FF000000FFFFFF07FFFFFF1FFFFFFF3FCD
:10984000FFFFFF3FFFFFFF7FFFFFFF7FFFFFFF7F68
:109850000000E07F0000C07F0000807F0000807F6C
:109860000000807FFF00807FFF00807FFF00807FFF
:10987000FF00807FFF00807FFF01C07FFF03E07F4C
:10988000FFFFFF7FFFFFFF7FFEFFFF7FFEFFFF3F2A
:10989000FCFFFF3FF8FFFF1FE0FFFF070000000095
:1098A00000000000000000000000000000000000B8
:1098B000E0FFFF03F8FFFF0FFCFFFF1FFEFFFF3F6E
:1098C000FEFFFF3FFFFFFF7FFFFFFF7FFF03E07F04
:1098D000FF01C07FFF00807FFF00807FFF00807F4F
:1098E000FF00807FFF000000FF000000FF0000007D
:1098F000FF010000FF030000FFFFFF07FFFFFF0F56
:10990000FFFFFF1FFFFFFF3FFFFFFF3FFFFFFF7F47
:10991000FFFFFF7FFF03E07FFF01C07FFF00807F2D
:10992000FF00807FFF00807FFF00807FFF00807F3F
:10993000FF00807FFF00807FFF01C07FFF03E07F8B
:10994000FFFFFF7FFFFFFF7FFEFFFF3FFEFFFF3FA9
:10995000FCFFFF1FF8FFFF0FE0FFFF070000000004
:1099600000000000000000000000000000000000F7
:10997000FEFFFF7FFEFFFF7FFEFFFF7FFEFFFF7FFB
:10998000FEFFFF7FFEFFFF7FFEFFFF7F0000807F67
:109990000000807F0000807F0000807F0000807FCB
:1099A0000000807F0000C07F0000E07F0000F07FAB
:1099B0000000F87F0000FC3F0000FE1F0000FF0FCA
:1099C0000080FF0700C0FF0300E0FF0100F0FF0080
:1099D00000F87F0000FC3F0000FC1F0000FE0F00AD
:1099E00000FF070000FF030080FF030080FF01006D
:1099F000C0FF0000C0FF0000E07F0000E07F00002B
:109A0000E07F0000E07F0000E07F0000E07F0000DA
:109A1000E07F0000E07F0000E07F00000000000029
:109A20000000000000000000000000000000000036
:109A3000E0FFFF01F8FFFF07FCFFFF1FFEFFFF3FF6
:109A4000FEFFFF3FFFFFFF7FFFFFFF7FFF03E07F82
:109A5000FF01C07FFF00807FFF00807FFF00807FCD
:109A6000FF00807FFF00807FFF00807FFF00807FFE
:109A7000FF01C07FFE03E03FFEFFFF3FFCFFFF1F33
:109A8000F8FFFF0FE0FFFF03F8FFFF0FFCFFFF1FD2
:109A9000FEFFFF3FFE03E03FFF01C07FFF00807F2E
:109AA000FF00807FFF00807FFF00807FFF00807FBE
:109AB000FF00807FFF00807FFF01C07FFF03E07F0A
:109AC000FFFFFF7FFFFFFF7FFEFFFF3FFEFFFF3F28
:109AD000FCFFFF1FF8FFFF0FE0FFFF030000000087
:109AE0000000000000000000000000000000000076
:109AF000E0FFFF03F8FFFF0FFCFFFF1FFEFFFF3F2C
:109B0000FEFFFF3FFFFFFF7FFFFFFF7FFF03E07FC1
:109B1000FF01C07FFF00807FFF00807FFF00807F0C
:109B2000FF00807FFF00807FFF00807FFF00807F3D
:109B3000FF01C07FFF03E07FFFFFFF7FFFFFFF7F8D
:109B4000FEFFFF7FFEFFFF7FFCFFFF7FF8FFFF7F31
:109B5000E0FFFF7F0000E07F0000C07F0000807F0B
:109B60000000807F0000807FFF00807FFF00807FFB
:109B7000FF00807FFF00807FFF01C07FFF03E07F49
:109B8000FFFFFF7FFFFFFF7FFEFFFF3FFEFFFF3F67
:109B9000FCFFFF1FF8FFFF0FE0FFFF0300000000C6
:109BA0000000000020302E0C00000000000000002B
:109BB00000000000000000000000000000000000A5
:109BC0000000000000000000000000000000000095
:109BD0000000000000000000000000000000000085
:109BE0000000000000000000000000000000000075
:109BF0000000000000000000000000000000000065
:109C00000000000000000000000000000000000054
:109C10000000000000000000000000000000000044
:109C20000000000000000000000000000000000034
:109C30000000000000000000000000000000000024
:109C40000000000000000000000000000000000014
:109C50000000000000E0030000E0030000E003005B
:109C600000E0030000E0030000000000000000002E
:109C700000000000000000000000000000000000E4
:109C800000000000000000000000000000000000D4
:109C900000000000000000000000000000000000C4
:109CA00000000000000000000000000000000000B4
:109CB00000000000000000000000000000000000A4
:109CC0000000000000000000000000000000000094
:109CD0000000000000000000000000000000000084
:109CE0000000000000000000000000000000000074
:109CF0000000000000000000000000000000000064
:109D00000000000000000000000000000000000053
:109D10000000000000000000000000000000000043
:109D20000000000000000000000000000000000033
:109D3000C0FFFF1F98FFFFCF38FFFFE778FEFFF35C
:109D4000F8FCFFF9F8F9FFFCF80300FEF80300FE49
:109D5000F80300FEF80300FEF80300FEFC0300FE1B
:109D6000FC01007FFC01007FFC01007FFC01007F03
:109D7000FC01007FFC00007F7C00007F3C00007E37
:109D80001C00007C0C000078000000700000000047
:109D9000060000300E0000381E00003C3E00003E71
:109DA0007E00003FFE00803FFE00803FFE00803FBF
:109DB000FE00803FFE00803F7F00803F7F00C01F8D
:109DC0007F00C01F7F00C01F7F00C01F3F00C01F5B
:109DD0009FFFCF1FCFFF9F1FE7FF3F1FF3FF7F1E98
:109DE000F9FFFF1CFCFFFF1900000000000000004D
:109DF00000000000000000C0000000E0000000F0D3
:109E0000000000F8000000FC000000FE000000FE62
:109E1000000000FE000000FE000000FE000000FE4A
:109E20000000007F0000007F0000007F0000007F36
:109E30000000007F0000007F0000007F0000007E27
:109E40000000007C000000780000007000000000AE
:109E500000000030000000380000003C0000003E20
:109E60000000003F0000803F0000803F0000803F76
:109E70000000803F0000803F0000803F0000C01FC6
:109E80000000C01F0000C01F0000C01F0000C01F56
:109E90000000C01F0000801F0000001F0000001E07
:109EA0000000001C0000001800000000000000007E
:109EB000C0FFFF1F80FFFFCF00FFFFE700FEFFF3A3
:109EC00000FCFFF900F8FFFC000000FE000000FEAF
:109ED000000000FE000000FE000000FE000000FE8A
:109EE0000000007F0000007F0000007F0000007F76
:109EF0000000007F0000007F0000007F0000007E67
:109F000080FFFF7CC0FFFF79E0FFFF73F0FFFF07DA
:109F1000E6FFFF03CEFFFF019EFFFF003E000000B3
:109F20007E000000FE000000FE000000FE000000B9
:109F3000FE000000FE0000007F0000007F00000027
:109F40007F0000007F0000007F0000003F00000055
:109F50009FFF0F00CFFF1F00E7FF3F00F3FF7F00D1
:109F6000F9FFFF00FCFFFF010000000000000000FF
:109F7000C0FFFF1F80FFFFCF00FFFFE700FEFFF3E2
:109F800000FCFFF900F8FFFC000000FE000000FEEE
:109F9000000000FE000000FE000000FE000000FEC9
:109FA0000000007F0000007F0000007F0000007FB5
:109FB0000000007F0000007F0000007F0000007EA6
:109FC00080FFFF7CC0FFFF79E0FFFF73F0FFFF071A
:109FD000E0FFFF33C0FFFF3980FFFF3C0000003E81
:109FE0000000003F0000803F0000803F0000803FF5
:109FF0000000803F0000803F0000803F0000C01F45
:10A000000000C01F0000C01F0000C01F0000C01FD4
:10A0100080FFCF1FC0FF9F1FE0FF3F1FF0FF7F1E8D
:10A02000F8FFFF1CFCFFFF1900000000000000000B
:10A0300000000000180000C0380000E0780000F0C8
:10A04000F80000F8F80100FCF80300FEF80300FE39
:10A05000F80300FEF80300FEF80300FEFC0300FE18
:10A06000FC01007FFC01007FFC01007FFC01007F00
:10A07000FC01007FFC00007F7C00007F3C00007E34
:10A080009CFFFF7CCCFFFF79E0FFFF73F0FFFF0731
:10A09000E0FFFF33C0FFFF3980FFFF3C0000003EC0
:10A0A0000000003F0000803F0000803F0000803F34
:10A0B0000000803F0000803F0000803F0000C01F84
:10A0C0000000C01F0000C01F0000C01F0000C01F14
:10A0D0000000C01F0000801F0000001F0000001EC5
:10A0E0000000001C0000001800000000000000003C
:10A0F000C0FFFF1F98FFFF0F38FFFF0778FEFF0329
:10A10000F8FCFF01F8F9FF00F8030000F803000075
:10A11000F8030000F8030000F8030000FC0300004F
:10A12000FC010000FC010000FC010000FC0100003B
:10A13000FC010000FC0000007C0000003C0000006E
:10A140009CFFFF00CCFFFF01E0FFFF03F0FFFF07D4
:10A15000E0FFFF33C0FFFF3980FFFF3C0000003EFF
:10A160000000003F0000803F0000803F0000803F73
:10A170000000803F0000803F0000803F0000C01FC3
:10A180000000C01F0000C01F0000C01F0000C01F53
:10A1900080FFCF1FC0FF9F1FE0FF3F1FF0FF7F1E0C
:10A1A000F8FFFF1CFCFFFF1900000000000000008A
:10A1B000C0FFFF1F98FFFF0F38FFFF0778FEFF0368
:10A1C000F8FCFF01F8F9FF00F8030000F8030000B5
:10A1D000F8030000F8030000F8030000FC0300008F
:10A1E000FC010000FC010000FC010000FC0100007B
:10A1F000FC010000FC0000007C0000003C000000AE
:10A200009CFFFF00CCFFFF01E0FFFF03F0FFFF0713
:10A21000E6FFFF33CEFFFF399EFFFF3C3E00003ECE
:10A220007E00003FFE00803FFE00803FFE00803F3A
:10A23000FE00803FFE00803F7F00803F7F00C01F08
:10A240007F00C01F7F00C01F7F00C01F3F00C01FD6
:10A250009FFFCF1FCFFF9F1FE7FF3F1FF3FF7F1E13
:10A26000F9FFFF1CFCFFFF190000000000000000C8
:10A27000C0FFFF1F80FFFFCF00FFFFE700FEFFF3DF
:10A2800000FCFFF900F8FFFC000000FE000000FEEB
:10A29000000000FE000000FE000000FE000000FEC6
:10A2A0000000007F0000007F0000007F0000007FB2
:10A2B0000000007F0000007F0000007F0000007EA3
:10A2C0000000007C0000007800000070000000002A
:10A2D00000000030000000380000003C0000003E9C
:10A2E0000000003F0000803F0000803F0000803FF2
:10A2F0000000803F0000803F0000803F0000C01F42
:10A300000000C01F0000C01F0000C01F0000C01FD1
:10A310000000C01F0000801F0000001F0000001E82
:10A320000000001C000000180000000000000000F9
:10A33000C0FFFF1F98FFFFCF38FFFFE778FEFFF356
:10A34000F8FCFFF9F8F9FFFCF80300FEF80300FE43
:10A35000F80300FEF80300FEF80300FEFC0300FE15
:10A36000FC01007FFC01007FFC01007FFC01007FFD
:10A37000FC01007FFC00007F7C00007F3C00007E31
:10A380009CFFFF7CCCFFFF79E0FFFF73F0FFFF072E
:10A39000E6FFFF33CEFFFF399EFFFF3C3E00003E4D
:10A3A0007E00003FFE00803FFE00803FFE00803FB9
:10A3B000FE00803FFE00803F7F00803F7F00C01F87
:10A3C0007F00C01F7F00C01F7F00C01F3F00C01F55
:10A3D0009FFFCF1FCFFF9F1FE7FF3F1FF3FF7F1E92
:10A3E000F9FFFF1CFCFFFF19000000000000000047
:10A3F000C0FFFF1F98FFFFCF38FFFFE778FEFFF396
:10A40000F8FCFFF9F8F9FFFCF80300FEF80300FE82
:10A41000F80300FEF80300FEF80300FEFC0300FE54
:10A42000FC01007FFC01007FFC01007FFC01007F3C
:10A43000FC01007FFC00007F7C00007F3C00007E70
:10A440009CFFFF7CCCFFFF79E0FFFF73F0FFFF076D
:10A45000E0FFFF33C0FFFF3980FFFF3C0000003EFC
:10A460000000003F0000803F0000803F0000803F70
:10A470000000803F0000803F0000803F0000C01FC0
:10A480000000C01F0000C01F0000C01F0000C01F50
:10A4900080FFCF1FC0FF9F1FE0FF3F1FF0FF7F1E09
:10A4A000F8FFFF1CFCFFFF1994F87841009304F0BB
:10A4B0003006102E70475A43091B161D491E62189C
:10A4C000531E019A1218521EFEF7F9FCFEF706FD04
:10A4D00001211E4800F083F8FEF7F8FAFEF7FAFCB7
:10A4E0000C9D00E0641E64B2012C28DB00270CE008
:10A4F0002904090EFEF7EDFAE9B2FEF7EAFA4FEA8F
:10A500006A0ABBF1010B0FD17F1C019801998010E1
:10A510007FB201EB5070B7EBE00FE3DA009816F969
:10A5200000A0761C4FF0080B5FEACA70E0D54FEA36
:10A530000841090EFEF7CDFA5FFA88F1DDE703B0B6
:10A54000BDE8F04F0121014800F047B80004024087
:10A55000F0B5002201230C6893401C409C4231D18D
:10A5600054000325A5400668ED432E4006600668AA
:10A5700091F90470A7403E43066091F90460012EF2
:10A5800018BF022E14D186682E408660866891F925
:10A590000570A7403E438660466826EA0303436091
:10A5A000436891F90660B6B29640B6B23343436051
:10A5B000C3682B40C360C36891F9075005FA04F4DF
:10A5C0002343C360521C102AC4D3F0BD006900228B
:10A5D000084218BF0122104670470183704741832B
:10A5E00070470AB1018370474183704710B5CB08AB
:10A5F00000EB830001F007018900036A0F248C40FF
:10A60000A343036202FA01F1036A1943016210BD18
:10A610001CB5DFF8E041A04203D1002001900023E7
:10A620000AE0DFF8D441A0421CBFDFF8D041A042CD
:10A6300009D10020019020234FF482700090002265
:10A64000204600F00EF813BD818101898907FCD5F1
:10A650000189C907FCD501890906FCD48089C0B2EB
:10A6600070472DE9F04385B006460C9C0D9D894648
:10A670001746984600A80DF0D5FE5E4960488E4208
:10A6800007D1416841F480514160484600F04DF8DF
:10A6900014E059498E4207D1016841F480410160BC
:10A6A000484600F05EF809E054498E4209D101683D
:10A6B00041F400410160484600F085F80020ADF803
:10A6C00004000020ADF80C80ADF80000ADF80E508D
:10A6D000ADF8024017B9ADF806000EE0012F09D021
:10A6E000022F04D10220ADF80600002005E0032F60
:10A6F00005D10220ADF806000120ADF808004FF4A6
:10A700000070ADF80A00002130460DF097FE30468B
:10A710000DF0DEFD00A930460DF006FE01213046A9
:10A720000DF08CFE05B0BDE8F08300B583B020B914
:10A7300000F010F8A021334805E0012804D10520DD
:10A7400000F068F830483BE0032804BF2948C046C1
:10A75000C04607BD05200190002303200090002281
:10A76000704700B5010083B027480ED100F021F8F2
:10A770004FF480610DF0EDFE0520019000230320D1
:10A7800000901A460C2121480CE0012904D100F068
:10A7900010F84FF4604105E0022904D1FFF7DAFF19
:10A7A0000D211B480CE0032904BF1348C046C046D6
:10A7B00007BD05210191002303210091002270476C
:10A7C0000DF0C7FE07BD00B583B020B9062000F02C
:10A7D00021F80F4807E0012806D10620FFF7BBFF4C
:10A7E0004FF4E0510948EBE7032804BF0348C04693
:10A7F000C04607BD0030014000380040003C00402A
:10A8000040380240000002400004024000080240BC
:10A8100000200240019000230320009000223821F4
:10A820007047704770477047704770477047704770
:10A830001748016841F080710160002115484160AE
:10A84000016841F0010101607047704712480068DB
:10A85000704711490968814200D20BE0081A70471D
:10A860000E48006870470D490968814200D201E036
:10A87000081A7047491E081A0DF0A4BE38B50446E0
:10A88000064805682846FFF7EEFF8442FAD231BD3C
:10A89000FCED00E0001000E0041000E0C0DC01204E
:10A8A0000CB41CB5044604A801900A46009401AB00
:10A8B00000A90748784418300DF088FE009900225E
:10A8C0000A7000285CBF0098001B16BC5DF80CFBEA
:10A8D0003703000006490860704706490860704762
:10A8E00005490860704702484AF6AA21016070478E
:10A8F0000030004004300040083000401849084350
:10A9000018490860704770B5037890F903401A46FB
:10A910000121ECB1134B1B68447803F4E063C3F5E9
:10A92000E0631B0AC3F10405AC4085780F2626FAC4
:10A9300003F32B4023430C4C1B01135500780B4BA6
:10A94000420900F01F0001FA00F043F8220070BD38
:10A950005009074A03F01F03994042F8201070BDC8
:10A960000000FA050CED00E000E400E000E100E08A
:10A9700080E100E07CB50024964E06EB84050121C1
:10A98000686A02F03DF800F03BF806EB440600A9C7
:10A99000B08A00F040F8686CFFF7DAFDB18A686CA5
:10A9A0000122FFF71EFE641C082CE5DB00F03AF8DC
:10A9B00000F026F84FF4006000F02DF800A9864C56
:10A9C0002046FFF7C5FD01224FF400612046FFF746
:10A9D00008FE00F027F8102000F018F801221021DE
:10A9E0002046FFF7FEFD00F01DF8202000F00EF8D5
:10A9F000012220212046FFF7F4FD00F017F873BD77
:10AA000000208DF804008DF806007047009000A922
:10AA10002046FFF79DBD009001208DF807008DF8BE
:10AA2000050070470121022001F0EABF00B585B0A2
:10AA30001C208DF8000001208DF8010002208DF807
:10AA4000020001208DF8030000A8FFF75CFF012140
:10AA5000012001F0E7FF40F2E730029001A96C20ED
:10AA6000ADF804000020ADF80C00ADF806004FF082
:10AA700080400EF00FFE01214FF080400EF08EFE60
:10AA8000012211464FF080400EF080FE01214FF070
:10AA900080400EF030FE05B000BD2DE9F8434D4E6C
:10AAA0004E4C7078DFF8389170B1206899F87B11BE
:10AAB000814207D24005000E00F0BCF92068401E1C
:10AAC000206001E000207070002501214FF08040DF
:10AAD0000EF065FE00287BD0DFF8FC804FF40061AB
:10AAE0004046FFF773FD00B9012599F800003D4F7E
:10AAF000484490F8A300022818BF03280AD1102167
:10AB00004046FFF763FD00B9012520214046FFF7CD
:10AB10005DFD00B16DB1FFF7A3FE00F069F8FFF72E
:10AB20009FFE7066307860BB387089F8F2050120AE
:10AB300024E099F8000031782B4D484490F8A300A8
:10AB4000022818BF032811D1012905D1FFF788FE7B
:10AB500070660220307001E0022912D1706EFFF79A
:10AB600082FEB9F8E21381420BD200E049B12878A5
:10AB700008B901203870002089F8F20589F8F1053C
:10AB80003070002706EB4700818A06EB8700406C97
:10AB9000FFF71CFD50B9B819007B18B9FFF760FE2C
:10ABA00000F026F8B8190121017303E0B81900215B
:10ABB000017301717F1C082FE4DB0C480168491CFC
:10ABC00001600121BDE8F4434FF080400EF0F1BD7B
:10ABD000BDE8F183003A002000040240D831002093
:10ABE0006CC90120CB310020CA310020C0DC01201B
:10ABF000206099F8790100F0BF0089F8790199F88F
:10AC00007A0100F017B90268531C03601170704795
:10AC10007CB50121042001F0F3FE00F071F84FF43F
:10AC2000007000F07CF8324D00F071F80121042032
:10AC300001F0E6FE01208DF804004FF4807400203E
:10AC40008DF80600009400F06BF800F060F8002228
:10AC50004FF4007100F060F800F05CF80121102062
:10AC600001F0CEFE01208DF804008DF806000220D0
:10AC700000F055F81F4D00F04AF81F4E96F8670196
:10AC800080064CBF00220122022100F045F896F810
:10AC9000670180064CBF01220022022100F03CF82F
:10ACA0000121082001F0ACFE00F02AF84FF480608A
:10ACB000009000A9114D00F02AF800224FF48061A5
:10ACC00000F02AF80121082001F09AFE01208DF8F9
:10ACD0000400009400208DF8060000A901208DF8E2
:10ACE00007008DF8050000F012F800F013F873BDAE
:10ACF00000080240001002406CC90120000C024014
:10AD000001208DF8040000208DF8060070472846C9
:10AD1000FFF71EBC012221462846FFF762BC0090C7
:10AD200001208DF807008DF8050000A9704700008C
:10AD300030B58BB0FDF7D6F90220FDF7BDFB012140
:10AD4000082001F05DFE01208DF810004FF4007422
:10AD500000208DF81200039401208DF813008DF867
:10AD6000110003A9DFF808552846FFF7F1FB21463B
:10AD70002846FFF734FC0121042001F053FEFE2099
:10AD800008904FF45860ADF81C000020ADF8240086
:10AD9000ADF81E0007A9DFF8DC5428460EF07AFC57
:10ADA000012128460EF0FAFC012128460EF0A3FCF2
:10ADB0000121022001F024FEDFF8BC540222092107
:10ADC0002846FFF713FC0020ADF80A00019402208A
:10ADD0008DF8080001A903208DF809002846FFF727
:10ADE000B7FBFF2000F026F801214FF4804001F06E
:10ADF00022FE092101200EF0E1FC01208DF81A004D
:10AE0000059400208DF8180010208DF8190005A871
:10AE10000EF0E8FC17208DF8000000208DF80100EE
:10AE20008DF8020001208DF8030000A8FFF76BFDEC
:10AE30000BB030BD30B50446DFF84004007885B073
:10AE400003280CBF01200020DFF8341409780D29F5
:10AE50000CBF01210021DFF82C24527902B101221C
:10AE6000084010421CBFDFF8200490F87B4170209E
:10AE7000ADF800000120ADF802000220ADF80C0092
:10AE8000029400A9DFF8EC5328460EF03EFC08219E
:10AE900028460EF073FCDFF8D80324B94FF4007194
:10AEA000FFF79BFB05E0FF2C04BF4FF40071FFF799
:10AEB00096FB05B030BD10B54FF400700EF0CBFC22
:10AEC000A8B1EB4CEC484FF40071FFF77FFB012871
:10AED0004FF40071204602D1FFF781FB01E0FFF73C
:10AEE0007CFBBDE810404FF400700EF0BFBC10BDFD
:10AEF00070B50546DFF83C4D2DED028B4FF61F0275
:10AF00004FF4007120460EF0BBFC002D00F0858050
:10AF1000002500EE105AF1EE000AB8EEC00AB0EEBD
:10AF2000608A00F023FFDFF8802DDFF8803D0DF010
:10AF3000F3F80EF0C3FC00EE100AF0EE480A0EF033
:10AF400086FEBDEEC00A10EE100AC01000F01F0011
:10AF500024F815006D1C2A2DDBDB0020062505FBDF
:10AF600000F18910490101F4FC6104EB400241F059
:10AF70001F01401CA2F854102A28F0DB0026C6F15D
:10AF8000290000EE100AB8EEC00A00F0EFFEDFF86C
:10AF9000942DDFF8B03D0DF0BFF841EC100B53ECF1
:10AFA000102B0DF0B9F80DF08BF8C01000F01F0059
:10AFB00004EB460140F4FC60761CA1F8A8002A2EA0
:10AFC000DDDB002010FB05F1090204EB400241F437
:10AFD000FC61401CA2F8FC102A28F3DB0020C0F121
:10AFE000290169438910490104EB400241F4784189
:10AFF000401CA2F850112A28F1DB002005FB00F1CB
:10B00000C91001F01F0104EB400241F47841401CDB
:10B01000A2F8A4112A28F1DB56E000EE105AF1EE56
:10B02000000ABAEECE0A0EF012FEBDEEC00A10EE15
:10B03000100AC01000F01F0024F815006D1C402DF0
:10B04000EBDB0020820104EB400102F4FC6242F0E1
:10B050001F02401CA1F880202028F3DB0020C10043
:10B06000C1F1FF01C91001F01F0104EB400241F4DE
:10B07000FC61401CA2F8C0102028F0DB002004EB8B
:10B080004001C20242F4FC62401CA1F800212028C9
:10B09000F5DB00208100C1F1FF018910490104EBBB
:10B0A000400241F47841401CA2F840114028F1DBF5
:10B0B000002004EB400100F01F0242F47842401CE3
:10B0C000A1F8C0212028F4DBBDEC028B70BD70B567
:10B0D000DFF8545C0446287A82B001F01EFB0021A0
:10B0E000DFF8486C56F83120944222BF06EBC102CB
:10B0F0005268A24203D3687901F00FFB02E0491CB9
:10B100000A29EFDB0A2156F83120944222BF06EBD0
:10B11000C1025268A24203D3A87901F0FEFA02E00C
:10B12000491C1A29EFDB584909781A2904BFE87924
:10B1300001F0F3FA0021009103462246AA211920CA
:10B14000FDF764FD73BD2DE9F0410746DFF8E04BE4
:10B1500094B000F082F820460DF0BAF80020ADF867
:10B16000000001904FF4007500F071F84FF4827602
:10B170000720ADF81000ADF8026000A920460DF0E0
:10B18000D3F8012100F06AF801214FF4800001F0AA
:10B1900037FCDFF8688D40460EF05CFD0997002013
:10B1A0001090119012900D9005A94FF480600B90B3
:10B1B00000200E90DFF8480D0690002013900C90B0
:10B1C0000A904FF400300F904FF0C060059040207F
:10B1D0000890DFF8280E079040460EF09BFD0121F5
:10B1E00040460EF0BFFD0122022120460DF056F927
:10B1F0004FF0C05140460EF0C2FD0028F8D04FF08D
:10B20000C05140460EF0CCFD002140460EF0AAFD94
:10B210000022022120460DF041F900F01EF82046E0
:10B220000DF056F80020ADF80000019000F00FF886
:10B23000ADF802600720ADF8100000A920460DF01F
:10B2400073F8012100F00AF814B0BDE8F081ADF800
:10B250000800ADF80A5003907047002120460DF019
:10B26000EDB84FF0C051DFF8940C0EF088BD00002F
:10B27000000C0240000800400004024045DC0120B0
:10B2800044DC012034DC01206CC901202DE9F74F9A
:10B290002DED0C8B99468EB04FEA0920DFF860AD9A
:10B2A000269D1FFA80FBDAF873010CF0FBFEDFF835
:10B2B000543D00220CF030FF06469AF868010F4614
:10B2C0000CF0F0FE02460B46304639460CF0BCFD51
:10B2D00041EC1A0B0020DFF8301D00F00AFD41ECB4
:10B2E000180B9AF80000DFF8244D0AEB8000FF26C7
:10B2F000D0F80100C4F81C01002000EB0A0191F80D
:10B30000F0148E42A8BF0E46401CFF28F5DD94EDD8
:10B310004B0ADFEDA70A20EE200A00EE906AF8EE55
:10B32000E00A9FEDA41A00EE810A84ED4B0A00F0BA
:10B330001DFD00F0F1FC0EF089FD00F0EDFC0CF0BD
:10B3400083FD0EF0BBFA00EE100A1B984844ADF8DE
:10B35000080000F00BFD41EC190B002D00F00381FB
:10B360001A981B99BDF8083000F1FF0292B289B219
:10B3700080B2FDF760F8DFF8545D10212846FFF732
:10B380002EF9DFF8546D01213046FFF728F92C2102
:10B39000DFF89C09FFF758F910212846FFF71DF93F
:10B3A0004FEA492080B2FFF7CEFE01213046FFF779
:10B3B00014F9D4F83001FFF756FA9AF88A11D4F844
:10B3C000185181420CD24FF4807007E005EB400128
:10B3D000A1F5007135F810200A80401C5845F5DBB6
:10B3E000D4F82071D4F81C01C01B0CF051FE00F001
:10B3F00080FC0CF065FE06000AD00CF049FE53EC10
:10B400001A2B0CF089FE0CF05BFEC019C4F8200169
:10B4100006F1FF00B0F5FF7F88BF00263046C4F874
:10B420002461012815DB002105E025F812607F1C4E
:10B43000FF2F03DD491C494521DA0027C61907EB18
:10B440000122FF2ECEBF002606EB012635F816603E
:10B45000EBE7002813D5002104E025F81760521E01
:10B4600003D5491C49450ADAFF22861802EB012759
:10B470004EBF002606EB012635F81660EDE7D4F83E
:10B480003001FFF7F0F90546BAF888010CF00AFE22
:10B4900000F0AFFD0022DFF81C3D0EF097FD0EF02E
:10B4A0000DFA0BEE100A9AF88A01A84224D2002560
:10B4B00000F060FC00F052FC00F04AFC00F044FC9C
:10B4C0000CF0FEFD80F30806DFF8680730F8160080
:10B4D000D4F81811ADF8000005EB0B0001EB4001AA
:10B4E00000F0F4FB6D1C00F0E3FBFF2DE0DDFFF747
:10B4F000B7F9C4F8300136E0002500F03BFC00F05D
:10B500002DFC00F025FC00F01FFC0CF0D9FD80F3B1
:10B510000806D4F8181105EB0B0001EB4001A1F56A
:10B52000007212788DF80520A1F2FF1212788DF8C2
:10B5300004200022DFF8FC76019B37F81270BB4232
:10B5400002D0521CFF2AF5DDB24209DADFF8E42608
:10B5500032F81620ADF8002000F0B8FB00F0A8FB90
:10B560006D1CFF2DC9DD1C980CF092FD02460B46A8
:10B570000020DFF8441C0CF067FC41EC1B0B0020A2
:10B58000DFF8341C00F0C0FB0CF09AFDC6B2304668
:10B590000CF07EFD0022DFF8183D0CF0BDFD41EC03
:10B5A0001C0B9AF8860138B942F2041B27E000BF51
:10B5B0003333333F9A99993E012808BF44F2082B50
:10B5C0001DD0022808BF46F20C3B18D0032808BF44
:10B5D00048F2104B13D0042808BF4AF2145B0ED077
:10B5E000052808BF4CF2186B09D006280FBF4EF291
:10B5F0001C7BDFF8401601EB4000B0F842B0D4F8F5
:10B600001C0141F28831B0FBF1F141F2883202FBBA
:10B6100011000CF047FD00F06CFB0CF051FD0CF03C
:10B6200037FD41EC1A0B201D2CC80AA92CC100F0D3
:10B6300018FB27DBD4E9442351EC1A0B0EF03AFD3A
:10B6400020D06FF0050500F03EFB53EC182B0CF0FA
:10B6500063FD53EC1A2B0EF0B9FC0CF031FDC0F178
:10B660007F080AA82818B8F1FF0F92BF80F806805B
:10B670000021817181797F2904BF002181716D1CB6
:10B68000062DE0DB0AF2F040C4F8280100251B98E3
:10B6900048440190401C069001983018059051ECE8
:10B6A0001C0B0CF00DFD099051EC1A0B0CF008FD71
:10B6B0000790D4F828019AF88411285CB1B994ED68
:10B6C0004B0A00F05DFB06460F4653EC192B4FF07A
:10B6D0003330DFF8CC1C0CF01FFD00F035FB0CF014
:10B6E000EFFC80F308000CF0D3FC01E00CF0DAFC76
:10B6F00000F00AFB0CF0E4FC064601989AF885710C
:10B700003018401C04901A9828180390022FC0F299
:10B710000A81681005EB90708010A5EB80080398F3
:10B7200094ED448BC01C089053EC182B51EC1A0B71
:10B730000EF0C0FC4FF0010900F0A880032F08BFF5
:10B74000B8F1000F4BD151EC180B0CF0B9FC089973
:10B75000091A421000EB9270801001EB80000090FB
:10B76000002738460CF094FC00F0FCFA0CF0A8FC22
:10B77000BDF8081000EB0108009904F11002895C83
:10B78000814200DB0FB900220DE00CF081FC53EC8C
:10B790001B2B0CF0C1FC0CF093FCDFF8981401EBB0
:10B7A0004000B0F8642000981FFA88F180B2FCF7DE
:10B7B00031FE7F1C052FD4DB00F057FABDF80800DE
:10B7C000009038460CF064FC00F0CCFA0CF078FCE9
:10B7D0000099411800F080FA7F1C052FEEDB00274E
:10B7E00038190079854211D1012D0FDB00F029FABB
:10B7F0002846FDF700F900F04BFA04F11000285C30
:10B80000864201DA00F03CFA4FF0000900F029FA14
:10B8100002BF0AA8385C854205D1012D03DB00F088
:10B8200014FA4FF000099AF88501032802BF0AA80C
:10B83000385C85421AD1012D18DB00F029FA04F199
:10B840001000285C864201DA00F01AFA4FF0000876
:10B8500007E0BDF8080000EB880000F0FCF908F1F3
:10B86000010809988045F4DB4FF000097F1C0C2F7C
:10B87000B6DBB9F1000F56D02819007CB04202DACD
:10B8800000F006FA4FE000F0FBF94CE0022F10D177
:10B8900000270AA8385C854205D1012D03DB00F0A2
:10B8A000D4F94FF000097F1C0C2FF2DBB9F1000F27
:10B8B00008D02819007CB04202DA00F0E9F901E072
:10B8C00000F0DEF99AF8850103282CD100270AA898
:10B8D000385C85420FD1012D0DDB4FF0000907E0E8
:10B8E000BDF8080000EB890000F0B5F909F1010985
:10B8F00009988145F4DB7F1C0C2FE8DBB8F1000FC1
:10B9000011D100F0B2F9BDF8089038460CF0C0FB38
:10B9100000F028FA0CF0D4FB00EB090100F0DCF990
:10B920007F1C052FEFDB00F09CF908DA2819007C5A
:10B93000B04202DA00F0ACF901E000F0A1F92819F8
:10B940006D1C0674FF2D7FF7B4AE00F08AF91BDB87
:10B950000DD1002500F0B6F900F004FA0CF0B0FBB0
:10B96000C2195B4600F068F96D1C052DF2DBD4E9C5
:10B97000442351EC1A0B0EF09DFB03D00AA82CC8EF
:10B98000211D2CC184ED44AB9AF8850101281BD1FF
:10B9900000252819007918B100F053F9FDF72BF8AC
:10B9A0006D1C0C2DF5DB002500F08CF900F0DAF9A8
:10B9B0000CF086FBC219002300F03EF96D1C052D2A
:10B9C000F2DB00208AF885019FEDDA9BBAF871510D
:10B9D000B0EE498AF0EE698AB0EE49AAF0EE69AAA3
:10B9E000B5F5006F08BF08260DD0B5F5806F08BF0C
:10B9F000042608D0B5F5007F08BF022603D0B5F5B0
:10BA0000807F08BF0126DAF873010CF04BFB074674
:10BA1000894628460CF046FB02460B463846494606
:10BA20000CF012FA41EC1B0B9AF8000000EB0A052F
:10BA3000B0EE4BCA95F8A300F0EE6BCA042846DAC4
:10BA4000022818BF03282AD1BAF8DE030CF02AFB1B
:10BA500041EC1A0B95F8D9000AEB40009FEDB7DBDB
:10BA600000F036FB53EC1D2B0CF056FB02460B4648
:10BA700051EC1A0B0EF0EAF900F04AF941EC180B00
:10BA800095F8D9000AEB400000F022FB53EC1D2B87
:10BA90000CF042FB53EC1A2B0EF098FA13E005F26F
:10BAA000A307F87E0AEB8000B0F8AE010CF0FAFABA
:10BAB00000F02EF941EC180BF87E0AEB8000B0F88C
:10BAC000B0010CF0EFFA00F023F941EC1A0B95F8F5
:10BAD000A30005F2D907042805D100F00EF900F003
:10BAE00017F900F0FFF895F8A300052818BF0628FD
:10BAF00005D100F002F900F00BF900F0F3F895F829
:10BB0000A350082D18BF072D13D10020DFF88C1B80
:10BB100000F0FEF841EC180B9AF8F70500281ABF60
:10BB20000020DFF87C1BDFF85C1C00F0EDF841EC36
:10BB30001A0B9AF868010CF0B5FA41EC190B304673
:10BB40000CF0A6FA41EC1B0B51EC180B00F0DCF8E2
:10BB500000F004F90CF0B4FA064651EC1A0B00F0B0
:10BB6000D3F800F0FBF80CF0ABFA8046802E28BF2B
:10BB70007F26B8F1800F28BF4FF07F08002D1CBF33
:10BB8000022D072D03D1C6F17F06C8F17F08012DD4
:10BB90001CBF032D082D04D1B0B208F17F0600F1BF
:10BBA0007F08042D18BF052D04D1B0B2C0F17F0667
:10BBB00000F17F08062D04BFC6F17F064FF07F0815
:10BBC0002078B04204BF6178414510D01A9D00F042
:10BBD00038F855FA80F0FCF70EFF1A98657800F0F7
:10BBE00030F84019FCF707FF267084F801804FF603
:10BBF000FF747F2E06D01A98059A019923463018B3
:10BC0000FCF7F9FEB8F17F0F06D01A98059A019952
:10BC100023464044FCF7EFFE1A98059A01994FF429
:10BC200078437F30FCF7E7FE0EB0BDEC0C8BBDE82F
:10BC3000F78F000074CF01204FF480710020FCF7D3
:10BC4000A7BE059A019900237047059A01995B46A2
:10BC50002846FCF7D0BE411C5A4689B2A8B2FCF770
:10BC6000D9BB9AF885010228704707980899091AE4
:10BC7000421000EB9270801001EB800800277047A3
:10BC800001994018421C049903980023FCF7E5BE73
:10BC9000049A06990398DFF8FC3AB0EE4B0AF0EEEE
:10BCA0006B0AFCF733BF000052B81E85EB51B83F5A
:10BCB000D4F8181101EB4000A0F2FF109DF800101D
:10BCC00001707047019F28460CF0E2B9A1F50071A0
:10BCD0009DF801200A7070475A4689B21FFA88F011
:10BCE000FCF798BB41EC180BB0EE49AAF0EE69AA3C
:10BCF000704753EC1A2B0CF0A7B8F87E0AEB400003
:10BD0000B0F8CE010CF0CEB953EC1B2B0CF09CB864
:10BD100053EC1C2B0CF098B802460B460020DFF8C1
:10BD2000781A7047F6285C8FA4310020845A0308E3
:10BD30000030014000000000000000000000000092
:10BD40000000E03FC2F5D83F32463B460CF0E4B974
:10BD500006460F461BEE100A0CF04EB853EC192B9A
:10BD60000CF0DAB953EC1C2B0CF0D6B910EE100A1B
:10BD70000CF042B805EB0A0094ED4B0A90F8F00382
:10BD8000BDEEC00A10EE101A401A0CF081B92DE970
:10BD9000FC419B4EDFF8044A96F87001DFF8005A28
:10BDA000012802D10FF6242103E002280BD10FF65F
:10BDB000282100F0CDF800200190234600F07AFA07
:10BDC0002A46002196E03078DFF8D879801990F87B
:10BDD000A30028B90FF60C2100F0BAF800F0A5F87E
:10BDE00000F0ACF8012805D10FF6002100F0B0F802
:10BDF00000F09BF800F0A2F8022805D10FF6F4112C
:10BE000000F0A6F800F07EF800F098F8032805D1BD
:10BE10000FF6E81100F09CF800F074F800F08EF8CE
:10BE2000042807D10FF6DC1100F092F896F9A6016C
:10BE300000F06AF800F082F8052807D10FF6CC115F
:10BE400000F086F896F9A70100F05EF800F076F8A9
:10BE5000062807D10FF6BC1100F07AF896F9A70171
:10BE600000F052F800200EF0DCF900F067F8082826
:10BE700005D10FF6A81100F06BF800F04AF800F0B9
:10BE80005DF8072805D10FF6A01100F061F800F069
:10BE900040F8DFF8140902F0A9FE96F88B01032898
:10BEA0001CD13078DFF80479DFF8041906EB800044
:10BEB000D0F80100884203D2384602F097FE0DE028
:10BEC000DFF80882012200F03EF8384602F08EFECC
:10BED0000520FEF7D3FC002200F035F8012086F89B
:10BEE000F805DFF8D008007800F017FC00F02BF917
:10BEF00023462A4600F0F2F8BDE8F3815864024078
:10BF00000C30014096F9A50137F81000A6F8FE059F
:10BF1000704796F9A50137F81000A6F8FE0596F8C7
:10BF2000F705401CC0B20EF07CB996F8A40100F0F1
:10BF30000F0037F81000A6F8FE057047307880191A
:10BF400090F8A30070474FF400714046FEF749BBDC
:10BF50002846FEF7A5BC7CB5294D95F87001002850
:10BF600046D12878401990F8A310072940DADFF865
:10BF700030680FF6C00404291ADA022918BF032911
:10BF800006D190F8D90005EB4000B0F8DE0115E0CD
:10BF900000F2A300C17EC07E05EB810105EB8000AD
:10BFA000B1F8B011B0F8AE01081A0CF071F807E062
:10BFB00090F8F40005EB4000B0F8CE010CF072F8F8
:10BFC00000F017F802460B4621463046FEF768FCA3
:10BFD000012085F8F805DFF8DC07407800F09DFBCC
:10BFE000DFF8B83700F0AFF83246282100F076F8D5
:10BFF00073BDDFF8C43700220BF026BF70CC0020E1
:10C000006CC901200000703F0088B340D037002089
:10C01000F0B5DFF8A867DFF8885730780FF63004FE
:10C02000801983B090F8A310042931DA022918BFCF
:10C03000032914D190F8D90006EB400000F048F82D
:10C04000FFF7D7FFCDE90001B6F8DE030CF02AF8C0
:10C05000FFF7CFFF0B4602460FF2E47125E000F236
:10C06000A307F87E06EB8000B0F8B0010CF01AF8D8
:10C07000FFF7BFFFCDE90001F87E06EB8000B0F8C6
:10C08000AE010CF00FF8FFF7B4FF02460B460BE0D1
:10C0900090F8F40006EB4000FFF732FEFFF7A9FF2F
:10C0A000CDE900010022002321462846FEF7F8FBD7
:10C0B000002001904FF6F07000902A46DFF8DC3641
:10C0C000B0210020FCF71FFAF7BD00000008024075
:10C0D000B0F8DE010BF0E6BF00040240DC20FCF704
:10C0E00012BA2DE9F04383B091461E460A9CDFF850
:10C0F000B0560B4602460FF268712846FEF7D0FB99
:10C10000DFF8B076B87800F008FBDFF8908600F032
:10C110001AF843462A468421FFF7E0FF009623469B
:10C120004A460FF248712846FEF7BAFBF87800F04D
:10C13000F4FA00210191009043462A46C621FFF7F8
:10C14000CDFFBDE8F7830090002101917047F0B565
:10C15000DFF8684694F8000683B018B900F0AEF82E
:10C1600000F0C1F894F800060FF20C75DFF82C66A9
:10C17000012807D100F037F800F020F80FF2007224
:10C1800000F0E9F894F800060FF20477022808D1CD
:10C1900000F014F80FF2F062C820FCF7B4F900F0D8
:10C1A00016F894F80006032803D100F01CF800F0FC
:10C1B0000EF8F7BD0000F03F000070400020019035
:10C1C00033464FF4784000904FF48371704700205D
:10C1D000019033464FF4784000903A464FF4837113
:10C1E000B420FCF790B90020019033464FF478401A
:10C1F00000902A464FF48371C820FCF784B97CB5BF
:10C20000DFF8BC452068FEF72EFBB0F57A7F4ED9EB
:10C21000DFF8B005DFF8885590ED000ADFF8A805D3
:10C22000D0ED000AB8EE400A20EE200AFFF79EFD8E
:10C2300002460B460FF260612846FEF731FBDFF83D
:10C240007405007900F069FADFF85065FFF77BFFAD
:10C2500033462A464FF48271FFF740FFDFF85C0552
:10C2600090F86711490622D52178C90706D500F054
:10C2700019FAFEF7F5FA4008400017E090F8F105CA
:10C2800030B9019033464FF6F070009091A205E06E
:10C2900000200190334600F00DF8BAA20021BE2024
:10C2A000FCF731F9FEF7DCFA40F00100206073BDC5
:10C2B0000000D03F4FF478400090704700B5DFF8A1
:10C2C000FC140A78511883B091F82D1100F004F98C
:10C2D00000F0EBF80FF2C852C820FCF714F9BDE8E3
:10C2E000074002F0E5BB30B5DFF8D054DFF8AC44CE
:10C2F0002878401983B090F8120128B90FF2A8529B
:10C3000000F08AF800F027F800F020F8012805D1A5
:10C3100000F08AF80FF2985200F01DF800F016F8BD
:10C32000022805D100F080F80FF28C5200F013F8CB
:10C3300000F00CF8032805D100F076F80FF28052D7
:10C3400000F009F8BDE8374002F0CBBB287840196F
:10C3500090F812017047B420FCF7D5B800B5DFF8AB
:10C360005C1491F80F1183B000F01CF8C1A200F02A
:10C3700011F8A0200BE000B5DFF8401491F810117F
:10C3800083B000F00FF880A200F004F88C20FCF7D6
:10C39000BAF807BDDFF804344FF48371704700002A
:10C3A0003333FB3F46F20C3009B14FF4FC600021FF
:10C3B00001910090704730B5DFF80054DFF8DC439E
:10C3C00095F8110183B028B900F026F80FF2F84271
:10C3D00000F01FF895F81101012805D100F024F8AC
:10C3E0000FF2EC4200F015F895F81101022805D182
:10C3F00000F01AF80FF2E04200F00BF895F8110186
:10C40000032805D100F010F80FF2D44200F001F833
:10C4100037BD7820FCF777B80190234646F20C3000
:10C4200000904FF4837170470020019023464FF431
:10C43000FC6000904FF48371704730B5DFF87C03E7
:10C44000D64C90F8F125D64D0FF29C4183B04AB1FD
:10C4500090F863212846FEF723FA002001904FF45C
:10C4600078400AE00278101890F848212846FEF734
:10C4700017FA002001904FF4FC60009023462A46F2
:10C480004FF483716420CFE000B5CC4991F8671177
:10C4900083B046F20C30C90748BF4FF4FC6000F08F
:10C4A00004F80FF24C42502071E7002101910090F6
:10C4B0004FF48371B94B704700B5C04991F86A11C8
:10C4C00083B000F009F8FFF7F0FF0FF22C423C2098
:10C4D0005DE700005258000046F20C3009B14FF4FD
:10C4E000FC6070472DE9FC47B44CDFF8B09294F83B
:10C4F0006B0104F26B1540F227189EA746F20C362A
:10C50000002804BF6978012909D100F044F89AA2F3
:10C5100000F03CF80020019000964B4615E00FF229
:10C52000E03A012814D16878D8B900F034F893A221
:10C5300000F02CF80020019000964B4690A24FF49A
:10C540008E7100F025F800F02CF83A46414614E0D0
:10C5500038B9687898B9019000964B46524600F079
:10C5600015F894F86B01012804BF6878012806D1FA
:10C5700000F017F852464FF4837100F009F8BDE857
:10C58000F387000054580000444E52004FF483716A
:10C590002820FBF7B8BF01904B464FF4FC60009099
:10C5A0007047002001904B464FF4FC6000907047AC
:10C5B00030B5824D7A4C95F8690183B018B90FF205
:10C5C000483100F034F895F86901012803D10FF2E1
:10C5D000403100F02CF895F86901022803D10FF2E0
:10C5E000383100F024F895F86901032803D10FF2DF
:10C5F000303100F01CF895F86901042803D10FF2DE
:10C60000283100F014F895F86901052803D10FF2DC
:10C61000203100F00CF8002001904FF4FC600090F5
:10C620002246FFF7B7FE1420FBF76DFF37BD20460B
:10C63000FEF736B930B504464FF6FF7583B02B468A
:10C64000BB22AB210020FCF7D6F92B46BB22AB2145
:10C650000C20FCF7D0F9514B0195002C03D00020A1
:10C66000009049A202E00020009048A20121AA20E7
:10C67000DAE70000414E460000B5504991F86D11CF
:10C68000002083B0890748BF4FF478400190002014
:10C6900000903FA2414B0D21AA2078E600988C40E3
:10C6A0000054954080B500200090D0231622BE2172
:10C6B000FCF79EF84FF478430422C8210F20FCF7C2
:10C6C000E4F84FF478430522C8210F20FCF7DDF889
:10C6D000FFF7F0FDC8230C22C8210020FCF718F852
:10C6E000FFF7E8FDC9230C2219460020FCF710F8DB
:10C6F000FFF7E0FDC72300F00BF8FFF7DBFDC623D3
:10C7000000F006F8FFF7D6FDC52300F001F801BDE3
:10C71000042219460220FBF7FBBF4FF6FF7110B948
:10C7200042F2041123E0012808BF44F208211ED080
:10C73000022808BF46F20C3119D0032808BF48F27E
:10C74000104114D0042808BF4AF214510FD0052814
:10C7500008BF4CF218610AD006280CBF4EF21C71BB
:10C76000072804D00B4901EB4000B0F84010084600
:10C770007047000054000000455152004551000030
:10C780005200000000F49040420000004100000010
:10C790005300000074CF012000E06F40343C0020C3
:10C7A0002CC90120E05D0308BFEB000809AC0108BB
:10C7B000007E5603A431002000408F406CC9012048
:10C7C000CCDC012064DB012098DC012049512034BD
:10C7D000386B2F323462200049512039366B2F31AB
:10C7E000366220004C534220000000005553422086
:10C7F0000000000043574C20000000004357522027
:10C8000000000000414D202000000000464D202087
:10C8100000000000464D32200000000052545459E0
:10C820002020202020200000525454592D4C20203C
:10C830002020000025312E31666B487A2000000050
:10C840004325352E3266205725352E3266000000EE
:10C850004C25352E3266204825352E3266000000E4
:10C86000253032642F2530326420000025303264B8
:10C8700025632530326400005246204F46000000F8
:10C880004453204F4E0000005246204F4E000000FF
:10C890004453204F4600000025342E3166560000D8
:10C8A0005052452020000000415454202000000038
:10C8B00041545420380000004154543136000000E7
:10C8C00041545432340000004E4230300000000029
:10C8D0004E423031000000004E4230320000000075
:10C8E0004E423132000000004147432531640000D0
:10C8F0004D4F4E49000000004543484F00000000E6
:10C9000045515254000000005020303025250000D1
:10C9100050203130252500005020323525250000DB
:10C9200050203530252500005020383025250000C6
:10C930005031303025250000564900220A700A7017
:10C94000012802D0042801D105200870704710B5D5
:10C9500051494A6802F00C02042A02D0082A02D087
:10C9600019E04F4A18E00A680B68C2F3805203F0DE
:10C970003F03002A14BF4A4A4A4AB2FBF3F20B684B
:10C98000C3F388135A430B68C3F301435B1C5B007A
:10C99000B2FBF3F200E0434A02604B68424A04688B
:10C9A000C3F303139B5C24FA03F343604B684468AE
:10C9B000C3F382239B5C24FA03F3836049684368D2
:10C9C000C1F34231895C23FA01F1C16010BD00F46A
:10C9D00040723249B2F5407F06D10A68334B22F4E7
:10C9E000F81203401A430A6000058A6E52EA10509A
:10C9F000886670472E49086070472E490860704766
:10CA00002D4A0029116814BF084321EA0000106074
:10CA100070472A4A0029116814BF084321EA000020
:10CA200010607047264A0029116814BF084321EAA4
:10CA3000000010607047234A0029116814BF0843A2
:10CA400021EA0000106070471F4A0029116814BFD6
:10CA5000084321EA0000106070471C4A0029116851
:10CA600014BF084321EA0000106070474109084ADA
:10CA7000012908BF116803D002290CBF116F516F43
:10CA800000F01F0021FA00F000F0010070470000E4
:10CA90000038024070380240043802400838024032
:10CAA00000127A000024F4001C3C0020FFFCFF0F61
:10CAB0003C0E4742400E4742303802403438024074
:10CAC00040380240443802402038024024380240B6
:10CAD00010B586B001210220FFF792FFC020009020
:10CAE00002208DF804008DF8050001208DF8060065
:10CAF0008DF8070000A9CB4C2046FDF729FD042244
:10CB000007212046FDF772FD042206212046FDF78D
:10CB10006DFD01214FF40010FFF784FFC24C204649
:10CB20000DF032FD0020ADF80C0001214BF6FF7036
:10CB3000ADF80E003320ADF810004FF48060ADF872
:10CB400012004FF48040ADF81400B848029020461F
:10CB50000DF0A6FD02A920460DF03FFD06B010BD68
:10CB60002DE9F1430C46B04E1546012130460DF03B
:10CB7000A1FDFDF775FE0746AD4900F07AF818B93A
:10CB800000F073F81928F7D300F06FF8192828BFC0
:10CB9000012068D20022A02130460DF09FFDFDF754
:10CBA0005FFE0746A34900F064F818B900F05DF88D
:10CBB0001928F7D300F059F8192828BF022052D2BB
:10CBC0009DF8011030460DF09BFDFDF749FE07462C
:10CBD000DFF8648200F04CF818B900F046F8192824
:10CBE000F8D300F042F8192828BF03203BD29DF863
:10CBF000001030460DF084FDFDF732FE074600F0D0
:10CC000037F818B900F031F81928F8D300F02DF8EA
:10CC1000192828BF042026D2002700E07F1CAF423D
:10CC200016DA14F8011B30460DF06AFDFDF718FE08
:10CC3000814600F01DF820B94846FDF714FE19287A
:10CC4000F7D34846FDF70FFE1928E7D3781D0AE011
:10CC5000012130460DF038FD784890F8ED0308B119
:10CC6000FDF70CFE0020BDE8F2833846FDF7FBBD62
:10CC7000414630460DF049BD2DE9F14715461920D2
:10CC80000C4600FB05F6684F81B0012138460DF0D7
:10CC900011FDFDF7E5FD8046DFF8949100F0D7F82F
:10CCA00018B900F0D1F81928F8D300F0CDF81928F8
:10CCB00080F0B3800022A02138460DF00FFDFDF773
:10CCC000CFFD80465B4900F0C3F818B900F0BCF80E
:10CCD0001928F7D300F0B8F8192828BF022030D25D
:10CCE000012138460DF0DCFC9DF8051038460DF0AA
:10CCF00007FDFDF7B5FD8046DFF83CA1514600F089
:10CD0000A7F818B900F0A0F81928F7D300F09CF89C
:10CD1000192828BF032014D29DF8041038460DF0BE
:10CD2000EFFCFDF79DFD8046514600F091F818B9E3
:10CD300000F08AF81928F7D300F086F8192828BFE0
:10CD400004206DD2012138460DF0B4FCFDF788FDBA
:10CD5000804600F07CF818B900F076F81928F8D36E
:10CD600000F072F8192828BF052059D20122A0210D
:10CD700038460DF0B3FCFDF773FD8046304900F0F6
:10CD800067F818B900F060F81928F7D300F05CF8DC
:10CD9000192828BF062043D2FDF762FD8046DFF840
:10CDA000A490ADB2E5B1012D0CD103E000213846CD
:10CDB0000DF09CFC00F04BF80028F7D0012138461C
:10CDC0000DF082FC00F043F828B138460DF09AFCD3
:10CDD00004F8010B6D1E00F037F8B042E1D303E018
:10CDE00000F032F8B04202D3ADB2E81D18E00121E4
:10CDF00038460DF07BFCFDF733FD04464FF400315F
:10CE000000F026F820B12046FDF72DFD1928F5D3B6
:10CE10002046FDF728FD192801D3012000E000205D
:10CE2000BDE8F6870004024000540040305705007A
:10CE30000100030082000700840007006CC9012084
:10CE400002000300400003004046FDF70CBD4946C8
:10CE500038460DF05ABC00007CB5044600F036FAA6
:10CE6000054600F0E8F945EA40054CB1002000F025
:10CE700002F90446012000F0FEF8204345EA80054F
:10CE8000DFF8BC4994F86D0100F0010000F0F3F800
:10CE9000064600F08AF8C00040EA860600F0B6FBBD
:10CEA00046EA001005434CD00020FBF7E8FADFF813
:10CEB0009469E80706D500F04EF80FF6EC12C8208A
:10CEC000FBF721FBA80706D500F045F80FF6EC129A
:10CED000B420FBF718FB680706D500F03CF80FF606
:10CEE000F012A020FBF70FFB280706D500F033F85F
:10CEF0000FF6F0128C20FBF706FBE80606D500F0D3
:10CF00002AF80FF6F4127820FBF7FDFA00F023F868
:10CF10000FF6F8121E20FBF7F6FA002001903346B8
:10CF20004FF4FC60009000210FF6F8120A20FBF786
:10CF3000EAFADFF8140901780029FCD00020FBF799
:10CF40009EFA002084F8F905C4F8FA0584F8000672
:10CF5000C4F8010673BD0020019033464FF47840B9
:10CF60000090002170471CB513465A1EDBB111F822
:10CF7000013B8DF80430002306E09DF804305B0887
:10CF80008DF80430009B5B1C0093009B082BEBDAB0
:10CF900043089DF80440C0B26040C0074CBF83F016
:10CFA0008C001846E9E7C0B216BD30B583B0002545
:10CFB000042201A90020FFF75FFE01220DF101010B
:10CFC0000420FFF759FE012200A90520FFF754FEB7
:10CFD000284601A9415C4D19401CEDB20428F8DB3C
:10CFE0009DF80100DFF85848854204BF9DF8000015
:10CFF000642822D0FFF76CFD042201A92020FFF74E
:10D000003BFE01220DF101012420FFF735FE012234
:10D0100000A92520FFF730FE0025002001A9415C72
:10D020004D19401CEDB20428F8DB9DF80100854243
:10D0300004BF9DF80000642807D12078019904EB13
:10D040008000C0F8011000203EBDFFF741FD2078B0
:10D05000DFF8F81751F8302001EBC00104EB800035
:10D06000496889184908C0F801100121DFF8E00774
:10D07000017001203EBD2DE9F0414FF480634FF473
:10D08000C06618B14FF400634FF42066DFF8C48720
:10D090004FF4B37241461846FFF7EEFD40F26514B7
:10D0A00000F0B0FA08F5B277DFF894577978884243
:10D0B00004BF98F86401642810D0FFF709FD4FF40D
:10D0C000B37241463046FFF7D7FD00F09BFA7978FE
:10D0D000884204BF98F8640164280AD14FF4B372FF
:10D0E000414628460DF01EFB0020FDF701FF002001
:10D0F0006AE0FFF7EDFC0020FDF7FAFE0220287041
:10D100000020DFF8481701EBC00351F830205B68BE
:10D110009A1805EB80035208C3F80120002305EBA1
:10D120004002A2F86D304219042382F8BE30401C40
:10D13000032382F8F43082F8D930002382F81231C8
:10D1400082F82D311B28DEDB00204119012281F8F5
:10D15000A330401C81F848210328F6DB0320411945
:10D16000401C81F8A32081F848210A28F7DB0A2017
:10D170004119042281F8A320401C012281F8482192
:10D180001B28F5DB85F86231022085F8630185F8FC
:10D190000F3185F8103185F811312246DFF8B806D5
:10D1A000C5F869002946052085F8BD00642085F88A
:10D1B0006401FFF7D8FE85F86501002000F006F84D
:10D1C000012000F003F80120BDE8F081F8B54FF42C
:10D1D00080644FF4C06518B14FF400644FF42065CB
:10D1E000DFF87066DFF858164FF4B37230460DF072
:10D1F00099FA40F26512314600F006FA86F86501A8
:10D20000002704EB4710202206EB471100F043FBF8
:10D210007F1C0C2FF5DB002405EB4410202206EBCD
:10D22000441100F038FB641C0C2CF5DBBDE8F24027
:10D230000020FDF75DBE70B5DFF8046606F26614E7
:10D240000A2221464FF40070FFF716FD09223146ED
:10D2500000F0DAF906F5B275E97A884204BF96F86B
:10D260006401642811D0FFF733FC0A2221464FF4F1
:10D270004070FFF701FD0922214600F0C5F9E97A67
:10D28000884204BFA87A642801D1002070BDFFF74E
:10D290001FFC0020A870E870092201202871214697
:10D2A000022068710120A8710020E871287268725C
:10D2B0006420A872FFF757FEE872DFF8A005017836
:10D2C00041F002010170012070BD00002DE9F04124
:10D2D000DFF86C4504F5B8754FF4207229464FF419
:10D2E0004060FFF7C9FC40F27F284246294600F023
:10D2F0008BF904F2E737397A884204BFF879642859
:10D3000012D0FFF7E5FB4FF4207229464FF480500E
:10D31000FFF7B2FC4246294600F076F9397A884296
:10D3200004BFF879642801D1002067E1FFF7D0FB42
:10D3300004F2DA306421C1708822002184F870116F
:10D340009FEDAF0A4FF40061A4F8711110EE103A8E
:10D350004BF68031C4F873114FF4FA7604F273116E
:10D360000A7102224A7101228A71FA22CA710A7272
:10D3700004F5BE72136004F5C072DFF8E434136084
:10D380002B224A74232303228A740222CA743C2269
:10D390000A754FF42F7104F5C472A4F888119370C4
:10D3A0000323D37001231371062353711423937144
:10D3B0000123D371DFF8AC349360DFF8AC34D36071
:10D3C000DFF8A8341361DFF8A83453610223137720
:10D3D000537706239377D37740F28A231384C823A5
:10D3E00053844FF4E173D38440F2EE231385C823B2
:10D3F00053854FF47A739385C823D38540F6FC0395
:10D400001386C823538640F6282393867823D38631
:10D4100040F6043313877823538740F6CC33938741
:10D420001423D3874FF44362A4F8C821002304F5E2
:10D43000E472538044F26823938040F68C23D380B7
:10D4400040F61C4313814FF47A63538141F27073A9
:10D4500093814FF4FA53D38142F21073138242F650
:10D46000E063538245F6C0539382C823D3824FF4BE
:10D47000967313834FF4C873538396834FF41676D1
:10D48000D6834FF4487616844FF4966656844FF050
:10D49000000C4FF4AF669684062284F8EE21042631
:10D4A00040F6D862C4F8EF21DFF8C823C4F8F321AE
:10D4B00010EE102AC4F8F72104F2EF121673567416
:10D4C0000726567396746FF001069673D67401267C
:10D4D000D67316756FF0080616745675C4F826C212
:10D4E00004EB8C0E4FF07E56CEF82A620CF1010C44
:10D4F0000026CEF896624FF07E56CEF802630026E4
:10D50000CEF86E63BCF11B0FEADB4FF0320C84F8EF
:10D51000DAC380F801C09FED690A4FF05A0C80F819
:10D5200002C04FF0200C82F816C04FF0400C82F879
:10D5300017C0D14ADFF844E3C4F8072210EE102ADE
:10D54000C4F80B22202284F80F2204F20F2282F862
:10D5500001C0DFF82CC3C4F811C210EE10CAC4F821
:10D5600015C24FF0210C82F80AC04FF0190C82F856
:10D570000BC04FF0010C82F80CC004F5077CCCF80E
:10D5800000E081804FF03C0C0121817182F811C0D4
:10D590000A21C1714FF0640C1421817203811E2194
:10D5A000C17282F812C00521017340F64F40A4F801
:10D5B000E7034FF0010C82F813C042F67A3078800E
:10D5C0004FF0280C82F814C02E2038714FF0640CF4
:10D5D00082F815C04B2078714FF0010C82F816C00C
:10D5E0006420BE71F87142462946FFF7BCFC3872D0
:10D5F0009A48017841F0040101700120BDE8F081F2
:10D600008FC2F53D224641466420ACE410B59D4CE6
:10D61000232221464FF4A050FFF72EFB00F03EF9E5
:10D6200094F82210884204BF94F82100652811D094
:10D63000FFF74EFA232221464FF4C050FFF71CFBA0
:10D6400000F02CF994F82210884204BF94F82100CD
:10D65000652801D1002010BDFFF73AFA8D22232161
:10D6600020460DF065F8DF20207022223C206070FB
:10D6700021462320A0700720E0708C2020715F20BD
:10D6800060717820A071CD20E071232020720A20E3
:10D690006072A072E0722073322060730720A07362
:10D6A000652084F82100FFF75EFC84F822006B48B7
:10D6B000017841F008010170012010BDBD378635A9
:10D6C00070B5634D5E4C28788CB0A8B3207804EB1D
:10D6D00080000026D0F801000290002002A9415CE1
:10D6E0008E19401CF6B20428F8DB042202A903A814
:10D6F0000DF018F803A8642141710671062203A9F0
:10D700000020FFF72DFAC2B27AB15F4E4BA130462E
:10D71000FDF7C6F8002001904FF4784000903246A3
:10D720005A4B0021AF20FAF7EEFE062203A9202073
:10D73000FFF716FA00202870484D287880071ED57C
:10D74000092204F5B371FFF75FFF84F86F0100262B
:10D750007001011900F5007000F09AF8761C0C2E8B
:10D76000F6DB00267001011900F5407000F090F81A
:10D77000761C0C2EF6DB287800F0FD002870287847
:10D78000C00709D594F86D0100F00100FFF71EFDF8
:10D79000287800F0FE0028702878400725D540F250
:10D7A0007F2204F5B871FFF72FFF84F8EF030026FE
:10D7B0007001011900F54060202201F5B87100F0F8
:10D7C0006AF8761C152EF3DB00267001011900F5AE
:10D7D0008050202201F5B87100F05DF8761C152EFE
:10D7E000F3DB287800F0FB0028702878000722D5AA
:10D7F000244C00F053F884F82200202221464FF4F4
:10D80000A050FFF7ADF9202204F120014FF4A15000
:10D81000FFF7A6F9202221464FF4C050FFF7A0F9E8
:10D82000202204F120014FF4C150FFF799F9287824
:10D8300000F0F70028700CB070BD000025326400C5
:10D840006CC90120343C00200C3A0020845A0308A3
:10D85000F5DC012074CF0120A0F33F04C931002082
:10D8600014AE473F965673074BC3C9010024F4001A
:10D87000AAA97D018FC2753D17B751380060EA46ED
:10D88000ACC52737A43100202CC901202C3C002036
:10D89000202201F5B37180B2FFF762B9222221463E
:10D8A0006520FFF760BB00004652414D2053657470
:10D8B0007570202072656C6F616400004652414DA6
:10D8C0002053656C6563742072656C6F6164000041
:10D8D0004652414D204D6F646520202072656C6F6B
:10D8E000616400004652414D20467265712020203F
:10D8F00072656C6F616400004652414D20436F6C4D
:10D900006F72202072656C6F61640000506C6561FD
:10D91000736520436865636B2053657474696E6733
:10D92000730000005072657373204D2E53454C20D8
:10D93000746F20636F6E74696E756500C91C036F28
:10D9400000228908B3EB810F06D3A3EB81020267A3
:10D95000C26E02EB8101C166104670472DE9F047A7
:10D96000804689461646002E54D0112E50D319F801
:10D97000012B113E1709EE2002F00F04024247D19D
:10D9800010214046FFF7DAFF5FEA000A30D008EBCB
:10D99000C40000EB87040021C4F824A0002519F876
:10D9A000010B01F80A004519491C1029F7D3690039
:10D9B0004046FFF7C3FFD8B10021606300220B4649
:10D9C00011F80AC003E020F813205B1C521C5FEA28
:10D9D0000C0EAEF1010CF6D15200491C1029EFD308
:10D9E000AE4215D3761B29464046FFF7A7FF08B97C
:10D9F000032010E06064002102E000F8012B491CC4
:10DA0000A942B0D219F8012B002FF6D10C2AF4DB71
:10DA1000062000E00020BDE8F0872DE9F843044629
:10DA200000256768267B20683A788846A9469EB913
:10DA300028B900F091FC18B96FF001001CE07F1CC0
:10DA40003A78401ED5B1002512B16FF0050013E001
:10DA5000FF21FF22397080264FEA4909324218BF60
:10DA600009F101097608A8F10108B8F1000FDED12B
:10DA70002673206067604846BDE8F283FF2AEAD13A
:10DA80000125F2E72DE9F24F044690466568277BB1
:10DA900021682A7800269B46B1464FF0100AB7B994
:10DAA00059B9A568636F4FF400722946204698471C
:10DAB000010003D16FF001002FE06D1C2A78491E90
:10DAC00096B100263ABBFF20FF22287080274FEA3C
:10DAD00049093A4218BF09F101090098401C009019
:10DAE0007F08401E007806E0FF2AEFD101260FE0F4
:10DAF0000BF1010B401E48B138F8023B9945F7D1B4
:10DB00002773216065609BF8000006E0AAF1010A16
:10DB1000BAF1000FC3D16FF00500BDE8F28F2DE917
:10DB2000F04F4FF0080E0268D0F88050046CD0F827
:10DB3000C060D0F8E080D0F820C0D0F860A0AB186A
:10DB4000551BA21B4FF4B5577A431213A419161B89
:10DB5000E2181B1BAC19AD1BD0F8A070ACEB08068B
:10DB6000E044A7EB0A0907EB0A0CA8EB0C074FF4FB
:10DB7000B55A0AFB07F7E04409EB060C41F6905A48
:10DB80000AFB0CFC42F6CF1A4FEA2C3C0AFB09F9BF
:10DB9000ACEB29393F13A9EB0809A7EB090A41F2BD
:10DBA00051177E4308EB02070760A2EB0802C0F89A
:10DBB000E020ACEB263609EB04020262A6EB0A0673
:10DBC000A4EB0902C0F8C0200AEB05020264A5EB31
:10DBD0000A02C0F8A020F21802669A1BC0F8802042
:10DBE000001DBEF1010E9ED120384FF0080E0FF639
:10DBF00038070268056984688669D0F80490D0F80F
:10DC000014C0D0F80CA002F50042AB18551BA21BA3
:10DC10004FF4B55808FB02F21213A419161BE218B0
:10DC20001B1BAC19D0F81C80AD1BA9EB0806C8441F
:10DC3000ACEB0A09D444A8EB0C0A4FF4B55B0BFB20
:10DC40000AFAE04409EB060C41F6905B0BFB0CFC76
:10DC500042F6CF1B0BFB09F941F2511B4FEA2C3C5A
:10DC60000BFB06F6ACEB2939ACEB263608EB020CC5
:10DC70004FEA8C3C4FEA9C5CA2EB08021CF807C000
:10DC800081F800C09203920DA9EB0809D25DCA7118
:10DC90004FEA2A3A09EB04029203920DAAEB090A11
:10DCA000D25D4A70A6EB0A06A4EB09029203920D1C
:10DCB0002030D25D8A710AEB05029203920DD25D8B
:10DCC0008A70A5EB0A029203920DD25D4A71F21896
:10DCD0009203920DD25DCA709A1B9203920DD25D8F
:10DCE0000A710831BEF1010E83D1BDE8F08F2DE934
:10DCF000F04F804685B0D8F8640000904FF0000ADD
:10DD000098F80E0098F80F1048430190D8F86890E2
:10DD10001DE00120691E00FA01F10E4204BFA6EBCE
:10DD20004100461C0FF24060205C57F82010009A1A
:10DD30007143091242F82010641C402C51D3009802
:10DD40004946FFF7ECFE09F140090AF1010A019882
:10DD5000801C824566D20198824502D200270020AD
:10DD600005E0AAEB0000471C380018BF012008EBB3
:10DD7000C004636C626B616A4046FFF783FE054630
:10DD8000002D38D408EB470BBBF9146012D029469C
:10DD90004046FFF742FE002801D5404240E0012105
:10DDA0006A1E9140084204BFA0EB4100401C861946
:10DDB000ABF8146007EB0800007C009908EB8000CA
:10DDC000476D3868704300120860FC210098001D00
:10DDD0000CF0E2FCA06A0390A06B0290D4F848B06B
:10DDE0000124029A03995B464046FFF74BFE054625
:10DDF000002DA4D001D5684212E0280904D00419EE
:10DE0000402C01D306200EE015F00F0594D02946D2
:10DE10004046FFF702FE0646002E7FF57AAF7042BD
:10DE200040B200E00020D0E02DE9F04F85B0C47B87
:10DE3000837BE4000194DB00C4695D18AC422CBF15
:10DE40001C46641A019E056AB618B5422CBF019D96
:10DE5000AD1AADF8081000956118491EADF80A100A
:10DE6000ADF80C20002500998918491EADF80E1058
:10DE70000FF2B452416E00E06D1C019EB54269D2B2
:10DE8000876EDDF804C007EBC506BCF1100F09D1A1
:10DE90004FEA550C07EBCC0707F5807E082D05D31C
:10DEA000403603E005EB030C07EBCC0E00273EE009
:10DEB0000EF1010E40F29B5A0AFB09FA16F8018B8B
:10DEC0004FEA6A2B0AEB9B5A08EBAA2A4FEA8A5AB6
:10DED0004FEA9A5A40F2DB2B1AF802A001F801AB84
:10DEE0000BFB09F94FF4B07A0AFB0C994FEA692A47
:10DEF00009EB9A59A8EBA9294FEA89594FEA995990
:10DF00007F1C19F8029001F8019B40F2167909FB79
:10DF10000CFC4FEA6C290CEB995C08EBAC2C4FEA3B
:10DF20008C5C4FEA9C5C1CF802C001F801CB9F425C
:10DF3000A2D29EF800C09EF84080ACF1800CA8F1FF
:10DF40008009102BB4D1082F08BF383607F001081C
:10DF5000C644AFE7417B23FA01F18C4216D2426EF0
:10DF6000134600250DE000F033F8761C00F030F881
:10DF700000F02EF8A642F6D30E1B06EB4606F31869
:10DF80006D1C009EB54238BF0026F3D3416E009D44
:10DF90000A4613466C4312F8015B12F8016B05F058
:10DFA000F8052D0206F0FC0645EAC60512F8016BDD
:10DFB00045EAD60523F8025B641EECD1836F02AA02
:10DFC0009847401E8041C00F40B205B0BDE8F08FB9
:10DFD00013F8017B02F8017B70472DE9F84F0446E6
:10DFE0000A980AB9052041E1E26623676167E067A4
:10DFF000002300206083002104EBC00202EB8102B9
:10E00000491C5362536353640229F5D3401C022810
:10E01000F1D30020024604EB8001401C4A6504282D
:10E02000F9D34FF4007100F023F90600A66000F068
:10E030000181022200F01FF9022840F01681307899
:10E04000717841EA00204FF6D87188421CD14FF018
:10E0500002090FF2143740F2012804E03078717899
:10E0600041EA00206083042200F005F9042861D110
:10E0700030787178F27841EA0020B17842EA0122E2
:10E08000032A71D3010AFF2940F0C080951E291D83
:10E09000C0B28944C03817D0401E022808D9C01E1B
:10E0A00049D0401E022881BF001F0228001F0228FD
:10E0B00040F2D1800C38FBD0401E00F07780401E2B
:10E0C00048D0801E30D0C8E0454571D200F0D7F866
:10E0D000A8422FD1F078317941EA0020E061B1788F
:10E0E000707841EA00202062707903286ED1002008
:10E0F00000EB40018919CA7950B9112A1CBF222AA4
:10E10000212A63D11309A37302F00F02E27301E025
:10E11000112A5BD10A7A042A80F29D800119401CE1
:10E120000A740328E4D39EE7454541D200F0A7F8DE
:10E13000A84293D099E045453AD200F0A0F8A84211
:10E14000F8D12A4631462046FFF708FC40B20028A5
:10E150002FD188E745452BD200F091F8A842E9D1AC
:10E16000B246002DF5D0412D50D31AF801BB413DE8
:10E170001BF0F0004AD14FF4807100F079F80028CC
:10E1800058D00BF0030104EB810148650021CA5D02
:10E190000FF2142C1AF8013B3CF812C00CFB03F3ED
:10E1A00040F82230491C4029F1D3DAE7454501D334
:10E1B00004205BE000F063F8A84256D1E069002833
:10E1C0001CBF206A002821D03078032843D10020CA
:10E1D00006EB40018A78002A18BF112A3BD10200C1
:10E1E00018BF012204EBC2014A6A7AB1896A69B197
:10E1F0000119097C04EB8101496D39B1401C0328E8
:10E20000E6D3E07BA17B11FB00F70FB906202DE0E0
:10E21000F80100F14005FF2D98BF4FF480752946A5
:10E2200000F026F8606628B1B81C810100F020F8E3
:10E23000A06608B9032019E04FEAC950C00DC0F527
:10E24000007200F018F880B1401E206066608020E7
:10E25000207300200AE0082008E0636F2A460021AE
:10E2600020469847A8423FF4FEAE0220BDE8F28F58
:10E270002046FFF763BB636F314620461847636F44
:10E280002A463146204618472DE9F84F0446A16733
:10E290000AB105205EE0002060730026A07B4FEAF3
:10E2A000C009E07BC00000900020A082E0822083B3
:10E2B0000546834601E000998B44216A8B4549D28B
:10E2C0004FF000082FE000F047F800283FD03978E1
:10E2D000401E41EA05218DB2BAF1010A33D16760CF
:10E2E00020604FF6D8710020207301EA05004FF638
:10E2F000D071884201BF05F00700B6B206F00701F1
:10E30000884226D10020A082E0822083761C01254D
:10E310002046FFF7ECFCE8B95A4641462046FFF795
:10E3200083FDB8B9C844E1698845C4D2608B002830
:10E33000EED029464D1C89B28142E9D16768206838
:10E3400000254FF0020A0028BDD07F1CBFE7022045
:10E3500000E00620BDE8F28FA768636F4FF40072FB
:10E360003946204618470000000108100902030A38
:10E3700011182019120B04050C131A212830292218
:10E380001B140D06070E151C232A313839322B2495
:10E390001D160F171E252C333A3B342D261F272E12
:10E3A000353C3D362F373E3F0020622CCF29A0253B
:10E3B000002024195111D408622C903DFE393134CB
:10E3C000622CDF2205183E0CCF29FE39A0362931F8
:10E3D000CF29D920A016890BA025313429313E2C14
:10E3E000A025901D5D14610A0020622CCF29A02574
:10E3F000002024195111D4082419DF22D920901D9E
:10E400002419C1139B0DEF0651110518A0165D14B8
:10E4100051119B0D5F09C704D4083E0C890B610A9A
:10E42000D408EF06C7046F020001020304050607C3
:10E4300008090A0B0C0D0E0F1011121314151617E4
:10E4400018191A1B1C1D1E1F2021222324252627D4
:10E4500028292A2B2C2D2E2F3031323334353637C4
:10E4600038393A3B3C3D3E3F4041424344454647B4
:10E4700048494A4B4C4D4E4F5051525354555657A4
:10E4800058595A5B5C5D5E5F606162636465666794
:10E4900068696A6B6C6D6E6F707172737475767784
:10E4A00078797A7B7C7D7E7F808182838485868774
:10E4B00088898A8B8C8D8E8F909192939495969764
:10E4C00098999A9B9C9D9E9FA0A1A2A3A4A5A6A754
:10E4D000A8A9AAABACADAEAFB0B1B2B3B4B5B6B744
:10E4E000B8B9BABBBCBDBEBFC0C1C2C3C4C5C6C734
:10E4F000C8C9CACBCCCDCECFD0D1D2D3D4D5D6D724
:10E50000D8D9DADBDCDDDEDFE0E1E2E3E4E5E6E713
:10E51000E8E9EAEBECEDEEEFF0F1F2F3F4F5F6F703
:10E52000F8F9FAFBFCFDFEFFFFFFFFFFFFFFFFFF17
:10E53000FFFFFFFFFFFFFFFFFFFFFFFFFFFFFFFFEB
:10E54000FFFFFFFFFFFFFFFFFFFFFFFFFFFFFFFFDB
:10E55000FFFFFFFFFFFFFFFFFFFFFFFFFFFFFFFFCB
:10E56000FFFFFFFFFFFFFFFFFFFFFFFFFFFFFFFFBB
:10E57000FFFFFFFFFFFFFFFFFFFFFFFFFFFFFFFFAB
:10E58000FFFFFFFFFFFFFFFFFFFFFFFFFFFFFFFF9B
:10E59000FFFFFFFFFFFFFFFFFFFFFFFFFFFFFFFF8B
:10E5A000FFFFFFFFFFFFFFFFFFFFFFFFFFFFFFFF7B
:10E5B000FFFFFFFFFFFFFFFFFFFFFFFFFFFFFFFF6B
:10E5C000FFFFFFFFFFFFFFFFFFFFFFFFFFFFFFFF5B
:10E5D000FFFFFFFFFFFFFFFFFFFFFFFFFFFFFFFF4B
:10E5E000FFFFFFFFFFFFFFFFFFFFFFFFFFFFFFFF3B
:10E5F000FFFFFFFFFFFFFFFFFFFFFFFFFFFFFFFF2B
:10E60000FFFFFFFFFFFFFFFFFFFFFFFFFFFFFFFF1A
:10E61000FFFFFFFFFFFFFFFFFFFFFFFFFFFFFFFF0A
:10E62000FFFFFFFFFFFFFFFF0000000000000000F2
:10E6300000000000000000000000000000000000DA
:10E6400000000000000000000000000000000000CA
:10E6500000000000000000000000000000000000BA
:10E6600000000000000000000000000000000000AA
:10E67000000000000000000000000000000000009A
:10E68000000000000000000000000000000000008A
:10E69000000000000000000000000000000000007A
:10E6A000000000000000000000000000000000006A
:10E6B000000000000000000000000000000000005A
:10E6C000000000000000000000000000000000004A
:10E6D000000000000000000000000000000000003A
:10E6E000000000000000000000000000000000002A
:10E6F000000000000000000000000000000000001A
:10E700000000000000000000000000000000000009
:10E7100000000000000000000000000000000000F9
:10E7200000000000000000000000000000000000E9
:10E7300000000000000000000000000000000000D9
:10E7400000000000000000000000000000000000C9
:10E7500000000000000000000000000000000000B9
:10E7600000000000000000000000000000000000A9
:10E770000000000000000000000000000000000099
:10E780000000000000000000000000000000000089
:10E790000000000000000000000000000000000079
:10E7A0000000000000000000000000000000000069
:10E7B0000000000000000000000000000000000059
:10E7C0000000000000000000000000000000000049
:10E7D0000000000000000000000000000000000039
:10E7E0000000000000000000000000000000000029
:10E7F0000000000000000000000000000000000019
:10E800000000000000000000000000000000000008
:10E8100000000000000000000000000000000000F8
:10E82000000000000000000030B583B0012104208A
:10E83000FEF7E6F80220009001208DF80400022087
:10E840008DF805000020ADF8060000A9464C2046D2
:10E85000FBF77EFE00F02AF8444D284600BF401E1C
:10E86000FCD1002200F023F800BF6D1EFCD100F0A7
:10E870001DF80F2000BF401EFCD103F04FFD42F2F7
:10E88000010422460321072003F0B0FD2246812126
:10E89000012003F0ABFD22461021062003F0A6FD67
:10E8A00022460221072003F0A1FD37BD01220221EB
:10E8B0002046FBF796BE10B52D4C94F8690148B977
:10E8C0004FF40052642100F055F84FF400526421D7
:10E8D00000F053F894F86901012809D14FF400526F
:10E8E000142100F047F84FF40052142100F045F8CD
:10E8F00094F86901022809D14FF400520C2100F06C
:10E9000039F84FF400520C2100F037F894F86901FF
:10E91000032809D14FF40052062100F02BF84FF4E0
:10E920000052062100F029F894F86901042809D161
:10E930004FF40052022100F01DF84FF40052022162
:10E9400000F01BF894F8690105280CD14FF400522F
:10E95000002103F04BFDBDE810404FF400520021B0
:10E96000042003F043BD10BD00080240FFFF0F006C
:10E970006CC90120052003F039BD042003F036BD29
:10E980001CB574486421017008200121FEF738F895
:10E9900000F039F801208DF807008DF80500FF2000
:10E9A000009000A96C4C2046FBF7D2FD0022FF210D
:10E9B00000F033F800F034F801210120FEF720F8D0
:10E9C00000F021F84FF48060009000A9634C2046CD
:10E9D000FBF7BEFD4FF480612046FBF700FE0121EE
:10E9E0000846FEF70DF801208DF8040000A900206C
:10E9F0008DF806004FF4407000902046FBF7A8FD0C
:10EA000000F008F813BD01208DF8040000208DF8F7
:10EA10000600704700224FF440712046FBF7E1BD2D
:10EA2000F8B54F4C4F49207804EB8000D0F8010036
:10EA3000884238BF00251DD34B49884238BF012585
:10EA400018D34A49884238BF022513D3484988421F
:10EA500038BF03250ED34749884238BF042509D360
:10EA60004549884238BF052504D34449884234BF0C
:10EA70000625072594F8F00508B145F08005354EC8
:10EA800031788D4213D0344F0022FF213846FBF7F6
:10EA9000A8FD94F8F00510B10122012103E08020C7
:10EAA000012220FA05F13846FBF79BFD3570F1BDD8
:10EAB00010B52B48294C017808184FF4806190F864
:10EAC0002D01012820461CBFBDE81040FBF787BD83
:10EAD000FBF785FD2046BDE810404FF48061FBF751
:10EAE0007CBD38B51E4D1D4C2878401990F8120198
:10EAF00008B9FFF78FFF2878401990F81201012814
:10EB000009D101224FF40071FFF787FF00224FF473
:10EB10008071FFF782FF2878401990F812010228CF
:10EB200009D101224FF48071FFF777FF00224FF4E3
:10EB30000071FFF772FF2878401990F8120103283E
:10EB400007D12046BDE8384001224FF44071FBF761
:10EB500048BD31BD5A3C0020000C0240000002407C
:10EB60006CC9012080841E00C0FB390000DD6D00EF
:10EB7000602A9D00C0E1E40000623D0140B6C6018C
:10EB800010B5474C94F88B010228B8BF0BF008FE73
:10EB900094F88B01022808BF0BF001FF94F88B0159
:10EBA00003280BD10CF02EF8207804EB8000BDE890
:10EBB0001040D0F8010040000CF026B810BD38B568
:10EBC000374D044695F88B010228BCBF20460BF058
:10EBD0005FFE95F88B01022804BF20460BF0EBFF87
:10EBE00002F05BFEBDE83140FFF71ABFF8B5014601
:10EBF0002B480278141800EB820394F8A350062DDA
:10EC00000BD194F8F440D3F8013000EB4404B4F88D
:10EC1000CE41640813FA84F32BE094F8A360B0F8B3
:10EC2000DE53022E03D1D3F80130EB1821E0032E7E
:10EC300003D1D3F801305B1B1BE094F8A3C090F81C
:10EC4000F75540F274464FF47A77BCF1070F05D1BF
:10EC500005B13746D3F80130FB180AE06446082CAA
:10EC600005D105B13746D3F80130DB1B01E0D3F8FD
:10EC7000013000EB4202B2F86D4024040CD590F84C
:10EC8000F10548B9B2F86D00420447BF054A104388
:10EC90008004800C03FA80F3BDE8F4405800084774
:10ECA0006CC9012000C0FFFF30B58DB000F0B8F88E
:10ECB000DFF8640600218160C16081614FF4C87192
:10ECC000DFF858060BF068FD0F20019001A9032022
:10ECD0008DF8080000208DF80B00DFF84406FBF7E4
:10ECE00037FC0220019001A9DFF83806FBF730FC61
:10ECF00012208DF8000001208DF8010000208DF811
:10ED0000020001208DF8030000A8FBF7FCFD0121A3
:10ED10004FF44070FDF78FFE07A80BF0A8FF03A883
:10ED20000BF0BDFF0BF074FF0020079001208DF861
:10ED300020008DF82100002009900B908DF8300004
:10ED4000012003904FF4403004900020059006907D
:10ED500007A9DFF8D44520460BF067FF03A80BF0A6
:10ED600090FF032120460BF0DFFF07230322002141
:10ED700000F053F807230122012100F04EF802228F
:10ED80000723114600F049F800F03DF840F207452E
:10ED900000F03EF8012120460BF087FF01212046BC
:10EDA0000BF0D6FF20460BF0CEFF20460BF086FF7F
:10EDB000DFF8784507A920460BF037FF03A80BF0D2
:10EDC00060FF022120460BF0AFFF07230122032141
:10EDD00000F023F807230222092100F01EF800F0BA
:10EDE00012F800F015F8012120460BF05EFF01211A
:10EDF00020460BF0ADFF20460BF0A5FF20460BF0A0
:10EE00005DFF0DB030BD4FF4702120460BF094BF74
:10EE10000122294620460BF0B1BF20460BF05CBF13
:10EE2000F8B5DFF80C65DFF80C752DED028BB6F840
:10EE3000E70300EE100AB8EE408A18EE100A08F058
:10EE4000DBFF0022DFF8F03408F0FEFF0446B6F8DE
:10EE5000E90300EE100AB8EE400A0D4600F0E0F8B3
:10EE60000022DFF8D83408F0EFFF22462B4609F0E5
:10EE700053F90AF023FD9FED630A88EE000A38601B
:10EE800087ED010ABDEC028BF1BD00002DE9F843CE
:10EE9000DFF89864DFF8804440F207452DED048BDD
:10EEA000294630460BF075FF00B300F0B1F8E16A77
:10EEB00011FA80F0E062182100F0ABF8616B11FAF2
:10EEC00080F0616A491CFA290AD3E16AFA22B1FB8F
:10EED000F2F1A162B0FBF2F020630021E1620020B8
:10EEE00061626063294630460BF061FFDFF83864E9
:10EEF000294630460BF04DFF00287BD0DFF83094D8
:10EF0000DFF8188499F8F10501280BD100F080F89A
:10EF1000216A28F82100182100F07BF8216A08EB0B
:10EF2000810148801C2100F074F8E16911FA80F732
:10EF3000206A401C282853D399F8F105012849D1AB
:10EF400000200021024638F92230834228BF1846AB
:10EF500008EB8203B3F902308B4228BF1946521CDA
:10EF6000282AF0DB206161619FED248B94ED020A79
:10EF7000B8EE400A9FED249B00F052F853EC192B99
:10EF800009F0CAF894ED040A00F046F853EC182B87
:10EF900009F0C2F842464B460BF018F809F0A6F803
:10EFA000A06094ED030AB8EE400A00F039F853EC83
:10EFB000192B09F0B1F894ED050A00F02DF853EC87
:10EFC000182B09F0A9F842464B460AF0FFFF09F05A
:10EFD0008DF8E0602820B7FBF0F0A061002700204A
:10EFE0002062E76129463046BDEC048BBDE8F4435E
:10EFF0000BF0DDBEBDEC048BBDE8F183CDCCCCCCF9
:10F00000CCCCEC3F00007A4A9A9999999999B93FEA
:10F01000142130460BF0A5BE8046B8EE400A894662
:10F0200010EE100A08F0E8BE7CB5BB4CC44DA06AD7
:10F0300040F6A17188423CBF226B8A4215D3002062
:10F04000207000A9FF206070A07000208DF80400DF
:10F050008DF806004FF4F04000F090F9009901227D
:10F0600089B22846FBF7BDFA73BD21780229FBD08F
:10F0700031B9A080E280FBF7F3FBA063012048E1F7
:10F08000A06BFBF7F0FB0A28EED3A188A06AA1F1E0
:10F090000902904224BF0931814208D3E288216BE2
:10F0A000A2F10903994224BF09328A4201D2002009
:10F0B0002FE1A0F1A802EF2A0BD2A1F28A52EF2A87
:10F0C0003CBF01226270A1F64D12EF2A3CBF002224
:10F0D000627040F6F4668C22A0F67D60A680E28025
:10F0E000EF283CBFA1F11500EF2808D20D2000F059
:10F0F0003DF94FF4804000F041F900F031F940F261
:10F10000AA50E080A680A06AA0F67D60EF283EBFEE
:10F11000206BA0F23350EF2808D20E2000F026F921
:10F120004FF4005000F02AF900F01AF940F69C1054
:10F13000E080A680A06AA0F67D60EF283EBF206B2D
:10F14000A0F62510EF2808D20F2000F00FF94FF499
:10F15000805000F013F900F003F940F69E40E08083
:10F16000A680A06AA0F67D60EF283EBF206BA0F6C7
:10F170002740EF2808D2102000F0F8F84FF4006084
:10F1800000F0FCF800F0ECF840F6B560E080A16A11
:10F19000206BA1F2A152A0F63E60EF2A3EBFEF28FD
:10F1A00011226270A1F63E12EF2A3EBFEF28122212
:10F1B0006270A1F62742EF2A3EBFEF281322627049
:10F1C000A680A1F67D615F4D594EEF2938BFEF282B
:10F1D00002D21420607085E06078012810D196F882
:10F1E0006601401C86F86601C0B2082804BF0020F2
:10F1F00086F8660101F005FA287840F002002870D0
:10F20000607880B996F86601401E86F86601C0B243
:10F210000828A4BF072086F8660101F0F2F92878D3
:10F2200040F002002870607811281CD100F093F89B
:10F23000042907DA02291ABF032900F2BE0000F2EE
:10F24000D90000E0F430017809B908210170017893
:10F25000491E00F079F8FCF77EFE96F86601012859
:10F2600008BFFCF7D5FE607812281CD100F073F8B7
:10F27000042907DA02291ABF032900F2BE0000F2AE
:10F28000D90000E0F4300178491CC9B2082908BF50
:10F29000002100F059F8FCF75EFE96F8660101289F
:10F2A00008BFFCF7B5FE6078132818D130788019B4
:10F2B00090F8A30020B930788019092180F8A310B4
:10F2C00000F049F8491E80F8A31000F03EF8FCF762
:10F2D00042FE96F86601012808BFFCF799FE6078A7
:10F2E000142815D100F037F8491C80F8A31000F05D
:10F2F00032F8092904BF002180F8A31000F025F896
:10F30000FCF729FE96F86601012808BFFCF780FE8D
:10F310000220207073BD00004CDB012074D5012059
:10F320000000024000040240002101400020014092
:10F330006CC9012098DC012000404F4100408F4003
:10F3400000100240C93100200170287840F001000F
:10F350002870FCF71CBD3078801990F8A310704716
:10F360000099002289B22846FBF73BB9607000A9DA
:10F3700001208DF804008DF80600704700900120F0
:10F380008DF807008DF805002846FBF7E1B800006E
:10F390002DE9F043DFF8DC6BDFF8DC4B96F86D11FC
:10F3A000A07BDFF8D89B83B0C9070DD5FDF7B5F971
:10F3B00000F07FFB4B460FF2880200F06FFB00F07D
:10F3C00047F89AA2422116E0FDF7A7F900F071FB79
:10F3D0004B460FF2740200F061FB00F039F894A282
:10F3E0002C2100F05BFB00F0A7FC002101910090B4
:10F3F0004B46CBA2372100F051FB00F09DFC009062
:10F40000282796F86601DFF8448E002100F09CFD65
:10F4100096F86D014FF4FC6580074EBF2846A07B2F
:10F42000FDF77BF900F0ACFD307806EB4000B0F85A
:10F430006D00000402D400F07FFC054600F075BDAD
:10F4400056464F2D412F000056464F2D000000001C
:10F45000002001904B464FF4FC60009070472DE96E
:10F46000F843DFF8886CDFF8884C7078DFF8848C1C
:10F47000DFF8849CDFF8FC7ADFF8805C012804BFA9
:10F48000687800283AD100F087F8FDF79FFE97F8DA
:10F490006D01C1074CBF00F0FE0040F0010087F88D
:10F4A0006D0100F079F8FDF7E6FD4846FFF79EFB99
:10F4B00097F88B01032804BF4046FFF797FB00F045
:10F4C0006BF8FDF7B7F8FCF762FCFCF744FDFCF7BE
:10F4D000F5FEFCF708FFFCF741FFFCF74CFFFCF7DB
:10F4E0006AFFFCF7AAFFDFF89C0D0121017020786C
:10F4F00040F0030000F046FA01206870B07801285F
:10F5000004BFA878002808D1FDF760FE0120FDF7B0
:10F510005DFE01F076F80120A870F078012804BFA4
:10F52000E878002813D197F86D0181074CBF00F0EF
:10F53000FD0040F0020087F86D01FDF79DF801F035
:10F5400060F8207840F0020020700120E8703079E7
:10F55000012804BF287900281CD1387807EB400027
:10F56000B0F86D100A0446BF4904490C41F400414B
:10F57000A0F86D104846FFF739FB97F88B01032878
:10F5800004BF4046FFF732FB00F08BFC01F039F876
:10F5900001202871BDE8F18397F86D0100F00100AA
:10F5A00070472DE9FC47DFF8CCA9DFF8CC690AF2F7
:10F5B00066154FF4FC64687880074EBF2046B07B28
:10F5C000FDF7ABF8009028279AF8660100F0C6FC1A
:10F5D0006878C0074EBF2046B07BFDF79EF800F06C
:10F5E00029F800F108024B46582100F057FA6879D3
:10F5F000002812BF2046B07BFDF78FF800F01AF804
:10F6000000F110024B4600F048FA287910B900F0DA
:10F6100048F904460020019000944B469AF8660190
:10F6200017FB008000F1180279E30000420000009F
:10F6300041000000009000219AF86601019117FB3B
:10F6400000807047F8B5DFF8A46ADFF8A44A707844
:10F65000DFF82079DFF8A45A012804BF6878002871
:10F660000FD197F86701810754BF40F0020000F006
:10F67000FD0087F8670100F0A4FF00F0C2FF012041
:10F680006870B078012804BFA878002821D197F8C5
:10F690006701C1070BD440F0010000F043F810D11E
:10F6A00097F8DD03C0F164010122C9B206E000F061
:10F6B000FE0000F037F804D101228021042002F07E
:10F6C00095FE00F07EFFFCF7DFFE00F09AFF0120C0
:10F6D000A87007F26717F078012804BFE8780028BF
:10F6E0000AD13979481E8041C00F387100F0CAFA3A
:10F6F00000F087FF0120E8703079012804BF2879E5
:10F7000000280CD1F978481E8041C00FF87000F035
:10F7100058FFFCF7D1FE00F074FF01202871F1BD05
:10F720002F42000087F8670197F8F105012870471C
:10F730002DE9F043DFF83C88DFF89C7C08F2661581
:10F7400083B0E87818B90FF2F40100F0A7F8E87870
:10F75000012803D10FF2F00100F0A0F8E8780228A8
:10F7600003D10FF2F00100F099F8E878032803D1F3
:10F770000FF2EC0100F092F8E878042803D10FF2C0
:10F78000EC0100F08BF8E878052803D10FF2E801CE
:10F7900000F084F8DFF8E06700F083F8DFF8DC477A
:10F7A00000F087F923463A4600F078F900F079F83E
:10F7B0000090282798F86601DFF8909A00210191BF
:10F7C00017FB009000F108022346582100F066F96B
:10F7D00000F067F80090002198F86601019117FB8E
:10F7E000009000F057F968780C21084208D100F029
:10F7F00058F800F056F90FF28C02FE2100F04EF995
:10F80000687800F00C00042808D100F04AF800F0F5
:10F8100048F90FF27802FE2100F040F9687800F014
:10F820000C00082808D100F03CF800F03AF90FF27B
:10F830006402FE2100F032F9BDE8F78350575230E0
:10F84000302525200000000050575231302525205A
:10F8500000000000505752323025252000000000E3
:10F86000505752353025252000000000505752389F
:10F87000302525200000000050575231303025251A
:10F88000000000002020204D4943000020204C496A
:10F890004E45000020202055534200003846FAF71C
:10F8A000FFBFB07BFCF739BF2DE9F041DFF83C68C2
:10F8B000DFF8C0867078DFF84458012804BF687804
:10F8C000002811D108F267108178491C8170C9B2F3
:10F8D0000629A4BF00218170FCF76AFEFEF7EBFF4A
:10F8E00000F08FFE0120687008F2F157B078DFF861
:10F8F000EC4A012804BFA87800280DD198F8F1053A
:10F9000000280EBF012101200021797088F8F1152F
:10F9100000F038F80120A870F078012804BFE878DA
:10F9200000280FD198F8F10510B90221012202E058
:10F93000012000210022797088F8F12500F022F8DA
:10F940000120E8703079012804BF2879002817D1F8
:10F9500098F86701001D88F86701C0B200F00C013B
:10F960000929A4BF00F0F30088F86701DFF8B40D9F
:10F97000017841F00201017000F043FE012028717E
:10F98000BDE8F081207000F03CBE2DE9F043DFF8C7
:10F99000E855A87B83B0FCF7C0FEDFF8D895DFF808
:10F9A000AC88DFF8844D0090282699F86601002184
:10F9B00016FB00820191234600F070F899F81B02B3
:10F9C000000604D5002001904FF4FC6003E000F035
:10F9D0006DF8002101910090234699F8660116FB0D
:10F9E000008000F10802582100F058F809F266176B
:10F9F000B879002812BF4FF4FC60A87BFCF78DFE9D
:10FA00000090002199F86601019116FB008000F03A
:10FA100041F8B878012806D100F048F800F041F824
:10FA20000FF2500221E0022804D100F03FF80FF25B
:10FA30004C020EE0042806D100F038F800F031F84E
:10FA40000FF2400211E0082807D100F02FF80FF262
:10FA50003C0200F02EF8234607E0102808D100F001
:10FA600025F800F01EF80FF60C52FE2100F016F8F3
:10FA7000BDE8F783205A4F4F4D310000205A4F4FB9
:10FA80004D320000205A4F4F4D340000205A4F4F46
:10FA90004D38000000F110022346B0210020F8F795
:10FAA00032BD00210191009023467047A87BFCF7EE
:10FAB00034BE00900021019170472DE9F04FDFF82E
:10FAC0002C76DFF82C46DFF8AC84DFF8306683B0A4
:10FAD0007878012804BF7078002826D198F8F105BD
:10FAE00068B198F86301401C88F86301C0B2062829
:10FAF000A4BF002088F86301B8F8AA010DE000F067
:10FB0000BBF8491C80F8481100F0B6F80629A4BFDC
:10FB1000002180F84811B8F8A8010BF064FD00F04E
:10FB2000C0F9FCF78AFC01207070B878DFF8045C3B
:10FB3000012804BFB078002824D1FAF791FE28608C
:10FB400098F81B02010612D500200190009049A2EE
:10FB5000DFF8E43B0021CF20F8F7D5FCDFF8DC0B21
:10FB60000021017098F81B0200F07F0001E040F0D6
:10FB7000800088F81B02207840F00400FFF702FFA5
:10FB80000120B07040F2D17BB878DFF8B49BDFF889
:10FB9000B4AB012804BFB07801281BD100F006FDEA
:10FBA000584517D398F81B0240F0800088F81B02D4
:10FBB0009123207840F0040000F01BFD04F0A3F92D
:10FBC00000F074F902F046FC00208AF800000120E1
:10FBD00089F80000F878012804BFF078002813D1D4
:10FBE000FAF73EFE286098F86C01411E20788941A2
:10FBF000C90F40F0020088F86C112070FCF772FC0D
:10FC000000F0FFFC0120F070F878012804BFF078C4
:10FC1000012817D100F0CAFC584513D3012088F8F9
:10FC20006C0100F02FF8002000F047F907F0ACF865
:10FC300000F03CF902F00EFC00208AF800000120E0
:10FC400089F800003879012804BF307900280ED1E6
:10FC500098F86801400088F86801C0B2102804BF15
:10FC6000012088F8680100F0CCFC01203071BDE86B
:10FC7000F78F000053514C0098F80000404490F872
:10FC800048117047207840F002002070FCF72ABC31
:10FC90002DE9FC47DFF8DC82B74C98F80F014FF4F0
:10FCA000FC66002812BF3046A07BFCF736FD0090B2
:10FCB000282598F866010FF6CC29DFF8C0A20021AC
:10FCC00015FB009201915346FFF7E8FE08F20F176B
:10FCD0007878002812BF3046A07BFCF71EFD00F0AC
:10FCE00023F800F1080253465821FFF7D7FEB878F1
:10FCF00010B900F021F80646002001900096534606
:10FD000098F8660115FB009000F11002FFF7C5FEA0
:10FD100000F012F800F008F800F118025346FE2136
:10FD2000FFF7BCFEBDE8F3870090002198F866015C
:10FD3000019115FB00907047A07BFCF7EEBC2DE90C
:10FD4000F84FDFF8A853DFF8A8436878DFF824827B
:10FD5000DFF8E0B9DFF8A473012804BF7878002841
:10FD600012D1FAF77DFDCBF8000098F80F11481E6C
:10FD70008041C00F88F80F0100F093F8FCF7EEFA0D
:10FD800000F03FFC012078706878DFF8B499DFF864
:10FD9000B4A9012804BF7878012819D1DBF8000044
:10FDA000FAF761FDB0F5FA6F12D9012088F80F015A
:10FDB000FCF7D4FA00F019FC07F047FA00F076F8E7
:10FDC00002F048FB00208AF80000012089F80000BA
:10FDD00008F20F16A878012804BFB878002814D1BB
:10FDE000FAF73EFDCBF80000707820B90120707062
:10FDF0000BF0EDFC01E00020707000F052F8FCF711
:10FE0000BAFA00F0FEFB0120B870A878012804BF00
:10FE1000B878012818D1DBF80000FAF724FDB0F516
:10FE2000FA6F11D901207070FCF798FA00F0DDFB31
:10FE300007F092FA00F03AF802F00CFB00208AF882
:10FE40000000012089F80000E878012804BFF87854
:10FE500000280FD1B078401CB070C0B20428A4BFF5
:10FE60000020B07000F01DF8FCF7A5FA00F0C9FB07
:10FE70000120F8702879012804BF387900280ED1B4
:10FE800000F01BF807F0BBFA00F010F802F0E2FAFD
:10FE900000208AF80000012089F800003871BDE8D0
:10FEA000F18F207840F0010020707047002088F822
:10FEB000F905C8F8FA0502F089BE009091234FF4C5
:10FEC00080721421F8F794BC2DE9F043294E2A4C96
:10FED0003078801983B090F82D014FF4FC6500282C
:10FEE00012BF2846A07BFCF718FC0090282796F844
:10FEF000660100F033F83078801990F8120100287C
:10FF000012BF2846A07BFCF708FC0090002196F861
:10FF1000660100F019F8FFF70FFF00F031F896F8CE
:10FF2000F00510B9FFF708FF054600200190009585
:10FF30004B4696F8660117FB008000F11802FE217F
:10FF4000FFF7ACFDBDE8F783019117FB008000F1DE
:10FF500008024B4658210020F8F7D5BA0FF62408BE
:10FF6000DFF8C497002117FB008201914B46002067
:10FF7000F8F7C9BA6CC90120A4310020343C002034
:10FF80000090002196F86601019117FB008000F1B6
:10FF900010024B46B0210020F8F7B5BA2DE9F8431E
:10FFA000524F534C7878DFF8A057544E012804BFC5
:10FFB0007078002810D12878401990F82D114A1E29
:10FFC0009241D20F80F82D21FFF76BFFFCF776F9F5
:10FFD00000F017FB01207070B878012804BFB078DA
:10FFE000002817D12878401990F81211491C80F880
:10FFF00012112878401990F812110429A4BF002189
:020000040801F1
:1000000080F81211FFF74DFFFCF76DF900F0F9FAD7
:100010000120B070F878012804BFF078002850D192
:1000200095F80006DFF8D080DFF82097401C85F8AF
:100030000006C0B2042803DB002085F8000600E0BB
:1000400048B900F061F84046FEF7D0FD00F058F8DE
:1000500001D100F05FF895F8000601280AD10122CD
:1000600000F053F84046FEF7C1FD00F049F801D119
:1000700000F050F895F8000602280AD100F044F884
:100080000020FEF79CFD00F03BF802D1002100F0BB
:1000900042F895F8000603280BD1012200F035F84C
:1000A0000020FEF78CFD00F02BF802D1002100F0BB
:1000B00032F8FFF7F6FEFCF74AF800F0A2FA01204A
:1000C000F0703879012804BF307900280CD195F8F8
:1000D000F005411E8941C90F85F8F015FEF7A0FC17
:1000E00000F08FFA01203071BDE8F1830C3A002056
:1000F000C931002009AC0108BFEB0008043A002018
:1001000095F88B010328704700224FF40071484690
:10011000FAF767BA012100200BF090BB2DE9FC41F2
:1001200000F08EF800F09CF800F08CF800F0ACF8CD
:10013000BDE8F341FBF76CBFF8B5DFF81466DFF8F4
:10014000E4457078DFF80076DFF80856012804BF30
:100150006878002819D100F047F807DA02291ABF99
:10016000032900F2BE0000F2D90000E0F43001786B
:1001700009B9082101700178491E00F03BF8FBF72E
:10018000EAFEFBF745FF01206870B078012804BF44
:10019000A878002819D100F027F807DA02291ABF39
:1001A000032900F2BE0000F2D90000E0F43001782B
:1001B000491CC9B2082908BF002100F01BF8FBF751
:1001C000CAFEFBF725FF0120A870F078012801BFC7
:1001D000E87800280120E8703079012801BF2879EB
:1001E000002801202871F1BD3878C01990F8A310BB
:1001F000042970470170207840F001002070FBF75F
:10020000C6BD2DE9FC4100F01BF800F029F800F014
:1002100019F800F039F800F015F800F019F800F1BD
:1002200010024346FFF739FC00F00CF800F010F81C
:1002300000F118024346FE21FFF730FCBDE8F381D0
:10024000DFF81475B87BFCF768BA00008407010872
:100250000090002195F86601019114FB0060704741
:10026000DFF8E4540FF21C56DFF8BC840090282419
:1002700095F86601002114FB0062019143460020BD
:10028000F8F741B9F5DC01200090002195F86601EE
:10029000019114FB006000F1080243465821002040
:1002A000F8F731B92DE9F041DFF8A474DFF87444B0
:1002B0007878DFF89454DFF89C64012804BF7078E4
:1002C00000281AD12878401990F8A30020B928787E
:1002D0004019092180F8A31000F062F8491E80F847
:1002E000A310FBF754FDFBF736FE00F05EF8207814
:1002F00040F00100207001207070B878012804BF20
:10030000B078002817D100F04BF8491C80F8A310F2
:1003100000F046F8092904BF002180F8A310FBF77C
:1003200036FDFBF718FE00F040F8207840F00100A1
:1003300020700120B070F878DFF82084012804BF15
:10034000F078002811D1287808B91B202870287867
:10035000401E287000F08EF9012088F800002078F7
:1003600040F0010020700120F0703879012804BFAE
:100370003079002812D12878401C2870C0B21B2880
:10038000A4BF0020287000F075F9012088F8000053
:10039000207840F00100207001203071BDE8F0812C
:1003A0002878401990F8A3107047287805EB800052
:1003B000D0F80100FAF78BBE80B500F011F8DFF835
:1003C00088030FF2C03290F86601282111FB00204B
:1003D000BDE80240006A00472CC90120CB31002053
:1003E0002DE9F84F2DED028BD94FCE4CDFF870A3DD
:1003F000DFF834B3DFF85083CE4DD64E82B0F879B3
:100400004FF028099FED9A8A012804BFF07900284F
:1004100029D1FAF725FA286000F0CBF804D500F0CE
:10042000D5F88AED008A03E041F40041A0F86D1090
:1004300000F074F998F88B01032804BFC948FEF74F
:10044000D5FB98F86601072801D100F0A9F898F8C3
:10045000670140F0800088F86701207840F00300D1
:1004600020700120F071F879012804BFF07901288B
:1004700057D100F09BF8B0F57A7F52D900F099F887
:1004800004D500F0A3F88AED008A03E041F40041AE
:10049000A0F86D1000F042F998F88B01032804BF12
:1004A000B048FEF7A3FB98F86601072801D100F0D9
:1004B00077F898F8670141061BD500F0BF0088F86F
:1004C000670198F8F10540B9A348807BFCF725F94E
:1004D000FFF7EFFA5B4695A207E0002001905B462C
:1004E0004FF47840009092A20021BE20F8F70BF85C
:1004F0000BE040F0400088F86701FAF7B1F940F0EE
:10050000010099490860FCF7CDF898F8670140F0C0
:10051000800088F86701207840F0020020700220F7
:10052000F0713878002836D0307801281FD100F0DB
:100530003DF8B0F5FA6F2ED998F8660100280CBF87
:100540000720401E88F866019123207840F00200C1
:1005500000F04FF801F0A8FF02F038FB01F07AFF3D
:1005600078480021017001217548017013E098F866
:100570006601401C88F86601C0B2082804BF00204C
:1005800088F8660100F03DF800F01BF8012030709B
:10059000FAF766F9286002B0BDEC028BBDE8F18F76
:1005A0000FF2E01119FB0010406A00472868FAF7C3
:1005B0005AB998F8000008EB4000B0F86D100A0432
:1005C0007047207840F00200207070474904490CC1
:1005D000A0F86D10002001905B461F200090CA21FA
:1005E0000FF29812C820F7F78EBF9123207840F0C1
:1005F000010020704FF48072002000901421F8F761
:10060000F7B851480FF27C1290F86601282111FBCF
:100610000020406A004770B54E4C607901281CBF2D
:10062000A079012823D04A4D6879002804BFA87911
:1006300000281CD06879444E012809D13078401C2C
:100640003070C0B21B28A4BF0020307000F012F838
:10065000A879012808D1307808B91B20307030788B
:10066000401E307000F006F801206071A07170BD6E
:10067000F02374C970B5344C3C4B207853F830608B
:1006800004EB800103EBC005D1F80120B24224BF86
:100690006E68964206D253F830006A681018400817
:1006A000C1F801003222207804EB80003223D0F818
:1006B0000110B1FBF2F25A43891A18BFC0F80120A9
:1006C00000F02CF894F88B01032804BF2548FEF7AE
:1006D0008DFA207804EB8000D0F80100FAF7F7FCDF
:1006E0001E48012101700F48017841F0010101709D
:1006F000FBF7E4FDFBF7F7FDFBF749FBFBF72BFCF2
:10070000FBF79BFE012084F8F8050D4800780028CF
:1007100004BFBDE87040FFF774BF70BD1448FEF71A
:1007200065BA0000C9310020343C00205258000056
:1007300054580000D0DC01202C3C0020A0DC01201B
:10074000CA310020CB3100206CC9012000080240D2
:100750000C3A0020043A0020A4310020F5DC0120EE
:10076000D431002009AC0108CCDC0120845A0308F4
:10077000BFEB0008205A4F4F4D780000202020206A
:10078000200000004D4F44452D2020004D4F444592
:100790002B00000042414E442D2000002042414EDB
:1007A000442B0000A50201080302010846494C54ED
:1007B0002D20200046494C542B00000020202020F2
:1007C00020200000202020202020000039010108E6
:1007D0001D01010850524520202020004154542082
:1007E0002000000052464F4646200000202042597B
:1007F000425300009DFF0008C9FE0008414E4620FC
:1008000020202000444E52202000000020204E4294
:10081000202000002020204E424C00003FFD000818
:1008200091FC0008414743202020200053514C20D8
:100830002000000045515F5258200000205A4F4FC1
:100840004D310000BBFA00088BF9000850575220C8
:1008500020202000544F4E452000000044544F4EAD
:10086000452000002020204D49430000A9F8000841
:1008700031F70008534C5045202020004D4F4E4981
:100880002000000045515F545820000020204543BF
:10089000484F000045F60008A3F5000856464F20D3
:1008A000412F42002020413D420000002053504C87
:1008B0004954000020202052495400005FF40008F1
:1008C00091F3000870B582B04FF6FF740094962340
:1008D000942296212C20F7F71BFF4FF478400090CC
:1008E000962300F053F8A0230094942219462C205C
:1008F000F7F70EFF4FF478400090A02300F046F881
:10090000002000909F23FC2298212C20F7F759FF0C
:10091000DFF8AC060021416001602C250E4622461E
:10092000952100F030F82246942100F02CF8224660
:10093000A12100F028F82246A22100F024F8F007B7
:100940004CBF0C350B35761C0A2EE8DBA624062599
:100950004FF47842952100F013F84FF47842942137
:1009600000F00EF84FF47842A12100F009F84FF49E
:100970007842A22100F004F811346D1EE8D173BD55
:10098000A0B2F7F747BDA8B2F7F744BDFC2219465D
:100990009520F7F7BDBE0000FEB52DED048BDFF806
:1009A000244686B0D4F8F30500EE100A01200BF0BF
:1009B000DDFAF3EE040A94F8EB0320EE200ABCEE15
:1009C000C00A00F02DFB30EE608AB5EE408AF1EEF1
:1009D00010FA98BF9FEDC98ADFF8EC6596ED010A21
:1009E000002000F0F4F896ED010AB4EE480AF1EEAA
:1009F00010FA05D586ED018AF9F732FFB0601DE0E7
:100A0000B068F9F730FFB0F57A7F17D99FEDBC0ACF
:100A100028EE000A00F001F9054670680F4607F05D
:100A2000EBF94FF0E242DFF8A43507F075FB2A46F8
:100A30003B4609F0CBFA08F041FF7060B0EE480A7F
:100A400000F089F84FF6FF77384696ED010A00F07E
:100A5000BEF896ED018A04F2EB30407800EE100A01
:100A6000F8EE408A18EE900A07F0C6F90022DFF887
:100A7000603507F051FB41EC190B18EE100A07F036
:100A8000BBF953EC192B0BF033FB16D2B3EE020A71
:100A900088EE800A88EE008ABCEEC80A10EE102AA2
:100AA0000FF28C5102A8F9F7FBFEBDEEC80A10EE5A
:100AB000100AC0B20A2837DB31E009F0C7F9B2EEFC
:100AC000080A044688EE800A0D4600F0A6F80246A1
:100AD0000B462046294607F0B7F908F0EFFE07F06D
:100AE0008BF900F069FA41EC180B07F0FFFA0FF2EE
:100AF0004851024602A8F9F7D3FE53EC182B002008
:100B0000DFF8D01409F062FADFF8CC34002207F0E5
:100B10009BF907F0D5FA0930C0B2092801DA09209B
:100B200002E01028A8BF0F20307002A80BF0F8FADE
:100B3000042824BF00208DF80C00002001900097AD
:100B400002AADFF8983400219120F7F7DCFC06B008
:100B5000BDEC048BF7BD70B582B000F05EF800F01C
:100B600067F800F05EF822462B4607F0D5FA07F04A
:100B7000A7FAD128A8BFD02002DA002848BF012058
:100B8000DFF83C44206025686068A84210DA002540
:100B9000DFF84C64206800F12C016068334605F1F1
:100BA00099022C3000F051F86D1C052DF2DB0BE0A2
:100BB0000021009100F12C0205F12C009E2392B23D
:100BC000992180B2F7F7FDFD2068606073BD70B5B4
:100BD000064600F022F800F02BF800F022F822463A
:100BE0002B4607F099FA07F06BFA0446D12CA8BF00
:100BF000D02402DA002C48BF012433469F229821DA
:100C000004F12C00F7F7F7FE334604F12D00BDE8A0
:100C100070409F229821F7F7EEBE10EE100A07F001
:100C2000EBB802460B460020DFF8B81307F00CB90A
:100C30000446E44890F8EC0300EE100AB8EE400ACF
:100C40000D4610EE100A07F0D7B82DE9F04704461C
:100C500082B00D4617461E4600F0ABF9DFF86483FC
:100C600098F87801000654BFA8206820F7F7B6FB73
:100C70004FF4A0731A46B9B2A0B2F7F7DCFBDFF865
:100C800068A310215046F9F7AAFCD84F0121384635
:100C9000F9F7A5FC00F087F910215046F9F79DFC03
:100CA00013E004F13C0080B2FF28C8BFFF2036F8F3
:100CB0001000ADF8000048469DF80110F9F7C4FC9B
:100CC0009DF8001000F072F9641CA542E9DA0121D8
:100CD0003846F9F782FC00F06CF998F878010006C4
:100CE00054BFA8206820BDE8F647F7F777BBC04897
:100CF00000218160C1600160416070470000000018
:100D00008FC2F53C2DE9F04FBA48B94E006883B068
:100D10007061B9480068306196ED050AB748D0EDBA
:100D2000000AB8EE400A20EE200AFFF776FF00F036
:100D300043F941EC100B53EC102B07F0EDF90022B6
:100D4000AF4B07F081F808F0B9FD306096ED000A6E
:100D5000B5EE400AF1EE10FA44BF0020306096ED87
:100D6000000AD6ED010AB4EE600AF1EE10FA16D5CB
:100D7000706807F041F8A34AA34B07F0CDF9044689
:100D800030680D4607F038F8A04AA14B07F0C4F9C7
:100D900022462B4609F01AF908F090FD30603068C1
:100DA0009C4D70607069332820D330697169884226
:100DB00016D270693169081800EE100A706931693D
:100DC000401A00F02DF980EE200AF2EE040A20EE1F
:100DD000200ABDEEC00A10EE100AB0F57A7F06DBDD
:100DE0000FF25C212846F9F75BFD0AE001200A2199
:100DF00090FBF1F201FB12030FF250212846F9F7A4
:100E00004FFD002001904FF6FF74744F00943B4655
:100E10002A4600213C20F7F776FB306806F0ECFF0D
:100E200002460B460FF230212846F9F739FD002023
:100E3000019000943B462A4690213C20F7F763FB43
:100E4000B06871694FF4FC65884207D20095B068BC
:100E50004FEA101870694FEA101B07E0002000905D
:100E6000B0684FEA101B70694FEA1018ABEB08002E
:100E700000EB800001907069B06000F09AF8DFF834
:100E800044A100F08CF854BFA8206820F7F7A6FA18
:100E900004EB0B02272392B223211FFA88F0F7F705
:100EA000CAFADFF844B110215846F9F798FBDFF889
:100EB0003C8101214046F9F792FB00F074F81021C3
:100EC0005846F9F78AFB002708E09DF8011000F06A
:100ED0006DF89DF8001000F069F87F1C0198B84289
:100EE000F3DA01214046F9F778FB00F062F800F0F0
:100EF00056F854BFA8206820F7F770FAF0683169F7
:100F0000884205D20095F06807093069050905E0B7
:100F100000200090F068050930690709E81B00EB24
:100F2000800001903069F06000F043F800F037F87D
:100F300054BFA8206820F7F751FA62191D2392B216
:100F40001921B8B2F7F777FA10215846F9F747FB9D
:100F500001214046F9F743FB00F027F810215846DD
:100F6000F9F73BFB002408E09DF8011000F01EF8A3
:100F70009DF8001000F01AF8641C0198A042F3DA02
:100F800001214046F9F729FB00F013F800F007F8BB
:100F900054BFA8206820BDE8FE4FF7F71FBA9AF8A3
:100FA000780100067047DFF870902C214846F9F769
:100FB0004BBB3620F7F7FEB90022184B07F0ACB850
:100FC00090DC01206CC9012060DC01203D0AEF3F6C
:100FD0000000E03F000024C000001940343C002025
:100FE00074CF012000006A40000802400004024063
:100FF00008DC012058DB012054DB01209CDC0120AF
:1010000000004940D7A3703D0AD7EF3F7B14AE479D
:10101000E17A743F2CC901200030014000002440D7
:1010200000EE900AB8EE400AF8EE600A7047000041
:101030005325642020000000532B2564200000006D
:101040005357523D3E313030000000005357523D5F
:101050002532642E25642000503D25312E31662036
:101060000000000000B587B00020FBF7C6FC01219E
:101070002B48FBF7D7FC01200BF06EF80120FBF7A3
:101080005BFC4120FBF7F2FC0028FAD04FF48070A3
:10109000FBF79DFC0120FBF7ADFC0BF0ABF803A8C0
:1010A0000BF084F8002003907F200490FF2005902F
:1010B00003A80BF057F802A900200BF0FEF801A9D5
:1010C00000200BF05AF93A20009000F02DF8FBF7C1
:1010D00008F807B000BD3EB5124C2068F9F7C3FB15
:1010E000B0F57A7F1AD320783A25C00748BF20256B
:1010F00002A900200BF0E1F801A900200BF03DF956
:1011000000F012F80095FAF7ECFFF9F7A9FB202D93
:1011100006BF4008400040F00100206037BD0000DD
:1011200000000410B8DC01209DF809309DF808206B
:101130009DF805109DF806007047000030B583B09B
:1011400001F0B6F801F02CF801210820FBF758FC5B
:1011500001208DF8040000208DF806004FF4807007
:10116000009001208DF807008DF8050000A9D64CED
:101170002046F9F7EDF900F04DF800A92046F9F7FF
:10118000E7F900F047F8D14CD14D04F11400A0600C
:1011900004F580401430E060B5F87101B0F5006FDF
:1011A00008BFCC4811D0B0F5806F08BFCA480CD03A
:1011B000B0F5007F08BFC94807D0B0F5807F08BFF1
:1011C000C74802D0802801D1C648606009F0F4FD0C
:1011D00005F2FB100BF016F9C349FF200870C34954
:1011E000087095F87001C00747BF05210120032151
:1011F00002200CF037FD012085F8F80500F0D4FD41
:1012000000F0F6F895F8F10500F00AF895F8F10508
:10121000207037BD01224FF480712046F9F7E1B903
:101220002DE9F04F85B0AA4CA84DDFF8C492A64E28
:10123000B04FDFF8C48204F2F041039109F5804A0F
:1012400004F57C71029105F510411431019105F509
:10125000004114310091002805F5804101F1140B83
:1012600053D001224FF400714046F9F7BAF9B4F8AF
:10127000AA010AF0B8F900F093FF00F0ACF800F012
:10128000A4F800F09CF800F089F800F081F800F074
:1012900079F805F588304FF480420021143007F0CA
:1012A0000CF800F081F8039800F07FF80020387007
:1012B0000CF0FAFE94F86B0118B104F500700BF015
:1012C000A1F800F05AF894F8670100F00C00082823
:1012D0000CBF0020A86800F086FF94F86701C007E3
:1012E00007D42078001990F8A300022818BF03281B
:1012F00004D100F042F8002000F036FF012200F097
:1013000059F800224FF4807131E07C4800210170CF
:10131000002200F04FF800F065F8B4F8A8010AF0D8
:1013200062F900F0C5FF00F03BFF00F054F800F058
:101330004CF800F044F800F031F800F029F800F023
:1013400021F800F031F8039800F02FF894F86C01C0
:1013500018B104F2FB100BF055F80020387000F0C3
:101360000CF8A86800F000FF00224FF4007140461E
:1013700005B0BDE8F04FF9F734B9B4F87101E96888
:101380008200704701984FF40042002106F095BF9B
:1013900000984FF48052002106F08FBF4FF40052A6
:1013A0000021504606F089BF02984FF48072002158
:1013B00006F083BF4FF480613046F9F712B94FF45D
:1013C00080420021484606F078BF4FF48042002159
:1013D000584606F072BF4FF48042002105F1140018
:1013E00006F06BBF01224FF480714046F9F7F9B85F
:1013F0001FB51D208DF8000002208DF8010000208F
:101400008DF8020001208DF8030000A8F9F77BFA9F
:1014100001210220FBF706FB40F2E73002906C202E
:10142000ADF804000020ADF80C00ADF8060001A9ED
:10143000334C204608F02EF90121204608F0AEF981
:1014400001220121204608F0A1F90121204608F0DF
:1014500052F91FBD2DE9F041294C0121204608F029
:101460009EF900282ED01A48184D90F8F1052978D9
:101470006870814203D0FFF7D3FE687828701D4E54
:101480003078C8B1F9F7E2F9DFF83C8007466878B0
:1014900028B10022FFF7A7FF0CF09CFE04E0002219
:1014A000FFF7A1FF0EF024F93846F9F7D2F92861C9
:1014B000FFF798FF002030702046BDE8F041012181
:1014C00008F077B9BDE8F081000C02405C3C0020D8
:1014D0006CC90120745E0308645E0308545E03084F
:1014E000445E0308345E0308583C0020593C002049
:1014F0000404001046DC012000080240ACDB01209F
:101500000004004010B586B001211020FBF778FAE6
:1015100001214FF48040FBF78EFA00208DF808007F
:1015200001208DF80A000C2000F033F801A9C34C0B
:101530002046F9F70DF80321042008F03FF90820B0
:1015400000F02EF8082000F01FF8092000F030F815
:1015500000208DF8080001A901208DF80A007020F4
:1015600000F017F82046F8F7F3FF0421042008F0F4
:1015700025F9102000F014F80C2000F005F80A20DE
:1015800000F016F806B010BD8DF8110003A808F0A1
:1015900029B9019001208DF80B008DF809007047E2
:1015A000039001208DF8120000208DF81000704784
:1015B0008DF8000000208DF801008DF80200012058
:1015C0008DF8030000A8F9F79EB92DE9F04110202D
:1015D00008F041F9002800F0AC80F9F741F998498A
:1015E000984D086095F8790100F0BF0085F8790101
:1015F00095F87A01F9F71EFCDFF84C82934E944F70
:101600008E484FF47A742021F8F7E0FF01283878EB
:101610002ED178B17079002838D1D6F80100017840
:10162000491C0170D6F801003278017891422DD121
:1016300000212AE0297805EB4100B0F86D20130461
:101640000ED553044EBF42F440419104890C0A3137
:1016500009B242F20773994230DB42F206712DE083
:1016600000F069F814BF02F57A7101F57A7150E063
:1016700088B1707950B9D6F80100017809B931788C
:101680000170D6F801000178491E0170387840F0E9
:101690008000387042E0297805EB4100B0F86D20F9
:1016A000130431D553044EBF42F440419104890CD8
:1016B0000A3909B2674B9942B8BF194602F4004291
:1016C000A0F86D208B04287805EB4000B0F86D2061
:1016D00052EA9342A0F86D20080408D5287805EB5B
:1016E0004000B0F86D1041F48041A0F86D1095F8FD
:1016F0008B01032804BF4046FDF778FA564801786D
:1017000041F00101017009E000F015F804D1A1F5E4
:101710007A71C0F8011001E0C0F801204F48FDF7D0
:1017200065FA4F48012101701020BDE8F04108F032
:101730009DB8BDE8F08105EB81002246D0F801108C
:10174000B1FBF2F262438B1A704738B5082008F0FB
:1017500082F8002870D0F9F783F83949394C0860CD
:1017600094F8790100F0BF0084F8790194F87A01C7
:10177000F9F760FB94F8F915304859B10421F8F7EE
:1017800025FF0128D4F8FA050CBF401C401EC4F800
:10179000FA054CE094F86711490648D494F9A4116D
:1017A000F022114228D0C1F303150421F8F70EFFEF
:1017B0000128D4F8FA050CBF401C401EB4F8FE15F1
:1017C000C4F8FA05D4F8FA25207804EB8000954295
:1017D00008DAD0F801208918C0F801100020C4F8F8
:1017E000FA0515E0002A13D5D0F80120511AC0F8E7
:1017F0000110C4F8FA550BE00421F8F7E7FE0128C0
:1018000000F030F80CBF11FA82F1891AC0F801100B
:1018100000F028F8B1FBF2F35343C91A18BFC0F81F
:1018200001300E48FDF7E2F90D4801210170082052
:10183000BDE8324008F01AB831BD00000010024087
:10184000D83100206CC9012009AC010834DC01202A
:10185000CA310020FAD8FFFFC9310020BFEB0008D1
:10186000F5DC01202078B4F8FE2504EB8000D0F8E8
:1018700001107047B5EE400AF1EE10FA02D5BFEE46
:10188000000A7047B5EE400AF1EE10FA02DDB7EE3D
:10189000000A70479FED9E0A704710B5954C2021B5
:1018A000201D08F079FF4FF07E5020620220606218
:1018B00000202070A062607010BD00002DE9FC4186
:1018C0008C4D2DED088B88460446696AA86A02296A
:1018D00008BF401C332824BF00206862A86200278C
:1018E00024E004EBC70600F025F9306895ED011AF5
:1018F00000EE900A00EE201A85ED011A00F01AF9A8
:10190000706895ED021A00EE900A00EE201A85ED3F
:10191000021A306800F00FF9306895ED031A00EEF6
:10192000900A00EE201A85ED031A7F1C4745D8D394
:101930002878401C2870C0B20828C0F2B18000EEA0
:10194000108AF8EE40AA95ED010AB4EE00BA80EED6
:101950002A0A20EE0B0A9FED688B00F0E7F8684A30
:10196000684B06F0D9FB064628690F4606F044FA94
:1019700000F0D8F800F0D2F807F0A0FF95ED020AC9
:1019800080EE2A0A0AEE100A20EE0B0A85ED01AA63
:101990009FED5D9B00F0CAF853EC192B06F0BCFBE1
:1019A000064668690F4606F027FA00F0BBF800F01B
:1019B000B5F807F083FF95ED030A80EE2A0A0BEED7
:1019C000900A20EE0B0AC5ED02BA00F0AFF853EC16
:1019D000192B06F0A1FB0646A8690F4606F00CFA83
:1019E00000F0A0F800F09AF807F068FF00EE900A07
:1019F000F5EE40BAC5ED030AF1EE10FA14BF8AEE17
:101A00002B0A9FED430A85ED070A2BEEAB0AB5EED4
:101A1000400AF1EE10FA05DD60EEA00A4AEE4A0A2D
:101A200080EE800AB5EE400AF1EE10FA02DD0FF00A
:101A300087FB01E0B7EE000A85ED080A95ED030A81
:101A4000B5EE400AF1EE10FA1FD0686AE8B9D5ED9C
:101A5000010A80EE800A0FF081FBDFED2E0AB4EE62
:101A6000600AF1EE10FA06DADFED2B0AB4EE600A36
:101A7000F1EE10FA07D56878052804DA0221401C37
:101A80006962687001E00120686268682861A8687E
:101A90006861E868A86100206860A860E860287054
:101AA00000200FE004EBC001401C0A6800EE102A81
:101AB0004A6895ED071A00EE902A01EE200A10EE12
:101AC000102A0A604045EDD300200CE004EBC00171
:101AD000401C4A68D5ED080A00EE102A20EE200AC4
:101AE00010EE102A4A604045F0D3BDEC088BBDE8EB
:101AF000F3810000303B00208195438B6CE7EF3F82
:101B0000FA7E6ABC749368BFFA7E6ABC7493683FBD
:101B100000000000DB0FC93EDA0FC9BE32463B466B
:101B200008F054BA53EC182B06F0F6BA10EE100A6F
:101B300006F062B9706800EE100A9BE62DE9F041EC
:101B4000069D0446884616461F460FF037FB204682
:101B50000FF068FCC4F8E475414604F2E4572046EF
:101B60007D60BE600FF079FB786800688047204692
:101B7000BDE8F0410FF04EBB80B50FF053FC0020E4
:101B800002BD1CB5044600A90FF0EFFD9DF8000052
:101B900010F01F0003D002280BD005D30EE000A9DF
:101BA00020460FF047FC10E000A920460FF0EEFCA5
:101BB0000BE000A920460FF002FD06E09DF80000B2
:101BC00000F0800120460FF0EDFB002016BD10B59F
:101BD000044604F2111041BB94F8112104F55D7123
:101BE000032A2CD1CB698A689A4210D2981AC8610C
:101BF000E378012B02D1CB68D318CB60904238BF79
